:020000040800F2
:10000000002000104DC50208B14B0208F906010896
:10001000AD4B0208A94B0208A54B020800000000E6
:10002000000000000000000000000000A14B0208DA
:100030009D4B020800000000994B020811B6000811
:10004000B5C50208B5C50208B5C50208B5C50208A0
:10005000B5C50208B5C5020879C00008A5C10008E9
:1000600069C100082DC10008F1C00008692400081A
:1000700059240008492400083924000829240008CC
:100080001524000801240008B5C50208B5C50208FA
:10009000C94F0208B5C50208B5C50208B5C00008B9
:1000A00099AC0008E9AC0008B5C50208F9AC000835
:1000B000D9AC0008C9AC0008B5C50208B5C502082E
:1000C000B5C50208B5C50208B5C50208B5C5020820
:1000D000B5C50208B5C50208B5C5020845B6000891
:1000E0003DC00008B5C50208EDAA0208B5C5020862
:1000F000A9AC0008B5C50208B9AC0008B5C502082E
:10010000000000000000000000000000B5C502086B
:10011000B5C50208B5C50208812D0108652D010885
:10012000ED230008D9230008C5230008B1230008E7
:100130009D230008B5C50208000000000000000073
:10014000B5C50208B5C50208B5C502080000000023
:10015000000000000000000000000000000000009F
:100160000000000000000000B5C50208B5C5020887
:10017000B5C50208000000000000000000000000FB
:0801800000000000B5C50208F3
:10018800002870B51EDB0928044620DD012303EB97
:1001980083035B00B0FBF3F2092AF8D87BB10E4E5B
:1001A800B4FBF3F00928CCBF57223022A6FB03E5A5
:1001B800024403FB1044EB0801F8012BF0D10023A3
:1001C8000B7070BD2D230B7040420131DBE73030DE
:1001D80001F8010BF3E700BFCDCCCCCC884230B49A
:1001E8004FF001042ED301FB04F4B0FBF4F58D426B
:1001F800F9D284B1AAB901E0B0FBF4F5092DCCBF5E
:10020800572230222A4404FB150003F8012BB4FBC3
:10021800F1F4002CF0D100221A7030BC7047B0FB0A
:10022800F4F5092DCCBF372230222A4404FB1500EF
:1002380003F8012BB4FBF1F4002CF0D100221A7062
:1002480030BC70470546002AEBD1D7E703685A1C33
:1002580002601970704700BF2DE9F047089C2578A7
:10026800002B804689460CBF4FF0200A4FF0300A19
:10027800661C35B3002A29DD334601E0024698B1F1
:1002880013F8011B501E0029F8D1971E60B13D4696
:10029800013D51464046C8476B1C002BF8DC2578C9
:1002A80027EAE770013055B1041B29464046C84784
:1002B800301916F8015B002DF7D1BDE8F087BDE8CD
:1002C800F087002A04DC2846BDE8F0870020EBE729
:1002D800571EDCE783684268D0ED037A00EB8301A0
:1002E8000133934281ED040A836004BF00238360D5
:1002F80000EB830393ED047A036870EE277A9A4241
:10030800C0ED037A77EEC77AC0ED037A0CDA0133D1
:1003180007EE103AF8EEC76AB7EE007A87EEA60A3B
:10032800036030EE070A704707EE102AB8EEC77A66
:1003380087EE870A704700BF90ED057A90ED004A76
:10034800D0ED066AD0ED014AD0ED047A90ED035A5B
:10035800D0ED025AA4EE007AB0EE406AB0EE470A39
:10036800B0EE667AA6EE247A67EEC07AA0EE457AF9
:10037800E6EE257A80ED057AC0ED067A704700BF73
:10038800D0ED057A90ED013AD0ED003AD0ED064A6D
:1003980090ED024A90ED077A90ED035A90ED086AC5
:1003A800D0ED045AC0ED067AF0EE406A27EE830AD3
:1003B800C0ED056AA3EEA60A80ED087AA4EE240A29
:1003C800A5EE470AA5EEC60A80ED070A704700BFEA
:1003D800D0ED007A90ED017A30EE670AE7EE007A08
:1003E800B0EE670AC0ED007A704700BF704700BFE3
:1003F8000A44914214D030B40139551E41F2210209
:1004080011F8014F082380EA042004044CBF82EA53
:1004180040004000013B80B2F7D18D42F0D130BCA2
:10042800704700BFE0B1D9B1F0B50E4B1B7800247E
:100438000A2B0CBF4FF00A0E4FF0080E2346022776
:10044800012617FB036511F813204D5D0133DBB25C
:1004580042EA0522734520F814201C46F1D3F0BD6A
:10046800704700BF000000202DE9F04FDFF81CB2F4
:10047800DFF81CE2BBF80020DEF80060BBF90430AE
:10048800BBF90250BBF90A80C2EB261404FB04F442
:1004980024135200C2EBE60203FB04F305FB02F24D
:1004A8009B1303EBE223B3F5FA364FEAE37589B001
:1004B80045F1FF373246A6FB0645CDE9024502FB6A
:1004C80007F205EB4202CDE90467029EBBF908403A
:1004D800039208FB02FC4FEAE87906FB09CC3A468E
:1004E800A8FB0689049ECBF81830E51704FB02F236
:1004F80006FB0522A4FB0667E14417444FEA1822CD
:1005080042EA096200924FEA292201923D03DDE99D
:100518000078340345EA16553F19BBF80660069083
:1005280048EB05083C1C48F5004503EB8302A4FB97
:10053800068906FB0599803213124FEA69064FEACD
:10054800E977079356EA07038A4600F09280DDE9C7
:100558000489BBF90E20DEF80440BBF910004946B7
:10056800C4F5801ED317DDE9024502FB01F108FB43
:100578000311A2FB08230B444FEA43492B46C1173A
:1005880000FB03F304FB0133A0FB0401BBF90C409F
:100598001944E30001937346DC170023009349EAEA
:1005A800D2394FEA4248DDE9002310EB080041EB5D
:1005B8000901E50712184FEACE744B4145EA5E057A
:1005C800A41A65EB0305221945EB050312196B41C3
:1005D80099019001801841EA926159418B0082008B
:1005E80043EA9073101943EB05018B00820043EA3C
:1005F800907310460019194632463B4669412BF064
:10060800CDFDBBF916204C13450B45EAC14502FB4D
:1006180004F6D31705FB0366A2FB05233344BBF995
:10062800146002FB04F405FB034406FB01FEA2FB75
:100638000523F717234400FB07EE540EA6FB0067BB
:10064800774444EAC3144FEAD64800194FEA636571
:1006580048EA473869414FEAE74918EB0008BBF90F
:10066800124049EB01094FEA182646EA09662001BB
:100678003618069B0BB1360A1E60BAF1000F02D07D
:10068800079BCAF8003009B0BDE8F08F7C4800200D
:10069800CC1E0020704700BF704700BF50F8043CD4
:1006A800012280F84520103803B11847704700BF71
:1006B80090F8203033B1012B03D14FF400638382CB
:1006C800704770474FF480638382704770B5044663
:1006D80082B01430E56D06236A464321A847B0B1BD
:1006E8009DF804009DF800609DF801109DF80250E7
:1006F8009DF803209DF8053041EA062143EA0023CE
:1007080042EA0522A187E287A4F84030012002B01E
:1007180070BD00BF70B5044682B00830656A062314
:100728006A463B21A847A8B19DF804009DF80060DF
:100738009DF801109DF802509DF803209DF80530A2
:1007480041EA062143EA002342EA0522E1822283A4
:100758006383012002B070BD70B40468037B226813
:10076800022101FA03F31A4213D042690A495C20B4
:1007780000FB02124FF6FE7650685289C568006881
:10078800296831402960C168D24392B20A40C260E8
:10079800636070BC704700BF9849002030B40A4BB2
:1007A8001D7875B1094B002003EBC5051A689988B7
:1007B8005062D4682143D160083323F8040CAB425B
:1007C800F4D130BC704700BF784C00207C4C00202E
:1007D80010B40268047B11680223A340194209D0AF
:1007E8000649406800240C7001684FF6FE742140E9
:1007F800016053605DF8044B704700BF3B3D00202B
:10080800F0B4334C00EB800004EB80046468002CE7
:100818005BD0304E49004FF42040CDB2B060A169A2
:10082800090444D460682C4F45F08071384041F485
:10083800903101434FF420406160B06003E0411EF5
:10084800002838D00846A1698F07F8D54FF4204012
:10085800A262B06002E0421E68B31046A2691106A7
:10086800F9D562681C4945F0007545F480350A40A1
:1008780015434FF420406560B06002E0421ED0B1DD
:100888001046A2699207F9D5A362A3694FF42040E4
:100898009B06B06005D4431E68B11846A3699B0641
:1008A800F9D52023B060E3610120F0BC7047411EF8
:1008B80008B10846B3E7094A138801339BB24FF0E1
:1008C800FF31B1601380F0BC70472046F0BC704720
:1008D8009C2B0020CC1E0020009800FC482C0020F7
:1008E800134600200A4668218AE726221921027049
:1008F800272200238270417001221A21027183711C
:10090800C1704271C37170472DE9F341056906460C
:100918000F467DBBD0F80080C8F30A0323B3002339
:10092800D6F80080019327F00BFF042819D1224C38
:10093800236943F001032361BBB2A8F8003027F014
:10094800FFFE04282ED108F102030193019B3F0CFE
:100958001F8027F0F5FE2369042823F00103236193
:1009680025D06FF0010505E027F0EAFE042805D040
:100978004FF0FF35284602B0BDE8F0810E4C2369E0
:1009880043F002032361C4F81480236943F0400351
:10099800236127F0D5FE2369042823F0020323618D
:1009A800BDD0E5E7236923F001032361D9E7336864
:1009B80004333360DEE700BF00200240F8B5044688
:1009C8000D468E180027B54201D12069F8BDE368AD
:1009D800591CE160234415F8012B1A720429F2D13D
:1009E800A1682046FFF790FFE7602061EBE700BFB2
:1009F800014B18680AF0C0BEB4520020F8B55D205B
:100A080027F01CFE1049114A8C89CB89104D0E190C
:100A18000134377C3074DB1B184400B282FB00239E
:100A2800C217C2EBE302323292B2A2EB8203DB00BE
:100A380003F6E8031BB204F00F0483F30A038C8166
:100A4800C8810A842B80F8BDCC1E0020ABAAAA2A34
:100A5800603D002008B5064B18680BF0E1FA30B18C
:100A68000AF08EFC034B0122586283F8282008BD47
:100A7800545B0020CC1E002027F04ABD70B5044608
:100A880090F85900002833D104F11405236E802210
:100A98006B212846984764200AF018FD236E2846E3
:100AA80003226B219847236E94F854201921284675
:100AB80098470F200AF00AFD236E94F85220284622
:100AC8001A219847236E284618221B219847236E1F
:100AD800284618221C219847236E284602223721CF
:100AE80098472846236E01223821BDE870401847F0
:100AF8000AF0A8F8054618B1202200238271C371B4
:100B0800284600210BF0A0F82146054B41F8103F7C
:100B1800284627F06FFC284601210BF05DFBB3E760
:100B2800A506000810B490E80600047B406902237B
:100B3800A3404B6013685DF8044B4FF6FE710B4001
:100B480013600AF0B9BD00BFF8B505015A4C5B4BFC
:100B5800625961199A4204EB050704BF01230B731C
:100B68000646387A26F074FD3B7A03F01F015B09CC
:100B78000122022B02FA01F278D0032B71D0012B4B
:100B880067D06319013618790AF05CF8F6B207469F
:100B980010B11223C6718371631958790AF052F89B
:100BA80010B11323C6718371631998790AF04AF852
:100BB80010B11423C671837166190E21F279384673
:100BC80009F0A0FC70790AF03DF8F2790E2109F0DD
:100BD80099FCB0790AF036F8F2790E2109F092FC06
:100BE8006359364A934251D0354A934259D0354ACF
:100BF800934240D02C44227B002A2FD1012002248A
:100C08009A8822F480521204120C9A80998889B228
:100C180041F4805199801A8802F4415242F4457295
:100C2800024322431A809A8822F470621204120C3A
:100C380042F4E0629A809A8B22F400621204120C49
:100C480007219A8319821A8892B242F040021A80C8
:100C5800F8BD1D4B996A0A439A6292E70020044640
:100C6800CEE7194B19690A431A618AE7164BD96806
:100C78000A43DA6085E702F5EA32116941F4004176
:100C88001161116921F400411161B3E702F5604275
:100C9800D16841F48051D160D16821F48051D1608C
:100CA800A8E702F5EC32116941F48041116111693C
:100CB80021F4804111619DE7F45900200030014082
:100CC80000380040003C004000100240427A02B95F
:100CD800704710B504460368406804F10A01984754
:100CE8000023637210BD00BF437A5A1C0344D2B27A
:100CF80042729972037A934200D802B9704710B5CC
:100D080004460368406804F10A01984700236372A7
:100D180010BD00BF10B40B49002301E0272B0CD0F5
:100D280011F8132082424FEA430403F10103F5D17D
:100D380021445DF8044B4878704700205DF8044B67
:100D4800704700BFFCDA020870B5448806460D46B5
:100D5800C4F30B042246002128462CF016FE336902
:100D6800094A934209D3094A934206D222462846A1
:100D78001946BDE870402BF01FBD23B12146284617
:100D8800BDE87040184770BD283603081A370308B5
:100D9800064B07498B4202D30023184670471A882E
:100DA800C2F30B029042F8D01433F3E7F031030892
:100DB80028360308024A136823EA000010607047C7
:100DC80004370020F8B5174D2B78A52B28D16B7860
:100DD800BE2B25D1022229464FF6FF70FFF708FBEC
:100DE800114FAC1C22884AB1A618BE4218D2052A57
:100DF80016D92146FFF7FCFA3446F3E721460222CA
:100E0800FFF7F6FA0222A118FFF7F2FA0634074BA9
:100E1800641B1C8041F60F53C31A58425841F8BD51
:100E28000020F8BD00F00308000004084A2C002048
:100E38002DE9F04FDFF848914C4F8BB00326A7EB14
:100E480009071822002104A82CF09FFD484BCDF873
:100E5800109005971A69120604D5464A5A6002F19D
:100E680088325A6001228DF824203422DA60424BFD
:100E7800424C1B88ADF800300222694604A8FFF7EF
:100E88009DFD022269464FF6FF70FFF7B1FADFF8C1
:100E9800F4A080464FF0000B544536D30AAC002529
:100EA80024F8245D0222214604A8FFF787FD0222C8
:100EB80021464046FFF79CFA40BAC043ADF8080007
:100EC800022202A904A8FFF779FD079860B106ABD2
:100ED800C0F10402294618442CF057FD069904A8CD
:100EE800FFF712FD079508909DF82430089A23B162
:100EF8001F490B6943F080030B61013E2DD0002A86
:100F08009FD1FFF75FFF50B32CE065888DF80DB0D7
:100F1800C5F30B05AB1DADF808302388C3F30B02EE
:100F2800ADF80A201B0B062202A904A88DF80C3084
:100F3800FFF744FD062202A94046FFF759FA616807
:100F480080462A4604A8FFF739FD616840462A46CC
:100F5800FFF74EFA143480469EE7002AD1D00520C8
:100F680009F0B0FF0BB0BDE8F08F00BF0000040827
:100F780000200240230167454ADB0208F0310308DC
:100F880000F00308283603080378202B024600F1F6
:100F98000100F9D0092BF7D02D2B2CD02B2B03BF18
:100FA8005378B7EE000A0246B7EE000AA3F1300103
:100FB800C8B209289FED467A10D8F2EE046A07EE07
:100FC800901AF8EEE77A12F8013FE7EE267AA3F1D5
:100FD8003001C8B20928B0EE677AF0D92E2B4CD070
:100FE80003F0DF03452B0BD0F7EE007A67EE276A94
:100FF80020EE260A70475378BFEE000A0246D5E76E
:1010080010B451782D2959D02B290ABF9178501C3A
:10101800901C0024A1F13003092B53D8002303EBC3
:10102800830301EB430310F8011FA1F13002092AE1
:10103800A3F13003F3D9B3F59A7F28BF4FF49A731D
:10104800072B42D9DFED236A1A46F7EE007A083AF1
:10105800072A67EEA67AFAD803F007032BB1F2EE57
:10106800046A013B67EEA67AFBD124B3C7EE276A70
:101078005DF8044B20EE260A70475378A3F130013F
:10108800C8B2092802F10102AAD8F2EE046AF0EE09
:10109800665A07EE901AF8EEE77A12F8013F87EEE3
:1010A800A66AA3F13001C8B2092866EEA56A37EE30
:1010B800067AEED994E767EE276AD9E7901C91780B
:1010C8000124A7E7F7EE007ACFE7F7EE007AC5E745
:1010D8000000000020BCBE4CB5EEC00ADFED317A3E
:1010E800F1EE10FACCBF30EE270A30EE670ADFEDDA
:1010F8002E7A20EE270A30B5FDEEC07A87B017EEBB
:10110800904A054684EAE470002303A9A0EBE47042
:1011180001930093029321F041FB002CACBF2023E4
:101128002D2303A88DF800302AF08EFB012803A98F
:1011380024D002282DD0032805BF302368466846EE
:101148008DF801302CF047FC68462AF07DFB033807
:10115800C4B22246694628462CF09BFC00232B5536
:1011680028462AF071FB2E22431C2A540DEB040159
:10117800E8182CF04DFC284607B030BD30236846EF
:101188008DF801308DF802308DF803302CF023FCF7
:10119800DAE7302368468DF801308DF802302CF0FC
:1011A8001AFCD1E76F12033A00007A442DE9F041A6
:1011B800064615460846B6FBF2F43CB905FB14642E
:1011C800124B1B5D00F8013BBDE8F081B4FBF2F760
:1011D80067B90E4B05FB174705FB1464DA5D00F889
:1011E800012B1B5D00F8013BBDE8F081B7FBF2F86D
:1011F800B8F1000F02D04046FFF7D8FF05FB18787A
:10120800024B13F8082000F8012BE3E72403030836
:1012180030B402681146531C036011F8024B016098
:10122800D31C517803609378151D05601B0443EAAD
:101238000123D078234343EA006030BC704700BFE5
:101248000368591C1A46016012F8021B026058789C
:1012580041EA0020704700BF03685A1C02601878F2
:10126800704700BF38B50446006815462BF0A4FA4D
:1012780022682A44226038BD036810B40A0A5C1C3C
:1012880004601A7003685A1C026019705DF8044BF8
:10129800704700BF03685A1C026010B419700368D5
:1012A8000A0A5C1C04601A7003680A0C5C1C04605F
:1012B8001A700368090E5A1C026019705DF8044B15
:1012C800704700BF03685A1C026019700368090A56
:1012D8005A1C0260197070472DE9F047002488B045
:1012E80080460F461E46A14605AD531C0393117850
:1012F80039B3252933D1931CCDF810900393507836
:1013080030284ED04FF0000AA0F13003DBB2092B91
:1013180042D96C2819D0642800F0938024D8252855
:101328001CD063D9582876D063281BD13178404621
:10133800B847039A531C03931178043601340029E3
:10134800D7D1204608B0BDE8F087039B5A1C03920A
:101358001B78642B7CD02AD8252B54D125214046D4
:101368000134B847039AC0E7732833D044D97528A5
:101378004FD106F1040E30682B4600220A2176462A
:10138800FEF72CFF049A0095534639464046FEF76F
:1013980063FF039A0444A8E704AA03A921F0DAF931
:1013A800B7E7D31C039390784FF0010AACE7732B8F
:1013B80010D05BD9752B3AD0782B96D1A3F158026F
:1013C800B2FA82F2306852092B4610210436FEF731
:1013D80005FFD7E73368049A00933946002340464F
:1013E800FEF73AFF04360444039A7EE70028B9D191
:1013F800204608B0BDE8F0876E28B3D1039A336859
:1014080004361C6071E72AD9582BD7D0632B8DD0AE
:101418006BE77828A6D1A0F15802B2FA82F23068B8
:1014280052092B461021FEF7D9FE0436AAE706F129
:10143800040E30682B4600220A217646FEF7CEFEBF
:10144800A0E7331D306829461E46FEF799FE99E746
:10145800331D306829461E46FEF792FE92E7002BA0
:101468007FF443AF204608B0BDE8F0876E2BC6D0A6
:101478003BE700BF0EB400B584B005AB019053F84C
:10148800042B0649039301A8FFF726FF019B0022BE
:101498001A7004B05DF804EB03B0704755020008F9
:1014A8000FB430B583B006AB0A490B4853F8042B88
:1014B800096800680193FFF70FFF084C054620688C
:1014C8000AF04EF90028FAD0284603B0BDE83040AB
:1014D80004B070471429002018290020B4520020B5
:1014E800DFED2B7AB4EEE70AF1EE10FA4ADDDFED14
:1014F800296A9FED297A01E0B0EE670AB4EEC70ABF
:10150800F1EE10FA70EE667AF6DC9FED247AF4EECE
:10151800C77AF1EE10FA38D5DFED1E6A9FED207A12
:1015280001E0F0EE407AF4EEC77AF1EE10FA37EE09
:10153800A60AF6D4DFED1B7AB4EEE70AF1EE10FA4C
:1015480014DDDFED137A37EEC00A60EE006A9FED16
:10155800166A9FED167ADFED167AA6EE867A20EEE9
:10156800266AE6EE877AA6EE270A7047DFED117A3B
:10157800B4EEE70AF1EE10FA44BFDFED087A37EE71
:10158800C00AE2E7F0EE407ABFE7B0EE670AD1E7BB
:10159800DB0F4940DB0FC940E4CB1641DB0F49C0E4
:1015A800E4CB16C1DB0FC93F92E741B99730083C3D
:1015B80015A82ABEDB0FC9BF80EAE073A3EBE0736E
:1015C8008B4205DB002801DD401A704702D17047C5
:1015D800002070470844704709B909E0194690FB94
:1015E800F1F301FB13030846002BF7D108467047B7
:1015F8000146FBE707EE901AF8EE677A9FED837ACB
:1016080027EE800A20EE070AFDEEC07A17EE903A20
:101618002033402B00F28C80DFED7D7AB4EEE70AB0
:10162800F1EE10FA40F3E880B0EE407A9FED796A67
:10163800DFED796A01E0B0EE677AB4EEE67AF1EEB2
:1016480010FA77EE467AF6DC9FED747AF4EEC77AF4
:10165800F1EE10FA40F1CD809FED6E6ADFED706A11
:1016680001E0F0EE477AF4EEE67AF1EE10FA37EEA2
:10167800867AF6D4DFED6B7AB4EEE77AF1EE10FAFB
:1016880051DCDFED697AB4EEE77AF1EE10FA44BF87
:10169800DFED627A37EEC77A27EE076ADFED635A25
:1016A800DFED637ADFED636A9FED635AE6EE257A34
:1016B80067EE065AE6EE276AF7EE007AA5EEA67AF6
:1016C800F0EE675AE7EE055AE7EE457A87EEA55A37
:1016D800DFED547A30EE277AFDEEC76A16EE903ABF
:1016E8002033402B29D99FED557AF6EE006AB7EEE4
:1016F800006AF7EE004AC4EEA57A002383614361CD
:101708000362C36180ED045A67EEA66A27EE866A13
:1017180027EE877AC0ED006AC0ED026A80ED016AA3
:1017280080ED037A7047DFED3A7A37EEC77AB3E790
:10173800B7EE005AF0EE455ACAE7B4EEE70AF1EE02
:1017480010FA5FDD9FED336ADFED336A01E0B0EE3A
:10175800677AB4EEE67AF1EE10FA77EE467AF6DCBE
:101768009FED2E7AF4EEC77AF1EE10FA47D59FED89
:10177800296ADFED2B6A01E0F0EE477AF4EEE67AAB
:10178800F1EE10FA37EE867AF6D4DFED267AB4EE6B
:10179800E77AF1EE10FA27DCDFED237AB4EEE77A88
:1017A800F1EE10FA44BFDFED1D7A37EEC77A27EE67
:1017B800076ADFED1E4ADFED1E6ADFED1E7AE6EEF0
:1017C800246A67EE064AE6EE267AB7EE006AA4EEC9
:1017D800A77AF6EE006A36EE476AF8EE007A27EE48
:1017E800277A66EE266A84E7DFED097A37EEC77A4C
:1017F800DDE7B0EE677A3DE7F0EE407A24E7B0EE39
:10180800677AC2E7F0EE477AAAE700BF27D4D23654
:10181800DB0F4940DB0FC940E4CB1641DB0F49C061
:10182800E4CB16C1DB0FC93FDB0FC9BF92E741B953
:101838009730083C15A82ABEF304353F0000008005
:1018480070B406688E4217D90139751E002311F845
:10185800014F0822634013F0800F4FEA430318BF7B
:1018680083F0D503013ADBB2F5D18D42EFD1721C7A
:101878000260337070BC70470023F8E710B44C095D
:10188800012250F8243001F01F0102FA01F10B4344
:1018980040F824305DF8044B704700BF4B0901F055
:1018A8001F0150F82320012303FA01F1114214BF4C
:1018B80018460020704700BFF0B41A4B1B78012B64
:1018C80022D0194B822703F1EA0628215A227825CB
:1018D80055242D201F7059709A70DD7019715A7136
:1018E8009C71D8714E33B342F4D1104B10491C2669
:1018F80021250124002230204E708D701C70D87074
:101908005A709A70F0BC70470A4A0B480B494FF45A
:10191800486640F22E4502241680158284700B70AA
:10192800CFE700BFC4250020B2350020D0420020F8
:101938006C3D00207049002088540020804200201F
:1019480038B500F0EF03C02B094B0A4C054608BF19
:101958000121186818BF00210AF03EFC236AA28CF6
:101968001A85284626F0A6FD236AA28C9A6138BDFE
:10197800545B0020245A00202DE9F8433C4CC37ADC
:1019880094F840203B4E9A423370894604D004F1C3
:101998002C013948FFF7D8F9DFF8FC80C4F84480F7
:1019A80005230025404688F8063088F8075025F0BA
:1019B8006DFE1E2308F8023CA8F10800202108F853
:1019C800015C09F0EBFE33780A2B3BD008232B4F40
:1019D80089F80030776026F077FE07F1100026F0CE
:1019E80041FE27480AF01CFBA8B1E36A9BB1254DCC
:1019F8002365A5F124030FCB85E80F0094F8643024
:101A080003F00F03E118012291F8545084F8643070
:101A180084F84C2002E0002384F84C3029460F203B
:101A28001AF05EFDC020FFF78BFF09F0A9FC726871
:101A3800636F5268E26601330022A066636722671B
:101A4800BDE8F8831048114989F80030104A036846
:101A5800096812680F4D75604B405340A36426F027
:101A680033FE05F1100026F0FDFD0D25B9E700BF96
:101A7800CC1E002000000020F031030890DB020893
:101A8800245B0020201F0020ACF7FF1FB0F7FF1FCA
:101A9800B4F7FF1F4CDB02082C5B002000B370B5C5
:101AA800104E402904464FF0F0000D4628BF40254F
:101AB800FFF746FF336AB28C1A85452026F0FAFCF8
:101AC80055B1013D54FA85F5013CFF2026F0F2FCA2
:101AD80004F8010FAC42F8D1336AB28C9A6170BD38
:101AE800704700BF245A00202DE9F047BA4C94F8FB
:101AF80028308AB0002B40D0814600254020D4F8F9
:101B0800248084F8285026F099FD00F00303022B66
:101B180000F0A78010F0210613D1B04F94F84C5074
:101B28003B780A2B00F03281002D00F0C08015218F
:101B38006846FFF7B3FF9DF80030552B00F0F180A1
:101B48003546C020FFF7FCFE94F87860DEB994F8BB
:101B58004C30A3BB09F014FCD4F88030A04AC01A5A
:101B6800904206D994F854301BB1236D002B40F0F5
:101B78008A8028460AB0BDE8F08794F8786003F0B8
:101B8800FF05002EE3D009F0FBFBE36FC01AB0F5A8
:101B9800FA7FDCD9D4F88430606C5A1C9B07C4F8EF
:101BA800842040F181800AF00BFAD020FFF7C8FEAC
:101BB800002384F8783094F84C30002BCAD0874F33
:101BC80009F0DEFB7E680246D6F800E0D4F888000B
:101BD800652101FB0EF1101A88420CD9616FC4F817
:101BE800882063299ABFC1F1640189B200210023CA
:101BF800A4F87A106367D4F88C10F368511A9942E4
:101C080029D8A06EE16E131A8B42B2D9B3FBFEF647
:101C1800012E98BF4218A020A266FFF791FE94F803
:101C28006430334403F00F03E2180F2092F8541085
:101C380084F864301AF054FCC020FFF781FE236F4B
:101C48007A681F2B19D81268E26601332846236781
:101C58000AB0BDE8F0870123C4F88C2084F87930F5
:101C6800CFE794F84C30002B40F0A880C020FFF755
:101C780067FE002594F8786068E79268594BE26639
:101C880000221A8075E7584EE36206F124030FCB51
:101C9800524D2D7884F84050012586E80F0084F8CD
:101CA8004C500EF057FD64E70AF090F97DE70521E6
:101CB8006846FFF7F3FE9DF80030AA2B7FF441AF8A
:101CC8007868DDF801604068636FE066C6F303106A
:101CD80001304649464A266506F00F0E01330027B3
:101CE8000928C4F8688028BF092001EB0E11636732
:101CF80002F11006276711F8013B1B1A02F8013F91
:101D08009642F8D194F8643003F00F03E2180F20DC
:101D180092F8541084F864301AF0E2FBC4F880801A
:101D28000FE7DDF80120236D9A427FF409AFFEF733
:101D380065FE636F7A68C4F8688052682667013365
:101D4800E2666367B9F1000F0DD00AAB53F8232D93
:101D5800C9F8002059689A68DB68C9F80410C9F8FE
:101D68000820C9F80C3094F86430013303F00F03ED
:101D7800E2180F2092F8541084F864301AF0B0FB7F
:101D880094F84C300225002B95D0DAE695B36846D6
:101D98001D21FFF783FE9DF80030582BEA4671D0CD
:101DA800AA2B6FD0562B6DD0354694F87860002E4C
:101DB8007FF4E9AEC020FFF7C3FDC8E694F86430AD
:101DC800013303F00F03E2180F2092F8541084F83F
:101DD80064301AF085FB49E7CC1E00200000002083
:101DE800400D0300603D0020FC1E0020D4DB0208EB
:101DF8001F1F002068461B21FFF750FE9DF800308A
:101E0800AA2BEA463ED039D9BB3B012B34D8636FA5
:101E180079689DF80B204968E1660133FF2AC4F808
:101E28006880256763675AD00AAD04F1540655F8EF
:101E38001D0D6968AA68EB680FC64FF0FF33A16CE7
:101E4800DDF80160CDF80510CDF80B300122E02057
:101E58006B60AB60EB602B616B612B8384F878203F
:101E6800C4F88080C4F87C802665FFF769FD514678
:101E7800252205201AF018FB002596E7562B01D0DD
:101E8800582BF9D1DDF80520A36C9A42F4D1DDF87E
:101E98000120236D9A42EFD1FEF7B0FD636F796898
:101EA8009DF800204968C4F8688001330025582A45
:101EB800E1666367256715D094F87860002E7FF493
:101EC80062AE94F86430013303F00F03E2180F2078
:101ED80092F8541084F864301AF002FB65E70DF1AB
:101EE8000B05AAE7B9F1000F10D00AAB53F81F2D64
:101EF800C9F800205A689868C9F80420D9681A698E
:101F0800C9F80800C9F80C10C9F8102094F87960CD
:101F18000EB90225D0E7284B218C1B88B4F87A200B
:101F280097F808908DF80F1003EB83035B009BB2C2
:101F38008DF80B301B0A080AB9F1400F4FEA12213D
:101F48008DF80C304FF0FF334FF0000528BF4FF0ED
:101F580040098DF813208DF81000FC228DF814101C
:101F6800CDF81930AA21CDF81530CDF81D30CDF8AF
:101F78002130E020FE238DF811308DF800108DF807
:101F880009508DF80A508DF80E508DF812508DF8C2
:101F98000D20FFF7D5FC4A46514605201AF084FA71
:101FA8001522012384F87950C4F87C803A7284F8A9
:101FB80078300225CAE500BFC85B0020B0F1FF3FBA
:101FC8000AD0022810B403DC5DF8044BFEF718BCF5
:101FD80000205DF8044B704700207047F0B55B4B5C
:101FE8005B4A97B01968914200AF00F0A380594945
:101FF800594A00234FF47000C1F888003B607B60A9
:10200800136843F48033136003E03B68B3F5A04FD3
:1020180009D0136803F400337B603B6801333B60ED
:102028007B68002BF1D04C4B1B6813F4003318BFAE
:1020380001237B607B68012B52D0464C464B474AB4
:10204800E260474A596A11605A6A42F080725A62DD
:102058005A6942F4FC025A610025032207F108017B
:10206800012341F6FF764FF09040FD60BE603A7361
:10207800BB731EF0C9FF4FF6FF7307F1080139481B
:10208800BB601EF0C1FF07F108013748374E1EF04C
:10209800BBFF07F1080136481EF0B6FF07F108013B
:1020A80034481EF0B1FF07F1080133481EF0ACFFB9
:1020B80007F108001EF0B8FDBB683049304AA1FBA3
:1020C800031330499B0CF0204FF0070E5C370B6070
:1020D800566084F823009560C2F800E0BD46F0BD64
:1020E800294A1D4B122111605A685A605A685A6071
:1020F8005A6842F480625A605A6822F47C125A6024
:102108005A6842F4E8125A601A6842F080721A60FB
:102118001A689201FCD559680F4A21F003015960E9
:10212800596841F002015960536803F00C03082B09
:10213800FAD182E700221A6062B6144B1B6883F357
:102148000888134B1B689847FEE700BFFC9F0020D8
:10215800EFBEADDE00ED00E0001002400005FA051C
:10216800084D002000040048000800483F190100FD
:10217800000C0048001000480014004883DE1B4390
:1021880010E000E0A05900200020024000D8FF1F06
:1021980004D8FF1F70B50F4C0F4DC0EBC00004EB07
:1021A8008004686926693043686182B09209667B59
:1021B800A1600025012101A863618DF804608DF8F4
:1021C80005208DF806508DF8071022F0DBFD02B0CF
:1021D80070BD00BFF81A002000100240074BC0EB8A
:1021E800C00030B403EB8000054C056963692B43DC
:1021F80063610176427630BC704700BFF81A002050
:10220800001002402DE9F04F5E4C54F8204083B096
:10221800002C71D0666D984691465B4B7268E264FB
:10222800A160236004F15A014FF4807304F5AD7284
:102238006161A261E36023610746307E25F008FAF8
:10224800F068A8B1514B00215A68904203F11C0371
:1022580000F0928001310C29F6D100207A1CD2B20C
:102268000C21FFF7BBFFE36CF26822632433A364FD
:10227800B068D8B1454B00215A68904203F11C035D
:1022880078D001310C29F7D100257A1CD2B20B2164
:102298002846FFF7A3FF2346F27E3D492846FFF76D
:1022A80079FFE36CB26862632833636494F8590079
:1022B80008F0C8FC054694F8580008F0C3FC18F06C
:1022C800080F824696F819B01AD0CDB118F0110F40
:1022D8004FF00B0307F1010714BF4E213E21EF71A8
:1022E8005A46AB71284608F00DF918F0010F45D091
:1022F800236B5BB3636B4BB3204603B0BDE8F08F31
:1023080018F0010F0CBF4FF02E084FF04E0819F0CF
:10231800020F09D045B10B227B1CAA71EB7128462C
:102328005A46414608F0EEF819F0010FE0D0BAF12C
:10233800000FDDD001370C238AF807705A46414652
:102348008AF80630504608F0DDF8D1E7337FB27ED0
:102358008DF804209B090021012201A88DF8053081
:102368008DF806108DF8072022F00CFD204603B0EA
:10237800BDE8F08FCDB288E7C8B26FE7284609F00C
:102388001FFEB5E77C2B0020D4DC0208F81A0020D9
:102398002D0B00080348D0F83C3113B100F59A70B2
:1023A80018477047F81A00200348D0F8203113B1B5
:1023B80000F58C7018477047F81A00200348D0F8C9
:1023C80004310BB1FC301847704700BFF81A0020E1
:1023D8000348D0F8E8300BB1E0301847704700BF29
:1023E800F81A00200348D0F8CC300BB1C430184795
:1023F800704700BFF81A00200348D0F8B0300BB17E
:10240800A8301847704700BFF81A00200348D0F8D2
:1024180094300BB18C301847704700BFF81A002071
:102428000248836F0BB1703018477047F81A0020C4
:102438000248C36D0BB1543018477047F81A002092
:102448000248036C0BB1383018477047F81A00205F
:102458000248436A0BB11C3018477047F81A00202D
:102468000248836803B11847704700BFF81A002074
:10247800F0B53E4C059D00EB800004EB80046468D9
:10248800002C71D03A4E49004FF42040CFB2B060D2
:10249800A169090454D46068DFF8E0E047F490319A
:1024A80000EA0E0001434FF420406160B06003E091
:1024B800411E002848D00846A1698907F8D54FF47D
:1024C8002040A262B06003E0421E00283CD01046C3
:1024D800A2695206F8D5274A6168DFF8A0E0B06023
:1024E80042EA0342174301EA0E0217436760C3B189
:1024F800013BDBB201332B44A0694FF4204210F0BA
:10250800040002F1FF3207D1511C26D0A06910F057
:10251800040002F1FF32F7D0626A05F8012B9D42F0
:10252800EAD14FF42040B06002E0431E60B1184683
:10253800A3699B06F9D52023B060E3610120F0BDB3
:10254800411E08B10846A3E70B4A138801339BB222
:102558004FF0FF311380B160F0BD0749B2600B88BE
:1025680001339BB20B80F0BD2046F0BD9C2B0020B0
:10257800CC1E002000240002482C0020009800FCFB
:102588002DE9F0410C460178012982B052D0022988
:1025980056D11D46836844F0800113B11C689B889E
:1025A8002385446840F2E93301E0002B6FD0268987
:1025B800013B16F0020F9BB2F7D0217304F10C0611
:1025C80040F2E93301E0002B71D02189013B11F081
:1025D800010F9BB2F7D033784468A3894FF0000C01
:1025E8004FF47A734FF6FF764FF0FF0E654502D130
:1025F8003AE0B34228D02189013B11F002019BB295
:10260800F7D084F80CE004F10C084FF47A7302E078
:10261800BBB2B34218D0218911F0010103F1FF3791
:10262800F6D098F80010C9B20AB1117001320CF155
:10263800010CDBE790F90450691C01D0022D1DDD67
:10264800002002B0BDE8F081224B9C4204D0A3F5E3
:1026580078439C4208D101211F4B03EB01114B89A0
:1026680001339BB24B814B898368002B30D01A68A9
:102678009B889361012002B0BDE8F0814179009206
:1026880028462246FFF7F4FE02B0BDE8F081114962
:102698008C4203D0114B9C429FD101230E4901EB80
:1026A80003135989013189B259815B8995E7094931
:1026B8008C4203D0094B9C428ED10123064901EB81
:1026C80003135989013189B259815B89446884E7C8
:1026D8000120B6E700300140F459002000380040DE
:1026E80070B582B06A460623F721FFF749FF9DF8C7
:1026F80001209DF804309DF800609DF803509DF876
:1027080002409DF80500074912011B0142EA063202
:1027180043EA053342EA141243EA10134A600B6095
:1027280002B070BDCC1E002000B583B0002000921E
:102738000A466821FFF79CFE03B05DF804FB00BF62
:10274800421C76D0022874DC2DE9F843142303FBDD
:1027580000F33D4FFA583B44002A6BD01C1D94E807
:1027680010030546907B24F073FF384B9C4263D0DE
:10277800374A136B23F0100313631023344A116B89
:102788006E1C0B431363F6B2B8F1000F04D0152387
:1027980088F8076088F80630142303FB0573404661
:1027A8005B7C002B14BF3E211E21042207F0AAFEE9
:1027B800B9F1000F04D0162389F8076089F80630AC
:1027C800142000FB057504226B7C002B14BF3E21EE
:1027D8001E21484607F096FE21682D7C1D4B1E4899
:1027E8001E4A21F0010121602168002D08BF03461F
:1027F8000A40226023612268002342F0010222601D
:10280800A360E360A360A36843F40043A360236864
:102818002360636823F0784323F4004363602368EC
:1028280023F400332360236843F001032360BDE8E9
:10283800F8837047BDE8F8830549094B0A6B22F015
:1028480020020A639AE700BF9C2B00200058004032
:1028580000100240300E50007A25E000FFE0CF0063
:10286800200000101749184B184A194810B4D1F81D
:10287800884044F47004C1F888401C6844F001049E
:102888001C605C6822405A601A6822F0847222F444
:1028980080321A601A6822F480221A605A6822F478
:1028A800FE025A60DA6A22F00F02DA621A6B00241A
:1028B80010404FF0006218639C608A605DF8044B1A
:1028C800704700BF00ED00E0001002400CC07FF828
:1028D800CCFC00FF2DE9F04F2DED0C8B364D99B057
:1028E8006B68099028469847002800F06F82B5F871
:1028F800B470002285F85520002F67D1B5F93C60E7
:10290800686AE96AB5F93E20AC6AB5F94030DFF883
:10291800B8B0301A5B1A121B286395F85610AB63CF
:1029280005F130006A631DF0C5FCDBF80030990042
:1029380042F19A80D5ED0D5A204CD5ED0C7A204AFB
:1029480094ED406AD4ED416A94ED427AD4F80C31A2
:102958001268B8EEE58AD5ED0E5AF8EEE77AF8EE89
:10296800E58A013377EE867A38EE268A78EE878A0A
:102978009342C4ED407A84ED418AC4ED428AC4F89A
:102988000C3101F0BB840F4B059393F800E0BEF1C6
:10299800140F03F089840023D4F814610693062EDB
:1029A80001F22286DFE816F0E117CE17E916A31820
:1029B800890D0C194B1700BF9C540020BC1F002028
:1029C800444500202C5C002030570020D94BDA49C0
:1029D800089391F801901B68D848DFF8BC830590EC
:1029E8004FF47A71B1FBF3F3C3EB431403EB8403A5
:1029F800DC00A4B2A7420678B8F9060003F02582E5
:102A0800D5F888E0B5F93C20EB6E0EF1010107EE30
:102A1800902A13440129C5F88810EB66F8EEE77A86
:102A280003F01E82D5ED1E5AD5ED206A07EE101A66
:102A380037EEE56AB8EEC75A012F86EE057A37EE0B
:102A4800257A77EEC77A85ED1F7AE7EE866A85EDF7
:102A58001E7AF0EE667AC5ED216AC5ED206A03F0AC
:102A6800AB85D5F89CE0B5F93E202B6F0EF101013E
:102A780007EE902A13440129C5F89C102B67F8EE3D
:102A8800E77A03F00682D5ED235AD5ED256A07EEDD
:102A9800101A37EEE56AB8EEC75A012F86EE057AA6
:102AA80037EE257A77EEC77A85ED247AE7EE866ADF
:102AB80085ED237AF0EE667AC5ED266AC5ED256ABE
:102AC80003F05385D5F8B0E0B5F940206B6F0EF1EF
:102AD800010107EE902A13440129C5F8B0106B676D
:102AE800F8EEE77A03F0EE81D5ED285AD5ED2A6A9B
:102AF80007EE101A37EEE56AB8EEC75A012F86EED0
:102B0800057A37EE257A77EEC77A85ED297AE6EEEB
:102B1800276A85ED287AF0EE667AC5ED2B6AC5ED51
:102B28002A6A03F01685A8F80600059B013F1E785F
:102B3800A5F8B4700899824C0023072E4B608B606F
:102B4800CB6040F04A8108F01BFC059BDFF8488207
:102B58001E78099BC01A94F81C31A8F800000A9343
:102B6800002B40F04081744B5B79002B01F0DD8233
:102B7800744B1B78013BDBB2072E84F81C3102F042
:102B8800FA8300230B93704B94ED499A93ED007AE6
:102B98006E4BD4ED48CA1B680693F7EE007A37EE01
:102BA800C9CA644B08932CEE07CA0026B4EEE7CADC
:102BB800F1EE10FA664BDFF8E4A1DFF8E4B1DFEDDF
:102BC800658A9FED65AADFED65BADFED659A9FED31
:102BD80065BADFED65AADFF8CC91DFF8CC81079301
:102BE80088BFB0EE67CA3746604B9AED008A334417
:102BF800D3ED007AF5EE407AF1EE10FA17D05C4B7F
:102C0800334493ED007A78EE476AB0EEE66AF4EE64
:102C1800C67AF1EE10FA08D5F5EEC06AF1EE10FAB0
:102C2800CCBF37EE878A37EE678A83ED008A514B2F
:102C38001A8893073AD0022F38D006994E4B91F84C
:102C48002E10334407EE901A93ED007A4B42F8EEBB
:102C5800E76A07EE903A26EE877AF8EEE77AB4EE5E
:102C6800E77AF1EE10FA0AD407EE901AF8EE677ACE
:102C7800F4EEC77AF1EE10FA88BFF0EE477A3F4BD0
:102C88003F4903EB470331F91700B3F90C30C01A79
:102C980007EE100AB8EEC77AD007E7EE687A41F176
:102CA800E081384B93ED008A27EE888A089B94F8D8
:102CB80058213344D3ED01DA38EE6DDA002A00F0FA
:102CC800E480314BD4F85C2109991B688A1A9A422E
:102CD80040F3DB80022F04F0EB852C4B1B6899072F
:102CE80000F196802A4BC8ED00BA1B689342C0F2E7
:102CF800C980F7EE007AB4EEE79AF1EE10FA40F1E7
:102D0800C4800899234BD1ED017A93ED007AF0EE57
:102D1800E77AF4EEC77AF1EE10FA40F1B680D1ED19
:102D2800027AF0EEE77AB4EEE77AF1EE10FA40F3C1
:102D3800AC803BE020570020885400202C5C002009
:102D4800BC1F002080420020643100206451002014
:102D580054400020CDCCCC3DAE47813F0000000060
:102D68000000C842610BB63B0000344358310020D4
:102D7800F0200020623D0020FC2000208C42002032
:102D8800D4510020403100206C310020A83E0020A2
:102D98006831002074310020305C0020E4200020DD
:102DA800503000206C40002060400020D1ED037AB4
:102DB800F0EEE77AB4EEE77AF1EE10FA65DD0F4B44
:102DC8001B689A075ED50E490E4B42E00E4B0F4C1E
:102DD8001E780593072E3FF4B6AE94F81C310A937B
:102DE800002B3FF4C0AE013B84F81C31012E01F0EA
:102DF800388419B0BDEC0C8BBDE8F08FA83E0020DC
:102E0800D45100208C4200202C5C0020BC1F0020E4
:102E1800D64BD749DFF8C4E331F917C09EED008AD5
:102E2800DFF8BCE3C8ED00BA03EB470028EE288AB8
:102E3800B0F90C00A0EB0C0007EE900AF8EEE77A68
:102E4800DEF8000027EE888A824238EE6DDA7FF7D6
:102E580050AFB3F90C20B1F900E0C648AEEB020E52
:102E680000688EEAEE72A2EBEE7282420DDAB3F9D6
:102E78000E30B1F90220D21A82EAE273A3EBE273B0
:102E8800984202DD002384F85831BB4B334493ED5C
:102E9800000A079B2CEE800A022F20EE0D0AA3ECF5
:102EA800010A079304F0C284B44B9BED007AD3ED7A
:102EB800007AB34BD8ED006A93ED006AB14B67EE28
:102EC800277A334427EE8C7AD3ED007A67EE277A97
:102ED800F0EE665AEDEE275AB1EE467AF4EEC75A8E
:102EE800F1EE10FA08D4B4EEE56AF1EE10FA8CBFF0
:102EF800B0EE657AB0EE467A94ED496AF7EE007A5C
:102F0800B4EEE76AF1EE10FAACBF0123002343B137
:102F1800F0EEE66AF0EEC77AF4EEE67AF1EE10FA31
:102F280001D588ED007A022F04F0FE83964A974B6C
:102F380052F827001B68B0EE6D0A9847944A954BE3
:102F480052F827001B689847069B93F8373023B13F
:102F5800914B1B88002B01F0EB80B0EE6B8A8F4BF6
:102F68009BED007A38EE400A334493ED008A83EDF6
:102F7800000A069B30EE480A93F84830C0EE077AFC
:102F88003BB3874B1B78DB0741F1618094F85831DC
:102F9800B7EE007AB4EEC79AF1EE10FAC1F2D6860F
:102FA800002B01F05481D4F85C31099AD31A7D4A78
:102FB80012689A420DDD7C4B93ED007AB0EECDDAC3
:102FC800B4EEC7DAF1EE10FA42F1BB86002384F8BA
:102FD8005831764B94F86821334493ED007A2CEEFF
:102FE800877A67EE277AC9ED007A32B9079BC8ED70
:102FF80000BA43ED01BAC9ED00BA0137032F0AF14F
:10300800040A09F1040908F1040806F104067FF42A
:10301800EBAD059B1B78072B01F0AD86012B02F069
:1030280097810023089394F87031002B41F04C836A
:10303800DFF8B0B15E4BDBF800C01A681CF48053AF
:1030480092F82C100C9341F08E805A4B06931E4632
:103058005948768B594BD0ED006A93ED006A584B6E
:10306800C4ED606A07EE906A564EC4ED5E6A96ED4E
:10307800037A84ED616AF8EEE77A76EE665A77EEBF
:10308800677A93ED007AC4ED5D5A012384F888319C
:10309800C7EE875A138D584206EE900A4A489FEDAC
:1030A8004B7A90ED005A4A48D0ED004A4948F7EE6D
:1030B800007AF4EEE75A90ED006A35EE245AF1EE04
:1030C80010FA88BFF0EE675A35EE065AF8EEE66A4F
:1030D800F4EEC75AF1EE10FA07EE903AB4EEE65A5B
:1030E800B8BFF0EE475AF1EE10FAC4ED635AB8EEE5
:1030F800677A01F19A84B4EEC75AF1EE10FA88BFE4
:10310800B0EE475A304BDFED344AD3ED017A304BFD
:1031180093ED014A2F4B77EE847A93ED016A77EEAF
:10312800867A25EE245AF4EEE76AF1EE10FA08DC06
:10313800B4EEE77AF1EE10FA8CBFF0EE676AF0EEC3
:10314800476A538D204A9FED247AD2ED027A204AAD
:1031580092ED026A5A4204EE102A77EE867AB8EEA9
:10316800C44A66EE876AF4EEC47A3DE08C420020D9
:10317800D45100207031002014310020200000209C
:1031880088310020203100205830002054300020A1
:10319800AC300020A8300020623D00201C21002017
:1031A800FC4800206C310020783100202C310020B0
:1031B80064510020DC4C0020F44000205C420020D8
:1031C800D82700204C5C002054400020000000005C
:1031D800604000206C4000206F12833A403100208C
:1031E8006831002030570020F1EE10FA0AD407EEBB
:1031F800103AB8EE474AB4EEE74AF1EE10FA88BF43
:10320800B0EE674AEA4BDFEDEB7A5B7824EE274AAB
:103218000BB9B1EE444A002941F0EF87B7EE003A06
:10322800DFF8B88398F80020002A02F0F587E24B0F
:103238009FEDE26AD3ED024A93ED017AD3ED037A6A
:1032480066EEA44AE5EE074AE4EE274A63EE244A0E
:10325800F4EEC64AF1EE10FAB4BFF0EE463AF0EEDC
:10326800643A98BFB0EE646A012ACDED104A03F0C3
:103278002E80D3ED067AD3ED052A93ED077A66EE14
:10328800A77AE5EE227AE4EE077A23EE277AB4EEFF
:10329800C67AF1EE10FAB4EEE37A8CBFF0EE467A15
:1032A800F0EE477AF1EE10FA98BFB0EE676AB4BF55
:1032B800F0EE637AF0EE477A022A8DED117A00F08B
:1032C800DE8093ED0A7AD3ED092AD3ED0B3A26EE88
:1032D800877AA5EE227AA4EE237A23EE077AB4EE53
:1032E800C67AF1EE10FAB4EEE77A8CBFF0EE463A01
:1032F800F0EE473AF1EE10FA98BFB0EE636AA8BF55
:10330800F0EE477A032A8DED127A00F0B88093ED3B
:103318000E7AD3ED0D2AD3ED0F3A26EE877AA5EE75
:10332800227AA4EE237A23EE077AB4EEC67AF1EE77
:1033380010FAB4EEE77A8CBFF0EE463AF0EE473A70
:10334800F1EE10FA98BFB0EE636AA8BFF0EE477AC4
:10335800042A8DED137A00F09280D3ED123AD3ED62
:10336800112A93ED137A66EEA33AE5EE223AE4EEDB
:10337800073A63EE233AF4EEC63AF1EE10FAF4EEA9
:10338800E73A8CBFB0EE467AB0EE637AF1EE10FA07
:1033980098BFB0EE476AA8BFF0EE637A052ACDED74
:1033A800143A6CD0D3ED163AD3ED152A93ED177A6B
:1033B80066EEA33AE5EE223AE4EE073A63EE233AE4
:1033C800F4EEC63AF1EE10FAF4EEE73A8CBFB0EE3E
:1033D800467AB0EE637AF1EE10FA98BFB0EE476A1B
:1033E800A8BFF0EE637A062ACDED153A47D0D3EDA3
:1033F8001A3AD3ED192A93ED1B7A66EEA33AE5EE55
:10340800223AE4EE073A63EE233AF4EEC63AF1EED6
:1034180010FAF4EEE73A8CBFB0EE467AB0EE637A73
:10342800F1EE10FA98BFB0EE476AA8BFF0EE637AE3
:10343800072ACDED163A22D093ED1E7AD3ED1D2A38
:10344800D3ED1F3A26EE877AA5EE227AA3EE847A88
:1034580027EE037AB4EEC67AF1EE10FAB4EEE77A04
:103468008CBFF0EE466AF0EE476AF1EE10FA8DED89
:10347800177A98BFB0EE666AA8BFF0EE477A77EE83
:10348800C67AF7EE006AF4EEE67AF1EE10FAC4EDC9
:10349800497A43F3788786EEA77A022ADDED117A16
:1034A80067EE244A67EE877ACDED104ACDED117AA2
:1034B8002DD0DDED127A67EE877A032ACDED127AE8
:1034C80025D0DDED137A67EE877A042ACDED137ADD
:1034D8001DD0DDED147A67EE877A052ACDED147AD2
:1034E80015D0DDED157A67EE877A062ACDED157AC7
:1034F8000DD0DDED167A67EE877A072ACDED167ABC
:1035080005D0DDED177A27EE877A8DED177A2C4BEB
:103518001B6813F0805A01F0D183F6EE005AC4ED0F
:10352800635A002A02F09986264B94F98811DB78B1
:103538000B93254B94ED616A94ED605A2348244F10
:10354800D0ED004A3F78D4ED5D6AD4ED5E7A07EE9F
:10355800101A19781F4B0793B3F906300D93069B81
:10356800BDEEC66A5B8B0E9316EE10EA0B9BBDEEA2
:10357800C56A01F001090CF01000B8EEC77A16EE22
:10358800101A0CF4800C002B41F0C880002841F080
:10359800FB8409489DED105A90ED006A0E4B25EE0C
:1035A800866AA5EE076AB0EE675AA6EE265A17E0B5
:1035B800CC4200206F12833A482700200000000008
:1035C800544200207C3D0020FC4800208C31002023
:1035D80094490020AC5F0020B4400020F05E002039
:1035E800BDEEC56A16EE10CA16EE107AF445A8BFED
:1035F80077466145C8BF0F4606EE107AB8EEC66A30
:10360800012A83ED006A00F0DC8090ED046A9DEDEC
:10361800115A25EE866AA5EE076AB0EE675AA6EE3D
:10362800265ABDEEC56A16EE10CA16EE107AF44593
:10363800A8BF77466145C8BF0F4606EE107AB8EEB8
:10364800C66A022A83ED016A00F0BB8090ED086A21
:103658009DED125A25EE866AA5EE076AB0EE675A06
:10366800A6EE265ABDEEC56A16EE10CA16EE107AF8
:10367800F445A8BF77466145C8BF0F4606EE107AE5
:10368800B8EEC66A032A83ED026A00F09A8090EDCC
:103698000C6A9DED135A25EE866AA5EE076AB0EE10
:1036A800675AA6EE265ABDEEC56A16EE10CA16EE81
:1036B800107AF445A8BF77466145C8BF0F4606EEA5
:1036C800107AB8EEC66A042A83ED036A79D090EDC1
:1036D800106A9DED145A25EE866AA5EE076AB0EECB
:1036E800675AA6EE265ABDEEC56A16EE10CA16EE41
:1036F800107AF445A8BF77466145C8BF0F4606EE65
:10370800107AB8EEC66A052A83ED046A59D090ED9E
:10371800146A9DED155A25EE866AA5EE076AB0EE85
:10372800675AA6EE265ABDEEC56A16EE10CA16EE00
:10373800107AF445A8BF77466145C8BF0F4606EE24
:10374800107AB8EEC66A062A83ED056A39D090ED7C
:10375800186A9DED165A25EE866AA5EE076AB0EE40
:10376800675AA6EE265ABDEEC56A16EE10CA16EEC0
:10377800107AF445A8BF77466145C8BF0F4606EEE4
:10378800107AB8EEC66A072A83ED066A19D090ED5A
:103798001C6A9DED175A65EE865AE7EE055AE6EE65
:1037A800A57AFDEEE77A17EE900A8645A8BF864609
:1037B8008142D8BF714607EE901AF8EEE77AC3ED5A
:1037C800077AB9F1000F01F0B680E54B1B68002BB2
:1037D80041F0BE80E34B1B78ABB198F8000078B19C
:1037E800DFF8A893DFF8A8A30027F8B2DAF80030CA
:1037F800B9EC010A984798F8000001378742F4DBD2
:10380800D94B1B689847059B1B78072B01F0A382AF
:1038180000230893DBF8009019F4806F41F02881A9
:10382800D24B079A1D68B2F906806A89904580F2E2
:1038380029864FF07E53C4F82031DFF858A3079A41
:10384800069BB2F900001F8B9AF904309AF8001011
:103858009AF801E0002BA0EB070383EAE37CACEBCA
:10386800E37C14BF01224FF0FF32BCF5FA7FA8BFFA
:103878004FF4FA7C614580F20186ACEB010307EE58
:10388800903AF8EEE77A8742C6ED007A03DDF1EE6A
:10389800677AC6ED007A079BB3F90200C31B83EA77
:1038A800E37CACEBE37CBCF5FA7FA8BF4FF4FA7C71
:1038B800614580F2DF85ACEB010307EE903AF8EE44
:1038C800E77A8742C6ED017A03DDF1EE677AC6ED45
:1038D800017A079BB3F90410CB1B83EAE370A0EBD2
:1038E800E370B0F5FA7FA8BF4FF4FA707045CCBF0B
:1038F800A0EB0E0E4FF0000E02FB0EFE07EE90EA54
:10390800F8EEE77AB942C6ED027ABCBFF1EE677A03
:10391800C6ED027A19F4805B00F08785B8F5FA6F76
:103928004246A8BF4FF4FA62B2F57A7F94F8903114
:10393800B8BF4FF47A72A2F57A72002B40F08E85E8
:103948008B49DFF854E281FB0230D317C3EB6013D5
:10395800581C6FF0630C3EF910003EF913E00CFBA5
:103968000323A0EB0E0003FB00F381FB0321DB170D
:10397800C3EB61139E440FFA8EFE07EE90EAB8EE91
:10398800E78A86ED038ABBF1000F41F07D80794B11
:103998001B8813F04002079200F0DD80764A7748D2
:1039A80092ED019A92ED026A90ED020A90ED043AC6
:1039B800D2ED030AD2ED003AD0ED038AD0ED015AD8
:1039C800D6ED011A96ED002A6D4A30EE435A39EECB
:1039D800467A73EEA07A25EE077A75EEE84A73EE1A
:1039E800E09A35EEA8AA24EEA71AB0EE474AAAEE46
:1039F800294A13F00301B0EE415A79EE067A70EEC7
:103A0800036AAAEE295AA6EEA74AA6EEE75AF0EEEE
:103A1800474AD6EEA74A34EE014AF6EE006A73EE3C
:103A280089AA26EEC44A35EE475A35EE807AF0EE7A
:103A3800647AEAEE694AA7EE2A4A77EEC17A36EE48
:103A4800607A73EE68AA25EE265AEAEE297AAAEE7B
:103A5800875A74EE814A24EE047A73EEC93A33EE3B
:103A6800283A64EEA64A75EEC05A36EE206A67EE2A
:103A7800A66AF0EE477AE3EE234AD5EE057AA5EE7C
:103A8800057AE5EE866AF1EE648AB0EE476AB0EE32
:103A9800677AF1EE663AA8EEA47A64EE260A26EE74
:103AA800A43AA3EEA66AB1EE450AE3EEA67AF0EED2
:103AB800609AB0EE431A64EE243AA6EEA67AE5EED2
:103AC800249AA0EE041AF0EE665AA8EEA46AF0EE64
:103AD800638A71EEA16AE0EE240AE5EE258A27EEF4
:103AE800217A32EE029AA5EE043A61EE211A66EEC8
:103AF800A96AE4EEA47AE0EE253A0CBFD6ED022AD4
:103B0800DFED202A82ED005AE2EE066AA9EE207A5D
:103B1800E2EE281A33EE033A67EEA27A73EEA33A7E
:103B2800B0EE006AA2EE837AE2EEA36AE1EE867A4C
:103B380084ED677A86ED017AC4ED666AC6ED006A9F
:103B4800C4ED687A82ED014AC2ED025AC2ED034A19
:103B580009B9C6ED027A0C4A126812F0140F1DE07A
:103B68004C300020BC4C002090490020D45F00203D
:103B78001F85EB51623D0020B0000020200000208E
:103B8800E800002000000000A83E0020B44000200B
:103B98008849002084420020D85F002003D013F415
:103BA800027F41F01B80DA4A12789AB1069A528B4A
:103BB80042450FDBD74A1278012A01F0E183192A1E
:103BC80001F0DE830E2A05D0082A03D00022B26055
:103BD800C4F8302194F8CA7117B1980741F04E83A0
:103BE80094F8D071002F40F09587069B9B7F002B9F
:103BF80000F01384022B01F03183032B41F035834D
:103C0800069B93F82030C3EB431203EB8202D200E9
:103C180092B2069BDB7F0233DBB2002F00F06E8589
:103C2800002A00F06B85BC490968B2FBF1F20FFA73
:103C380082F8A4F80082ABB307EE908AF8EEE77A30
:103C4800F7EE006A86EEA77A012BD6ED007AD4ED5E
:103C5800856A77EEE67A67EE877AC4ED817A21D0B5
:103C6800D6ED017AD4ED866A77EEE67A022B67EE16
:103C7800877AC4ED827A15D0D6ED027AD4ED876AB8
:103C880077EEE67A032B67EE877AC4ED837A09D05C
:103C9800D6ED037AD4ED886A77EEE67A67EE877A0E
:103CA800C4ED847A059A1278092A03F0E581B8F1FF
:103CB800000F40F3B8839BB394ED857AD4ED817AF5
:103CC80077EE877A012BC4ED857AC6ED007A21D08C
:103CD80094ED867AD4ED827A77EE877A022BC4ED5A
:103CE800867AC6ED017A15D094ED877AD4ED837A79
:103CF80077EE877A032BC4ED877AC6ED027A09D06E
:103D0800D4ED887A94ED847A77EE877AC4ED887A50
:103D1800C6ED037A013B022BB8BF0223DBB20A933C
:103D2800002F0A9818BF02202B78DFED806AAA7846
:103D380007EE903AF8EEE77AB0EE007A67EEA67AE8
:103D4800059BF4EEC77AF1EE10FA197840F358861D
:103D5800DFED736A37EEC77AB0EE676AA7EE266AB8
:103D6800F0EE466A96ED007A9FED6E6A27EE066AD7
:103D7800F0EEC65A84ED506AC4ED535A9AB107EE74
:103D8800102AB8EEC75A9FED697A66EE064A25EE04
:103D9800075AB7EE007A37EE457A64EEA54AA4EEE4
:103DA800857A26EE076A9FED607A6B7926EE877A28
:103DB80027EE067ACBB1DFED5D6A9FED5D6A65EEB1
:103DC800A65A06EE903AF8EEE66A66EEA56AF4EEB2
:103DD800C66AF1EE10FA01F30382F7EE005A75EEA7
:103DE800E66A85EEA66A27EE067A0C299FED518AC7
:103DF800DFED516A00F07087B4EEC87AF1EE10FA80
:103E080098BFB0EE478AB4EEE68AF1EE10FAB8BF72
:103E1800B0EE668A84ED4A8A002800F0F580B0EE9C
:103E2800007AF4EEC77AF1EE10FA05DD37EEC77ABC
:103E3800DFED3B6AE7EE267A96ED017ADFED396A27
:103E480027EE267AF0EEC75A84ED517AC4ED545A1B
:103E58009AB106EE902A9FED356AF8EEE66A27EEEB
:103E6800075A66EE866AB7EE006A36EE666A25EE8F
:103E7800255AA5EE266A27EE067ADFED2B6AAB797E
:103E880067EEA67A67EE877AABB107EE103AB8EE1E
:103E9800C77A9FED266ADFED266A27EE257A27EE98
:103EA800067AB4EEE67AF1EE10FA41F38781DFED97
:103EB8001B6A67EEA67A0C2900F02987DFED1D6AD8
:103EC8009FED1D7AF4EEE67AF1EE10FA88BFF0EE77
:103ED800667AF4EEC77AF1EE10FAB8BFF0EE477AD8
:103EE8000128C4ED4B7A40F38F806B78DFED0F6AC1
:103EF80007EE903AF8EEE77AB0EE007A67EEA67A27
:103F08006B7AF4EEC77AF1EE10FA1DDD16E000BF09
:103F1800F21C0020CC420020B44200200000C8421D
:103F2800D7A368416F12033B000048430AD7233CDC
:103F3800A4707D3F00C0F94400C0F9C437EEC77AC9
:103F48005FED096AE7EE267A96ED027A5FED0B6A75
:103F580027EE267AF0EEC75A84ED527AC4ED555A08
:103F68009BB106EE903A1FED0F6AF8EEE66A27EE6F
:103F7800075A66EE866AB7EE006A36EE666A25EE7E
:103F8800255AA5EE266A27EE067A5FED196AEB79BF
:103F980067EEA67A67EE877AFBB107EE103AB8EEBD
:103FA800C77A1FED1E6A5FED1E6A27EE257A27EE97
:103FB800067AB4EEE67AF1EE10FA01F30D81B5EE69
:103FC800C07AF1EE10FA02F11E83B7EE006A36EEFF
:103FD800477AC6EE076A67EEA67A0C2900F074865F
:103FE8005FED2C6A1FED2C7AF4EEE67AF1EE10FA0A
:103FF80088BFF0EE667AF4EEC77AF1EE10FAB8BF31
:10400800F0EE477AC4ED4C7A092900F04986069B00
:1040180093F82150002D40F0FE85002384F8D0311C
:10402800A04B1B7823B9A04DAB78002B41F03B8106
:10403800059B1E78072E7EF4D9AE07F0A1F9059AE4
:104048009A4B1678089A801AD880FEF7CFBE94F853
:104058005831002B3EF4BDAF002384F85831FEF7E9
:10406800B8BFB1F9002094ED537AB1F90200D4ED4C
:10407800546A8F4982EAE273A3EBE273F4EEC76AEB
:1040880080EAE072F1EE10FAA2EBE072B8BFF0EE4F
:10409800476A9342B8BF134607EE103A0B78B8EE5A
:1040A800C77A27EE287A002B40F0A280814B93ED47
:1040B800006AB4EECA6AF1EE10FA41F1DA80F7EE5E
:1040C800005A75EEC65A3AEEC77A65EE8B5A7A4BA5
:1040D800A5EE876A93ED007A26EE076AB5EEC06A08
:1040E800F1EE10FA40F2E685C9EE865AB7EE007A8C
:1040F800B0EE476AA6EEE56AF0EE466AF4EEC76AE5
:10410800F1EE10FA88BFF0EE476AF5EEC06AF1EEFC
:1041180010FAB8BFF0EE6B6A684B93ED007A67EE61
:10412800877AA7EEA68AFEF7C1BD0123FEF724BD54
:10413800634B644A334493ED007AD2ED007A624BC4
:1041480067EE277AF7EE006AF4EEE67AF1EE10FAF7
:1041580093ED007A88BFF0EE667A67EE877A27EEED
:10416800888AFEF7FCBE594B594E1B7896ED037AA8
:1041780013F0010F574B069304BF1B8BA4F87C3137
:10418800554B188807EE900AF8EEE77AB4EEE77A0E
:10419800F1EE10FA41F2D187504B1B8807EE903AA6
:1041A800F8EEE77AB4EEE77AF1EE10FAC1F2EF80B2
:1041B8004B484C4BD0ED006A93ED006A4A48C4ED79
:1041C800606ABCEEC75A76EE665A15EE103AC4ED30
:1041D8005E6AC4ED5D5A84ED616AA4F87C310123FE
:1041E80077EE677A90ED007A84F88831FEF750BF51
:1041F800314B93ED005AB5EEC05AF1EE10FA40F388
:1042080059853A4BD3ED004AF5EEC04AF1EE10FA63
:1042180040F3508534EEC77A66EEE95A87EE246A91
:10422800C5EE856AB7EE007AB4EEC76AF1EE10FA09
:1042380088BFB0EE476AB5EEC06AF1EE10FA76EEC6
:10424800876AB8BFB0EE6B6A66EE266A56E7284AF8
:1042580092ED007AF0EEE76AF4EEC76AF1EE10FA32
:104268007EF7B7AE234A92ED007AF0EECD6AF4EE0F
:10427800C76AF1EE10FA7EF7ACAE1F4A9AED007AE3
:10428800D2ED006AB0EEC77AB4EEE67AF1EE10FA33
:104298007EF59FAE01220999C4F85C1184F8582173
:1042A800FEF785BE3D510020D2360020305C00204C
:1042B8004C31002054310020483100204431002086
:1042C800082100203C31002038310020FC48002023
:1042D8004C5C0020DC4C0020DC270020DE2700207E
:1042E800C82700205C420020E4270020503100202D
:1042F8007C3100207831002080310020DF4A05928F
:1043080007EE103A1278DFF8B483C4F80C71B8EEEF
:10431800C77AF7EE006A132A86EE879AB8F904007E
:10432800B4F8106195ED080A01F01A85D44BD54A06
:1043380093ED001AD3ED053A93ED122A93ED173A4F
:10434800D3ED091AD3ED0E4A93ED016A93ED064AAF
:1043580093ED0A7AD3ED0F5AD3ED132AD3ED186AE9
:1043680093ED045AD3ED030A67EE897A69EE288A39
:1043780029EE088AE1EE273A02EB86070021A2EE31
:10438800283AC4F80011C4F80411E1EE884AA6EEF0
:10439800274AE7EE085A93ED167A93ED0D6A93EDE6
:1043A800021AD3ED0C1AC7ED003AE2EEA86A25EE20
:1043B800635A27EE437A93ED0B2AD3ED152AC7EDFE
:1043C800204AA0EEE34A26EE646AD3ED143A83ED60
:1043D800054AA1EE275AF0EE477AE1EEE45AA2EE3A
:1043E800086AE2EEC36AE3EEA87A83ED065AC3EDE3
:1043F8000E5A83ED0F6A87ED403AC3ED176AC3ED95
:10440800187AC4F80811731C03F01F03A4F81031BC
:10441800A8F80400059BFEF7B8BAA4F8003298463D
:10442800002F3FF4FDAD02207EE4069B5A8B904599
:10443800C0F2D283B8F5FA6FD4BFC2EB0803C2F555
:10444800FA634FF47A7101FB03F194F89001C2F515
:10445800FA63B1FBF3F200283FF472AA94F89131A1
:10446800894902FB03F281FB0213D217C2EB6312E4
:10447800FFF766BADFED857AFFF723BADFED837AB7
:10448800FFF701BAB8F5FA6F80F2A283297AA8EB90
:10449800020303FB01F3C2F5FA6293FBF2F3C3F1E3
:1044A800640307EE903A9FED7A7AF8EEE77A67EEC2
:1044B800877AC4ED487AFFF7C0B9764B1A78D4F8F2
:1044C8001871DFF8FCC19FED717AF8000CEB00035E
:1044D80083ED007A002A7BD06F49B0EE476AF0EE90
:1044E800476A0023F1EC017A013367EEA77A05EEFB
:1044F800903AB4EEE77AF1EE10FAF8EEE55AB8BF62
:10450800B0EE677A934276EEA76AA7EEA56AE9D17C
:10451800F5EEC06A0CEB0003F1EE10FA83ED007AB9
:1045280056DDC6EE265A5D4B5D4A1288F7EE007AD4
:1045380075EEE75AD3ED007A65EEA77AFDEEE77AD5
:1045480017EE903A812B42F375809342A8BF134629
:1045580007EE903AF8EEE77A524BC11903EB810364
:1045680093ED057AD3ED003A93ED066A93ED014A8F
:10457800D3ED046AD3ED034A93ED025AA3EEA77A6A
:10458800A4EE276A66EEC76AA7EE646ABDEEC77A2C
:10459800E5EE276A17EE101A812983ED056AC3ED47
:1045A800066A42F344808A42A8BF0A4607EE902A68
:1045B800F8EEE77AFCEEE77ACDED077ABDF81C3025
:1045C8000CEB000293801FB9BEF1130F02F0E386D3
:1045D800BEF1150F41F023816044DFF8E080838845
:1045E80028F81730D4F814612F4B013683FB0623C3
:1045F8009A19F317C3EBA203C3EBC303F61AC4F863
:1046080014612A4B1B78002B40F0A681284FDFF855
:10461800B49007F5F47607F51578F7EC017A95ED7F
:10462800080AD5F81432F8EEE77A304627EE800A01
:104638009847A6F1E000D5F834319847A6F1700004
:10464800D5F8A4319847D7F8F400D5F8B83098478A
:104658002436B045A9EC010ADFD1059B1E78FEF788
:10466800B9BB144B144A19681288144BC9691980CC
:104678005A8019B0BDEC0C8BBDE8F08F2C5C002083
:10468800D4470020684500201F85EB51000000003A
:104698000AD7233C4A450020BC1F00204C45002077
:1046A800484500206847002093244992404500204F
:1046B800CC540020444000204C2C0020305C0020CA
:1046C8004048002024570020DA4BDFF88C831B7801
:1046D80098F80020DE0700F18383002A00F0848523
:1046E800D54BD649D6480693920028F065F8D54BA5
:1046F800DFF868B3D44E0793FFF767B8B4F80082C1
:1047080008F1FF380FFA88F8B8F1000FA4F8008212
:104718003FF7D1AA002F7FF486AE81E4002800F08D
:104728004387B9F1000F42F0F182C848002F42F0E8
:104738009D8190ED006A9DED105AC14B25EE866A69
:10474800FDEEE44AA5EE076AB0EE675AA6EE265AD1
:1047580014EE901ABDEEC56A16EE10CA16EE107A5F
:10476800F445A8BF77466145C8BF0F4606EE107AE4
:10477800B8EEC66A012A83ED006A00F0DF8090ED8A
:10478800046A9DED115A25EE866AA5EE076AB0EE19
:10479800675AA6EE265ABDEEC56A16EE10CA16EE80
:1047A800107AF445A8BF77468C45B8BF0F4606EE89
:1047B800107AB8EEC66A022A83ED016A00F0BE805C
:1047C80090ED086A9DED125A25EE866AA5EE076AF5
:1047D800B0EE675AA6EE265ABDEEC56A16EE10CAA6
:1047E80016EE107AF445A8BF77468C45B8BF0F4639
:1047F80006EE107AB8EEC66A032A83ED026A00F064
:104808009D8090ED0C6A9DED135A25EE866AA5EE03
:10481800076AB0EE675AA6EE265ABDEEC56A16EECE
:1048280010CA16EE107AF445A8BF77468C45B8BF73
:104838000F4606EE107AB8EEC66A042A83ED036ABC
:104848007CD090ED106A9DED145A25EE866AA5EE8F
:10485800076AB0EE675AA6EE265ABDEEC56A16EE8E
:1048680010CA16EE107AF445A8BF77468C45B8BF33
:104878000F4606EE107AB8EEC66A052A83ED046A7A
:104888005CD090ED146A9DED155A25EE866AA5EE6A
:10489800076AB0EE675AA6EE265ABDEEC56A16EE4E
:1048A80010CA16EE107AF445A8BF77468C45B8BFF3
:1048B8000F4606EE107AB8EEC66A062A83ED056A38
:1048C8003CD090ED186A9DED165A25EE866AA5EE45
:1048D800076AB0EE675AA6EE265ABDEEC56A16EE0E
:1048E80010CA16EE107AF445A8BF77468C45B8BFB3
:1048F8000F4606EE107AB8EEC66A072A83ED066AF6
:104908001CD090ED1C6A9DED175A65EE865AE7EEAD
:10491800055AE6EEA57AFDEEE77A17EE900A864587
:10492800A8BF86468142D8BF714607EE901AF8EEB6
:10493800E77AC3ED077A002A3EF447AF92003F4971
:104948003F4827F039FF424B1B68002B3EF442AF2B
:1049580010F040FEFEF73EBF3E4E0694DFF8009191
:10496800DFF800A1059C06F5BC7800272378D5ED73
:10497800087A172B4DD096ED007AB8EEC78A082B27
:1049880028EE278A07D1B0EE480A079328F040F8A6
:10499800079B2AF81700DBF8002092000BD5002FA0
:1049A80002F0DC87B0EE480AD5F8143208F170003E
:1049B8009847B0EE408AB0EE480AD5F83431A8F1ED
:1049C80070009847D5F8A431404698472378032BC0
:1049D800B0EE408A18D0D6F8F800D5F8B830B0EE66
:1049E800480A98470137032F08F12408A9EC010A5F
:1049F80006F10406BAD1059B069C1E78FEF7EAB9B3
:104A0800F0EE676AFFF7AEB928F002F82AF8170047
:104A1800E1E796ED007A05EB4702B8EEC78A928F78
:104A28002AF8172028EE278AB5E7B0EE665AFEF76F
:104A380069BB00BFFC480020DC4C002090310020FE
:104A4800B4400020AC5F00204C5C002048270020C8
:104A58004C300020CC540020F05E0020305700205D
:104A680024570020305C0020CD4B0593CD4CC8E581
:104A7800AB68002B3EF4D4AECB49A1F15000984767
:104A8800DBF80090FEF7CCBE1D21C848FCF706FFF6
:104A9800002841F07783C64B03F1500203E004334A
:104AA8009A423EF474AF19782629F8D193F802E0B7
:104AB800D8788645F3D2BF4BDB78002B7EF467AFFE
:104AC800BA48FCF7EBFEDFEDBC7ABC49002802F0DF
:104AD8003A8438EE678AC7F57A72FDEEC87A12B260
:104AE800CDED077ABDF91C301B0381FB0301DB17F1
:104AF800C3EBA11302FB03F343F30F333B4407EE6D
:104B0800903AB8EEE78A012386ED038A84F8893162
:104B1800FEF73DBFAA4AA54BD2F8EC201B6844F625
:104B280020618A42A8BF0A46B2F57A7FB8BF4FF41F
:104B38007A7292B2D906A4F8D22144D5BBF1000FFB
:104B480001F06E859F4BD3F800E0BEF832004008B4
:104B58009A49D4F8D431D6ED037AA1FB021291090F
:104B6800642292FBF1F2142ABDEEE77A04EB430CBF
:104B7800A8BF142201339A42C4F8D43117EE108A20
:104B8800DCBF0023C4F8D43104EB4303ACF8D8816C
:104B9800B3F9D83107EE103AB8EEC77A77EEC77A8C
:104BA800FDEEE77ACDED0B7ABDF92C2082EAE273AF
:104BB800A3EBE273834201F3C086834A4FF07E532E
:104BC8001360FFF712B819F0805FB7D1FFF70DB87F
:104BD8002B7AC3F1640364E4594636E47B4A1278BD
:104BE80012F0100201F0F48294F8A411D4F8A8216C
:104BF80096ED017A00290CBF01214FF0FF3102FB2D
:104C080001F207EE902AF8EEE77A77EE877AC6ED9A
:104C1800017AFEF7C8BF1E216448FCF73FFE002852
:104C28003FF4FBA9079B002B7FF4F7A994F82432E3
:104C3800AB4242F0B281644BD4ED8A7AD3ED056A77
:104C480094ED4C5ADFED625A9FED626A27EEC57A01
:104C580068EE277AA8EE267AE5EE267AB4EEE57AAB
:104C6800F1EE10FA88BFB0EE657AB4EEC67AF1EECE
:104C780010FAF4EEE57AB8BFB0EE467AF1EE10FA23
:104C880088BFF0EE657AF4EEC67AF1EE10FAB8BF96
:104C9800F0EE467A84ED4A7AC4ED4C7AFFF7BDB956
:104CA800FDEEC87A4C4A17EE903AA2F80480D380F9
:104CB800FFF7ADB9DFED496AFFF72EBA1CF4800F94
:104CC8007EF42BACFEF72DBCBDEEE77A424B17EE17
:104CD800102A9A80FFF784B9B4EEC87AF1EE10FA78
:104CE80098BFB0EE478ABDEEC77AB4EEE68A3A4F6F
:104CF800F1EE10FA17EE103AB8BFB0EE668A84EDFE
:104D08004A8A3B8000287FF48AA8FFF780B99FED84
:104D1800307ADFED306A304AF4EEC77AF1EE10FAF5
:104D280098BFB0EE677AFDEEE77AB4EEE67AF1EE78
:104D380010FA17EE903AB8BFB0EE667A012884ED03
:104D48004B7A53803FF7D1A8FFF761B9002B3EF4A7
:104D580040A9FEF728B906F013FB059B08991B78B4
:104D68001D4A401A072B90807EF452AD06F008FBCE
:104D78000890FEF74FBD06F003FB059B0B9A1B78C6
:104D8800DFF85480801A012BA8F8020000F0E282B4
:104D9800072B7EF446A906F0F3FA0890FEF743B90C
:104DA8002C5C0020BC1F0020EC5400205442002042
:104DB800D04200207C3D002000007A44D34D621090
:104DC800900700206451002020000020784800202F
:104DD80000C0F94400C0F9C4305C002000000000A5
:104DE800002A00F00182D4ED543A94ED536AEB4B5B
:104DF800D4ED5E7AD3ED005A94ED5D7A94ED514A84
:104E0800D4ED504AE648E74BF4EEC63AF3EE046AAE
:104E1800F1EE10FA37EEA65A40F11C8390ED016AC4
:104E280026EE646AB0EE674AA6EE074AB4EEC54AB3
:104E380034EE666AF1EE10FA48BFB0EE656A012AF0
:104E480083ED006A00F0D08190ED056A26EE646A71
:104E5800B0EE674AA6EE074AB4EEC54A34EE666A73
:104E6800F1EE10FA48BFB0EE656A022A83ED016AD6
:104E780000F0BA8190ED096A26EE646AB0EE674ADE
:104E8800A6EE074AB4EEC54A34EE666AF1EE10FAA9
:104E980048BFB0EE656A032A83ED026A00F0A48178
:104EA80090ED0D6A26EE646AB0EE674AA6EE074AF0
:104EB800B4EEC54A34EE666AF1EE10FA48BFB0EEB9
:104EC800656A042A83ED036A00F08E8190ED116A09
:104ED80026EE646AB0EE674AA6EE074AB4EEC54A03
:104EE80034EE666AF1EE10FA48BFB0EE656A052A3C
:104EF80083ED046A00F0788190ED156A26EE646A05
:104F0800B0EE674AA6EE074AB4EEC54A74EE666A82
:104F1800F1EE10FA48BFF0EE656A062AC3ED056A9D
:104F280000F06281D0ED196A66EEE46AB0EE674A75
:104F3800A6EE874AB3EE046AB4EEC54A74EE466A32
:104F4800F1EE10FA48BFF0EE656A072AC3ED066A6B
:104F580000F04A81D0ED1D6A934A069266EEE44A53
:104F6800924ADFF850B2924E0792E4EE877AF4EE56
:104F7800C57A77EEC67AF1EE10FAB8BFF0EE657A28
:104F8800C3ED077AFEF721BCB9F1000F41F0D881D3
:104F980083489DED105A90ED006A824B25EE866A93
:104FA800A5EE076AB0EE675AA6EE265ABDEEC56AA8
:104FB80016EE10CA16EE107AF445A8BF774661457A
:104FC800C8BF0F4606EE107AB8EEC66A012A83ED0E
:104FD800006A3FF4B3AC90ED046A9DED115A25EEDA
:104FE800866AA5EE076AB0EE675AA6EE265ABDEEA7
:104FF800C56A16EE10CA16EE107AF445A8BF7746B1
:105008006145C8BF0F4606EE107AB8EEC66A022A96
:1050180083ED016A3FF492AC90ED086A9DED125A57
:1050280025EE866AA5EE076AB0EE675AA6EE265AFE
:10503800BDEEC56A16EE10CA16EE107AF445A8BF82
:1050480077466145C8BF0F4606EE107AB8EEC66AC5
:10505800032A83ED026A3FF471AC90ED0C6A9DED72
:10506800135A25EE866AA5EE076AB0EE675AA6EED1
:10507800265ABDEEC56A16EE10CA16EE107AF44529
:10508800A8BF77466145C8BF0F4606EE107AB8EE4E
:10509800C66A042A83ED036A3FF450AC90ED106AA7
:1050A8009DED145A25EE866AA5EE076AB0EE675A9A
:1050B800A6EE265ABDEEC56A16EE10CA16EE107A8E
:1050C800F445A8BF77466145C8BF0F4606EE107A7B
:1050D800B8EEC66A052A83ED046A3FF42FAC90ED5A
:1050E800146A9DED155A25EE866AA5EE076AB0EE9C
:1050F800675AA6EE265ABDEEC56A16EE10CA16EE17
:10510800107AF445A8BF77466145C8BF0F4606EE3A
:10511800107AB8EEC66A062A83ED056A3FF40EAC2B
:1051280090ED186A9DED165A25EE866AA5EE076A77
:10513800B0EE675AA6EE265ABDEEC56A16EE10CA3C
:1051480016EE107AF445A8BF77466145C8BF0F46EA
:1051580006EE107AB8EEC66A072A83ED066A3FF4AF
:10516800EDAB90ED1C6A9DED175A65EE865AE7EE99
:10517800055AE6EEA57AFDEEE77A17EE900A86451F
:10518800A8BF86468142C8BF8E4607EE90EAF8EE71
:10519800E77AC3ED077AFFF7CEBB00BF8C3100205A
:1051A80048270020B4400020DC4C0020AC5F0020E1
:1051B8004C5C0020305700200000C842B5EEC07A91
:1051C800F1EE10FA01F12382B7EE006A36EE477A63
:1051D800C6EE076AFEF76DBE5FED096AFEF7FBBE15
:1051E8001FED0B6AFEF7FFBD824B0693824BDFF87B
:1051F8005CB2824E0793FEF7E8BA814A5379002BD6
:105208003EF40CA87F4B1B78002B3EF407A81278BD
:10521800DFED7D4A07EE902A7C4AB8EE677A12885D
:1052280007EE903A06EE102AF8EEE77AB8EE466AEC
:1052380067EE277AB7EE007A87EE863AB4EEE43A5C
:10524800F1EE10FA88BFB0EE643AB4EEC73AF1EE68
:1052580010FAB8BFB0EE473AFDF7E2BFB4F8D22172
:1052680002F57A7292B2FEF7D4BC694B5A88FEF7FF
:10527800D0BC684B93ED006AFEF730BF664B9FEDDC
:10528800677AD3ED087AF4EEC77AF1EE10FA00F2F5
:105298000D859FED637AD6ED037A77EE877AC6EDB2
:1052A800037AFEF79DBC5F4E3278013A0A2A1CD871
:1052B800DFE812F0A40637076B064F061B001B0039
:1052C80039062307CD0610070B00574A574952687D
:1052D8000968C8328A4203D321F00CF828B1AB78A8
:1052E800032B02F02B8201233370EB78002B3EF462
:1052F8009FAE4F4B1B78DB0740F189864B4FD4F8A4
:1053080030223B689A4200F28E863378012B3EF4B5
:105318008FAE94F82C22002A3EF48AAE0B2B0DD8BF
:1053280001229A4040F6030112EA01050BD112F45A
:10533800C06F03D0093B012B42F258823A4B3A68BE
:105348005A600B233370002384F82C32FEF770BEAA
:10535800DFF8FC8006F014F8364AD4F86C3112688D
:105368000890C31A9A1AC4F86C01A8F80430A8F86F
:105378000620FDF758BE06F003F80B90FDF703BCB6
:105388002D4A927B002A3EF421ACFEF723BCB4F8E8
:105398007C3183420FD8294B03F1500003E00433DA
:1053A800984200F062871F78262FF8D193F802E020
:1053B800DF78BE45F3D294F88931002B40F0558749
:1053C8001F48204BD0ED007A93ED007A1E48C4EDBB
:1053D800607A77EE676AC4ED5E7A0123C4ED5D6A90
:1053E80084ED617A90ED007ADFED0D7A84F88831EA
:1053F800FDF74EBEDC4C0020AC5F00204C5C00206A
:105408006C3D00204A5C0020713DAA3FC85B00202B
:10541800DC51002048310020C82500208FC2753C8F
:1054280000000000CF360020604200209C59002078
:10543800FC480020B4420020B8530020D04200208D
:10544800C82700205C420020E427002030570020B5
:10545800305C002090ED026A26EE446AF0EE674A5E
:10546800E6EE074AF4EEC54A34EEE66AF1EE10FAC3
:1054780048BFB0EE656A012A83ED006A3FF4B4AE16
:1054880090ED066A26EE446AF0EE674AE6EE074AB1
:10549800F4EEC54A34EEE66AF1EE10FA48BFB0EE13
:1054A800656A022A83ED016A3FF49EAE90ED0A6AAE
:1054B80026EE446AF0EE674AE6EE074AF4EEC54A7D
:1054C80034EEE66AF1EE10FA48BFB0EE656A032AD8
:1054D80083ED026A3FF488AE90ED0E6A26EE446AC8
:1054E800F0EE674AE6EE074AF4EEC54A34EEE66A9D
:1054F800F1EE10FA48BFB0EE656A042A83ED036A3C
:105508003FF472AE90ED126A26EE446AF0EE674AF6
:10551800E6EE074AF4EEC54A34EEE66AF1EE10FA12
:1055280048BFB0EE656A052A83ED046A3FF45CAEB5
:1055380090ED166A26EE446AF0EE674AE6EE074AF0
:10554800F4EEC54A74EEE66AF1EE10FA48BFF0EEE2
:10555800656A062AC3ED056A3FF446AED0ED1A6ABD
:1055680066EEC46AF0EE674AE6EE874AB3EE046A6E
:10557800F4EEC54A74EEC66AF1EE10FA48BFF0EED2
:10558800656A072AC3ED066A3FF42EAED0ED1E6A9F
:10559800DF4A069226EEC44ADE4ADFF8A0B3DE4EA2
:1055A8000792E4EE077AE2E4DC48002F41F05880E5
:1055B80090ED006A9DED105AD94B25EE866AFDEEF6
:1055C800E44AA5EE076AB0EE675AA6EE265A14EE2C
:1055D800901ABDEEC56A16EE10CA16EE107AF4459A
:1055E800A8BF77466145C8BF0F4606EE107AB8EEE9
:1055F800C66A012A83ED006A3EF4E3A890ED046AC6
:105608009DED115A25EE866AA5EE076AB0EE675A37
:10561800A6EE265ABDEEC56A16EE10CA16EE107A28
:10562800F445A8BF77468C45B8BF0F4606EE107AFA
:10563800B8EEC66A022A83ED016A3EF4C2A890ED6C
:10564800086A9DED125A25EE866AA5EE076AB0EE45
:10565800675AA6EE265ABDEEC56A16EE10CA16EEB1
:10566800107AF445A8BF77468C45B8BF0F4606EEBA
:10567800107AB8EEC66A032A83ED026A3EF4A1A83E
:1056880090ED0C6A9DED135A25EE866AA5EE076A21
:10569800B0EE675AA6EE265ABDEEC56A16EE10CAD7
:1056A80016EE107AF445A8BF77468C45B8BF0F466A
:1056B80006EE107AB8EEC66A042A83ED036A3EF451
:1056C80080A890ED106A9DED145A25EE866AA5EE25
:1056D800076AB0EE675AA6EE265ABDEEC56A16EE00
:1056E80010CA16EE107AF445A8BF77468C45B8BFA5
:1056F8000F4606EE107AB8EEC66A052A83ED046AEC
:105708003EF45FA890ED146A9DED155A25EE866A61
:10571800A5EE076AB0EE675AA6EE265ABDEEC56A30
:1057280016EE10CA16EE107AF445A8BF77468C45D7
:10573800B8BF0F4606EE107AB8EEC66A062A83EDA1
:10574800056A3EF43EA890ED186A9DED165A25EEBE
:10575800866AA5EE076AB0EE675AA6EE265ABDEE2F
:10576800C56A16EE10CA16EE107AF445A8BF774639
:105778008C45B8BF0F46FEF702B86A4FD4ED017AE0
:1057880094ED006A38887B6977EEA77AF0EE006AB4
:10579800B0EE677AA6EE267A013804EBC002D6EEA0
:1057A800267A083A1033F6EE003A27EE237A67EEA7
:1057B800A37A84ED207AC4ED217A5B4C274604F164
:1057C800800192ED027A92ED036AD7ED036AD7ED74
:1057D800027A53ED014A13ED025A37EE674A76EE24
:1057E800C65A77EE277AE4EE845A0138A2F1080205
:1057F800E5EE047A07F1080703F1080336EE267A86
:1058080001F10801E4EE877AE5EE475A67EEA37ADC
:1058180025EEA37AC1ED007A81ED017AD1D1BEF1EE
:10582800140F7EF4E1AE05F0ABFD069BDFF81081A6
:10583800C01AA8F80200D4F81461FEF7D5BED4F84F
:105848001891B4F810C1394BCCF1200A5FFA8AFAE2
:105858000CEB491703EB87075FEA9A0301F0A98568
:10586800013318013249334A07EB000807F11003E6
:1058780013ED024A13ED035A13ED016A13ED047A8E
:1058880051ED024A51ED035A51ED016A51ED047A86
:1058980064EE244A65EE255A66EE266A67EE277A94
:1058A8001033984542ED024A42ED035A42ED016A2F
:1058B80042ED047A01F1100102F11002D8D11E491B
:1058C800A0F11002174401EB020822441AF0030366
:1058D80009D0B7EC017AF8EC017A67EE277A013B38
:1058E800E2EC017AF5D1BCF1000F41F03580BEF150
:1058F800140F7EF479AE05F043FD069BDFF8408077
:10590800D4F81461C01AA8F80200FEF76DBE00BFF3
:10591800DC4C0020AC5F00204C5C002048270020B5
:10592800B440002050450020BC1F002068450020DE
:10593800F8460020CC1F0020E84600203057002001
:10594800305C0020C94FCA48BA68B98925F01CFFE5
:10595800059B93F800E0BEF1140F01F04E85D4F8D2
:1059680014610136C4F8146108E7C04F39887A68B1
:105978004FEA51094FEA89005FEAD10804EB0003B6
:1059880004EB810600F0A28000F1100108F1010883
:10599800DFF8F8E203EB08183144103302F1100C79
:1059A80006F1100050ED032A50ED043A1EED043ABA
:1059B8001EED032A50ED026A10ED016A1EED021A6F
:1059C8005EED010A11ED044A11ED035A53ED044A44
:1059D80053ED035A13ED027A53ED017A51ED021A91
:1059E80011ED010A73EE238A32EE228A4EED048A03
:1059F8000EED038A71EE268A30EE868A4EED028A13
:105A08000EED018A74EE848A35EE858A43ED048AA8
:105A180003ED038A77EE218A37EE808A43ED028A06
:105A280003ED018A73EE633A75EE655A1CED035A6D
:105A380032EE623A74EE644A25EE638A1CED044A3B
:105A480023EE052A64EE652AA3EE048A10339845EE
:105A580024EE843AA3EE842A0EF1100E0CF1100CF9
:105A6800A5EE853A00F1100001F11001E4EE852A57
:105A780000ED078A00ED082A01ED073A41ED082AF2
:105A88005CED055A1CED065A71EE666A30EEC66A80
:105A980031EEC77A70EE677A26EE253A65EEE63A79
:105AA80025EE674A67EE054AE6EE053AA6EE853A20
:105AB800A7EE254AE7EEA54A00ED063A40ED053A7D
:105AC80001ED064A41ED054A7FF46CAF1FFA89F9EA
:105AD8004946674822F04AFE49467A68304622F02D
:105AE80045FE059B1B78142B7FF4A5AE9BE6614F02
:105AF8003A785FEA920C01F055855F480CF101098C
:105B08004FEA491900EB090800F12003A0F17001E0
:105B180013ED076A53ED056A13ED037A53ED017A25
:105B280053ED025A13ED084A53ED064A13ED045A91
:105B380026EE066A66EEA66A27EE077A67EEA77A69
:105B4800A4EE046A20339845E4EEA46A01F110013A
:105B5800A5EE057AE5EEA57AF1EEC65AB1EEE66A4B
:105B6800F1EEC76AB1EEE77A41ED085A01ED076A2E
:105B780041ED066A01ED057ACAD1A9F12003034473
:105B880004EB0C1012F0030118BF08330FD053EDCB
:105B9800017A13ED027A67EEA77A0139E7EE077A00
:105BA80003F10803B1EEE77AA0EC017AEFD1BEF178
:105BB800140F01F005840136C4F81461FEF77FBCA8
:105BC800D4F818212D4B2E492E4E1846D3001944CF
:105BD8001A448B88016800EE103A10EE103A643BC4
:105BE800C82BA8BFC823782BB8BF782307EE903AF4
:105BF800B8EEC07AF8EEE77A06EB820677EE670A27
:105C080077EE876A67EE877A20EEA67AB8EE400AC2
:105C1800C7EE870A3046D6F814A0D6F81890D6F8FA
:105C28001C80376A23F082F8059BC6F814A093F805
:105C380000E0C6F81890BEF1140FC6F81C80376251
:105C480001F0CE83D4F818310F4AD4F81461013327
:105C580082FB0312A2EBE37909EB4902A3EB0209E9
:105C68000136C4F81891C4F81461EAE550450020DB
:105C7800BC1F00204A4500203C200020205700205F
:105C880040480020B456002056555555CC1F0020DA
:105C9800306E99BC2716983DA40DC93F843459BE6F
:105CA800DB0F4940D06D393A00000000F0EEE76A9A
:105CB800B7EE005A35EE665A1FED0B4A5FED0B5AE8
:105CC8001FED0A6A1FED0C7A94ED730AF1EEC54ACE
:105CD800E6EE845AF5EEC07AA6EEA56AF1EE10FA61
:105CE800A6EE867A48BF5FED127A27EE247A48BF7F
:105CF80037EEC77A27EE000A26F08AFEB0F5617FF4
:105D080000F39A8607EE900AF8EEE76A5FED1B7AD1
:105D180066EEA76A07EE907ABDEEE67AF8EEE77AC5
:105D280017EE103A2033402B41F24D841FED220A22
:105D380026F06EFE00B207EE900AB8EEE77AFFF79B
:105D4800AABAD44B9AED007AD3ED006AB0EEC77ABE
:105D5800B4EEE67AF1EE10FA7DF73BA9FDF736B915
:105D6800CD4FDFF8689397ED004A97ED057AD7EDA8
:105D7800014A97ED066AD7ED046A97ED035AD7ED05
:105D8800025A67EE897A09EB8603A4EE277AA4EE15
:105D9800A76A66EEC76AA5EE476AE5EEA76A20EE2F
:105DA800070A87ED056AC7ED066A29EE088A69EED3
:105DB800288A83ED007A26F02BFED7ED0E5AD7ED10
:105DC800176A97ED091AD7ED121A97ED0F5A97ED42
:105DD800187A97ED0A2AD7ED132A97ED0D6AD7EDB1
:105DE800167A97ED0C3AD7ED0B3A97ED154AD7EDA1
:105DF800144AE1EE085A002209EB8601E8EEA16A8E
:105E080000B2C4F80021A2EE085AC4F80421C4F86C
:105E18000821A8EEA27A26EE656A67EEE67AA3EE76
:105E2800655AA3EE886AA6EEC47AE8EEA47A87EDEE
:105E38000E5AC1ED205A87ED0F6AC1ED406A87ED11
:105E4800177AC7ED187AFEF7DEBAB5F93C306A6200
:105E580007EE903A0122F8EEE77AEB66C5F888205B
:105E68000023012FC5ED1F7AC5ED1E7AC5F88030D5
:105E780001F06582A7427CF4F4ADB5F93E302B679A
:105E880007EE903A00220123F8EEE77AAA62C5F8F5
:105E98009C300023012FC5ED247AC5ED237AC5F87F
:105EA800943001F04882A7427CF40CAEB5F940303A
:105EB8006B6707EE903A00220123F8EEE77AEA6270
:105EC800C5F8B0300023012FC5ED297AC5ED287A31
:105ED800C5F8A8307CF427AE9FED708A032E1CD03D
:105EE800B9F1000F09D007EE909AF8EEE77AF4EED0
:105EF800C87AF1EE10FA01F1AC83694A6B6F126847
:105F0800A8F80600002103EB540393FBF4F4EC62B9
:105F180091621163D162FCF708BEB0EE480A26F020
:105F280077FD00B2DCE720F0C3F95E4B00210520C5
:105F38008DE80300A3F108020291532018F046FEF1
:105F480000287FF4D2A9584A082310603370FFF75D
:105F5800CCB920F0ADF9554A0292A2F10C032621E2
:105F680001930091A2F10A035021163A492018F032
:105F78002DFE00287FF4B9A94B4B4FF0FF310722C3
:105F8800186059603270FFF7B0B9DFF81C8120F053
:105F98008FF9474AD8F80430126864339342BFF443
:105FA800A4A9402020F068F900287FF49EA9D8F819
:105FB8000030404FDFF818A14FF040090FE020F003
:105FC800BDF9DAF80020D8F80030013A0133B9F108
:105FD8000109CAF80020C8F8003001F0BE83FB5C54
:105FE8001846002BEBD100234FF0FF32C8F80030E1
:105FF8000423C8F804203370FFF777B92E4B1B78B9
:10600800DA0701F12C83EB78002B3EF411A80CF091
:1060180017FB00283FF472A9254B1B6803F59C5316
:106028000833C4F830323378012B7EF401A894F891
:106038002C32002B7DF4FCAFAB78032B01F093835B
:1060480018F08EFE012384F82C32FDF7F1BF1A20D8
:1060580012F026F8D0B1194B1B88BBB9184B452054
:106068001F6820F06BF90E2020F068F9384617F009
:1060780051FD099F384617F04DFD124A124B126820
:106088001A6038460A23337017F0B4FD18F072F816
:10609800FFF72BB980310020D44700200000000012
:1060A800444000201CDF02086042002062DD020834
:1060B8009C590020FCDC0208FC480020D840002045
:1060C800D4400020E8400020E0400020684500203F
:1060D800AC530020874B1B78002B01F027811A2036
:1060E80011F0DEFF002841F0218194F82C32002BBA
:1060F80041F01C8109233370C8E720F0D9F818F063
:106108006FF800283FF4F1A820F0F4F800283FF4D5
:10611800ECA8794A794B12681A600A233370FFF7A2
:10612800E4B8774B774A1B685360774900231360BC
:1061380003220B603270FFF7D8B8744B7448D3ED64
:10614800006A744B90ED006A1B78C4ED606A84EDB8
:10615800616A002B00F05F8276EE665ABCEEC76A71
:106168006D48C4ED5D5A16EE103AC4ED5E6AA4F8A7
:106178007C31FF2377EEC77A90ED007A84F8883176
:10618800FCF786BF654BDB78002B7EF484ACDFED33
:10619800647A644938EE678AC7F5FA63FDEEC87A0F
:1061A8001BB2CDED077ABDF91C20120381FB020159
:1061B800D217C2EBA11203FB02F343F30F333B44A4
:1061C80007EE903AB8EEE78A86ED038AFEF763BCDD
:1061D8009AF80300B4F9AC11002800F07F83A8EB0B
:1061E800010E9AF802008EEAEE77A7EBEE77874267
:1061F80040F3B9868845C8BF404207EE900AF8EEDA
:10620800E77A012737EE888AC4F8B02184F8B47198
:1062180086ED038AFDF7C7BC434BDFED447A1B6864
:10622800C4ED497A13F0805A40F0E9831CF4800ADF
:1062380000F004824FF0000AB6EE007A67EE877A23
:10624800F4EEE75AF1EE10FA48BFF0EE675A40F163
:10625800D683C4ED635AFDF764B9354B1978354BCD
:10626800079301F00109FDF7ACBA284B2848D3ED94
:10627800007A284B90ED007A1B78C4ED607A84EDA3
:10628800617A002B00F0548377EE676A2248C4EDE8
:106298005E7AC4ED5D6AFF2390ED007ADFED267A21
:1062A80084F88831FCF7F4BE05F06AF8059B06907F
:1062B80093F800E0BEF1140F05BFDFF88080D4F832
:1062C8001461D4F81461A8F80060FCF768BB73EE99
:1062D800C67AB7EE007AF4EEC77AF1EE10FAC4ED9A
:1062E800497A41F3508084EEA77A8DED107AFDF754
:1062F8000EB900BF20430020E8400020E040002005
:106308009C59002060420020AC530020F44000203B
:10631800CC27002094490020E02700207C3D002065
:1063280000007A44D34D62105442002000000080DF
:10633800FC480020AC5F002000000000305C00201A
:10634800C3480C9B9DED105A90ED006A002B00F09D
:10635800D58625EE866ABF4BA5EE076AB0EE675A6A
:10636800A6EE265ABDEEC56A16EE10CA16EE107ACB
:10637800F445A8BF77466145C8BF0F4606EE107AB8
:10638800B8EEC66A012A83ED006A3DF41EAA90EDB4
:10639800046A9DED115A25EE866AA5EE076AB0EEED
:1063A800675AA6EE265ABDEEC56A16EE10CA16EE54
:1063B800107AF445A8BF77466145C8BF0F4606EE78
:1063C800107AB8EEC66A022A83ED016A3DF4FDA987
:1063D80090ED086A9DED125A25EE866AA5EE076AC9
:1063E800B0EE675AA6EE265ABDEEC56A16EE10CA7A
:1063F80016EE107AF445A8BF77466145C8BF0F4628
:1064080006EE107AB8EEC66A032A83ED026A3DF4F6
:10641800DCA990ED0C6A9DED135A25EE866AA5EE6F
:10642800076AB0EE675AA6EE265ABDEEC56A16EEA2
:1064380010CA16EE107AF445A8BF77466145C8BF62
:106448000F4606EE107AB8EEC66A042A83ED036A90
:106458003DF4BBA990ED106A9DED145A25EE866AAD
:10646800A5EE076AB0EE675AA6EE265ABDEEC56AD3
:1064780016EE10CA16EE107AF445A8BF77466145A5
:10648800C8BF0F4606EE107AB8EEC66A052A83ED35
:10649800046A3DF49AA990ED146A9DED155A25EE0B
:1064A800866AA5EE076AB0EE675AA6EE265ABDEED2
:1064B800C56A16EE10CA16EE107AF445A8BF7746DC
:1064C8006145C8BF0F4606EE107AB8EEC66A062ABE
:1064D80083ED056A3DF479A990ED186A9DED165A89
:1064E80025EE866AA5EE076AB0EE675AA6EE265A2A
:1064F800BDEEC56A16EE10CA16EE107AF445A8BFAE
:1065080077466145C8BF0F4606EE107AB8EEC66AF0
:10651800072A83ED066A3DF458A990ED1C6A9DEDA3
:10652800175A65EE865AE7EE055AE6EEA57AFDEEAD
:10653800E77A17EE902A9645A8BF96468A42A8BFE2
:10654800714607EE901AF8EEE77AC3ED077AFDF781
:106558003CB901297FF7C0AC07EE10EAB8EEC77A5C
:10656800C7EE876AB1EEE68AB8E4012940F3E3860C
:1065780007EE10EAB8EEC77AC7EE876AB1EEE68A88
:10658800032E13D0B9F1000F09D007EE909AF8EE58
:10659800E77AF4EEC87AF1EE10FA01F15A802B6F1F
:1065A80003EB540393FBF4F3AB627CE4B0EE480ACC
:1065B80026F02EFA00B2E5E7012940F3C08607EE7F
:1065C80010EAB8EEC77AC7EE876AB1EEE68A032EFC
:1065D80013D0B9F1000F09D007EE909AF8EEE77AD8
:1065E800F4EEC87AF1EE10FA01F13380EB6E03EBAA
:1065F800540393FBF4F36B623CE4B0EE480A26F0D4
:1066080007FA00B2E5E7F7EE006AFDF7E4BCF7EE3B
:10661800006AFDF74EBC76EEC65AF0EE466A9DE576
:106628000D4BD3F800E0BEF93200FEF791BA822391
:10663800FDF7C6BFDFED097AFDF78EBFB6EE007A2B
:10664800F4EEC75AF1EE10FA3FF7F6ADFCF769BF62
:1066580048270020B4400020645100200000024375
:1066680090ED006A9DED104AEB4B25EE866AFDEE33
:10667800E43AA4EE076AB0EE674AA6EE264A13EE9D
:10668800901AB4EEC45AF1EE10FAB0EE446A88BF1C
:10669800B0EE646ABDEEC66A16EE10CA16EE107A3F
:1066A800F445A8BF77466145C8BF0F4606EE107A85
:1066B800B8EEC66A012A83ED006A3DF482A890ED1F
:1066C800046A9DED114A25EE866AA4EE076AB0EECB
:1066D800674AA6EE264AB4EEC45AF1EE10FAB0EEB6
:1066E800446A88BFB0EE646ABDEEC66A16EE10CA88
:1066F80016EE107AF445A8BF77468C45B8BF0F460A
:1067080006EE107AB8EEC66A022A83ED016A3DF4F5
:1067180058A890ED086A9DED124A25EE866AA4EE07
:10672800076AB0EE674AA6EE264AB4EEC45AF1EEFE
:1067380010FAB0EE446A88BFB0EE646ABDEEC66A6D
:1067480016EE10CA16EE107AF445A8BF77468C45A7
:10675800B8BF0F4606EE107AB8EEC66A032A83ED74
:10676800026A3DF42EA890ED0C6A9DED134A25EEC1
:10677800866AA4EE076AB0EE674AA6EE264AB4EE29
:10678800C45AF1EE10FAB0EE446A88BFB0EE646AFB
:10679800BDEEC66A16EE10CA16EE107AF445A8BF0A
:1067A80077468C45B8BF0F4606EE107AB8EEC66A33
:1067B800042A83ED036A3DF404A890ED106A9DED68
:1067C800144A25EE866AA4EE076AB0EE674AA6EE7A
:1067D800264AB4EEC45AF1EE10FAB0EE446A88BF05
:1067E800B0EE646ABDEEC66A16EE10CA16EE107AEE
:1067F800F445A8BF77468C45B8BF0F4606EE107A19
:10680800B8EEC66A052A83ED046A3CF4DAAF90ED67
:10681800146A9DED154A25EE866AA4EE076AB0EE65
:10682800674AA6EE264AB4EEC45AF1EE10FAB0EE64
:10683800446A88BFB0EE646ABDEEC66A16EE10CA36
:1068480016EE107AF445A8BF77468C45B8BF0F46B8
:1068580006EE107AB8EEC66A062A83ED056A3CF49D
:10686800B0AF90ED186A9DED164A25EE866AA4EE43
:10687800076AB0EE674AA6EE264AB4EEC45AF1EEAD
:1068880010FAB0EE446A88BFB0EE646ABDEEC66A1C
:1068980016EE10CA16EE107AF445A8BF77468C4556
:1068A800B8BF0F4606EE107AB8EEC66A072A83ED1F
:1068B800066A3CF486AF90ED1C6A9DED174A65EEBA
:1068C800865AE7EE045AE6EEA57AB4EEE75AF1EEF8
:1068D80010FAC8BFF0EE647AFCF763BFA8EB0102B8
:1068E8009AF8027082EAE27EAEEBE27EBE4540F3A1
:1068F800468302EBD27201205210C4F8C02184F8FA
:10690800C40184F8B401D4F8A8210A44B2F5FA6F96
:10691800A8BF4FF4FA62B2F57A7FB8BF4FF47A7223
:1069280007EE902AF8EEE77AC6ED037AFDF73BB951
:1069380077EEC76AF0EE477AA8E4BEF834309FEDE8
:10694800377A07EE903AF8EEE77A354B67EE877AB2
:10695800C3ED007AFDF749B9324B4FEA8A075FEA7F
:106968009C0A394403EBC919274437D00AF1010AB4
:106978004FEA0A1A09EB0A0809F1100301F110009D
:1069880007F1100213ED024A13ED035A13ED016AE1
:1069980013ED047A50ED024A50ED035A50ED016AA6
:1069A80050ED047A64EE244A65EE255A66EE266AAE
:1069B80067EE277A1033984542ED024A42ED035AB2
:1069C80042ED016A42ED047A00F1100002F1100272
:1069D800D8D1AAF1100AD144514457441CF0030CF1
:1069E8003EF485AFB9EC017AF1EC017A67EE277ACB
:1069F800BCF1010CE7EC017AF4D1FEF778BFB7EEF1
:106A0800007A77EE677AF4EEE75AF1EE10FA88BF6B
:106A1800F0EE675A1DE400BFB44000206F12833ABD
:106A2800200000206845002084F9223F92E741B900
:106A38009730083C15A82ABE07EE907A5FED066AE3
:106A4800F8EEE77A66EEA65A1FED085A1FED086AB7
:106A58001FED087AA5EE856A26EEA55AA5EE867A78
:106A6800E5EE076A26EEA70AFFF762B990ED006A1D
:106A78009DED104AA44B25EE866AFDEEE43AA4EE9D
:106A8800076AB0EE674AA6EE264A13EE907AB4EE8D
:106A9800C45AF1EE10FAB0EE446A88BFB0EE646AE8
:106AA800BDEEC66A16EE10CA16EE101AF445A8BF57
:106AB80071466745C8BF394606EE101AB8EEC66A71
:106AC800012A83ED006A3DF439AF90ED046A9DED2B
:106AD800114A25EE866AA4EE076AB0EE674AA6EE6A
:106AE800264AB4EEC45AF1EE10FAB0EE446A88BFF2
:106AF800B0EE646ABDEEC66A16EE10CA16EE101A3B
:106B0800F445A8BF7146BC45B8BF394606EE101A11
:106B1800B8EEC66A022A83ED016A3DF40FAF90ED24
:106B2800086A9DED124A25EE866AA4EE076AB0EE61
:106B3800674AA6EE264AB4EEC45AF1EE10FAB0EE51
:106B4800446A88BFB0EE646ABDEEC66A16EE10CA23
:106B580016EE101AF445A8BF7146BC45B8BF3946B1
:106B680006EE101AB8EEC66A032A83ED026A3DF4EF
:106B7800E5AE90ED0C6A9DED134A25EE866AA4EE0B
:106B8800076AB0EE674AA6EE264AB4EEC45AF1EE9A
:106B980010FAB0EE446A88BFB0EE646ABDEEC66A09
:106BA80016EE10CA16EE101AF445A8BF7146BC4579
:106BB800B8BF394606EE101AB8EEC66A042A83ED45
:106BC800036A3DF4BBAE90ED106A9DED144A25EEC4
:106BD800866AA4EE076AB0EE674AA6EE264AB4EEC5
:106BE800C45AF1EE10FAB0EE446A88BFB0EE646A97
:106BF800BDEEC66A16EE10CA16EE101AF445A8BF06
:106C08007146BC45B8BF394606EE101AB8EEC66ADA
:106C1800052A83ED046A3DF491AE90ED146A9DED6A
:106C2800154A25EE866AA4EE076AB0EE674AA6EE14
:106C3800264AB4EEC45AF1EE10FAB0EE446A88BFA0
:106C4800B0EE646ABDEEC66A16EE10CA16EE101AE9
:106C5800F445A8BF7146BC45B8BF394606EE101AC0
:106C6800B8EEC66A062A83ED056A3DF467AE90ED74
:106C7800186A9DED164A25EE866AA4EE076AB0EEFC
:106C8800674AA6EE264AB4EEC45AF1EE10FAB0EE00
:106C9800446A88BFB0EE646ABDEEC66A16EE10CAD2
:106CA80016EE101AF445A8BF7146BC45B8BF394660
:106CB80006EE101AB8EEC66A072A83ED066A3DF496
:106CC8003DAE90ED1C6A9DED174A65EE865AE7EEDB
:106CD800045AE6EEA57AB4EEE75AF1EE10FAC8BF08
:106CE800F0EE647AFDEEE77A17EE901A8E45A8BFAB
:106CF8008E468F42D8BF774607EE907AF8EEE77A4D
:106D0800C3ED077AFDF717BEB44000200C9B002B9B
:106D180000F08C83E8489DED104A90ED006A25EE5E
:106D2800866AA4EE076AB0EE674AA6EE264AB0EE77
:106D3800446A37B1B4EE445AF1EE10FAC8BFB0EE67
:106D4800646AFDEEE44ABDEEC66A14EE909A16EE49
:106D5800101A894514EE90CA00F3D9847145A8BF6A
:106D6800714606EE101AD54BB8EEC66A012A83EDB5
:106D7800006A3CF42AAD90ED046ADDED114A25EE77
:106D8800866AA4EE876AF0EE674AE6EE264AB0EE17
:106D9800646A002F00F0A584B4EEE45AF1EE10FA0C
:106DA80040F39F8449467145A8BF714606EE101A04
:106DB800B8EEC66A022A83ED016A3CF406AD90ED8E
:106DC800086ADDED124A25EE866AA4EE876AF0EEBF
:106DD800674AE6EE264AB0EE646A002F00F0778430
:106DE800B4EEE45AF1EE10FA40F371844946714565
:106DF800A8BF714606EE101AB8EEC66A032A83EDDC
:106E0800026A3CF4E2AC90ED0C6ADDED134A25EE23
:106E1800866AA4EE876AF0EE674AE6EE264AB0EE86
:106E2800646A002F00F04984B4EEE45AF1EE10FAD7
:106E380040F3438449467145A8BF714606EE101ACF
:106E4800B8EEC66A042A83ED036A3CF4BEAC90ED42
:106E5800106ADDED144A25EE866AA4EE876AF0EE24
:106E6800674AE6EE264AB0EE646A002F00F01B84FB
:106E7800B4EEE45AF1EE10FA40F315844946714530
:106E8800A8BF714606EE101AB8EEC66A052A83ED49
:106E9800046A3CF49AAC90ED146ADDED154A25EECF
:106EA800866AA4EE876AF0EE674AE6EE264AB0EEF6
:106EB800646A002F00F0EE83B4EEE45AF1EE10FAA3
:106EC80040F3E88349467145A8BF714606EE101A9B
:106ED800B8EEC66A062A83ED056A3CF476AC90EDF6
:106EE800186ADDED164A25EE866AA4EE876AF0EE8A
:106EF800674AE6EE264AB0EE646A002F00F0C183C6
:106F0800B4EEE45AF1EE10FA40F3BB8349467145FA
:106F1800A8BF714606EE101AB8EEC66A072A83EDB6
:106F2800066A3CF452AC90ED1C6ADDED174A65EE3A
:106F3800865AE4EE875AE5EEA67A002F00F0998388
:106F4800F4EEC57AF1EE10FA40F193834A467245A1
:106F5800A8BF7246944607EE90CAF8EEE77AC3EDEA
:106F6800077AFCF732BC94F8B40100283FF4CBACA4
:106F7800D4F8BC0184F8B421C4F8B801C3E494F887
:106F8800B421002A3FF4BFACD4F8BC2184F8C40172
:106F980084F8B401C4F8B821B5E407EE905ADFEDDF
:106FA800486A9FED487A84F82452F8EEE77A67EE4B
:106FB800A67A77EE876ABDEEE66A16EE103A2033B7
:106FC800402B40F2A582DFED406A404BBDEEE77AE8
:106FD800C3ED056A17EE103A2033402B00F2DF822A
:106FE8009FED3B7AF4EEC77AF1EE10FA40F3938303
:106FF800DFED385A9FED386A01E0F0EE477AF4EE9B
:10700800C67AF1EE10FA37EEE57AF6DCDFED337A80
:10701800B4EEE77AF1EE10FA40F18083DFED2D5AF5
:107028009FED2F6A01E0B0EE677AB4EEC67AF1EE12
:1070380010FA77EE257AF6D49FED227AF4EEC77A25
:10704800F1EE10FA40F3B3829FED217A77EE677A7A
:1070580067EEA75A9FED235A9FED236A9FED237A87
:10706800A5EE856A27EEA55AA5EE867AE5EE077A9B
:10707800C4ED8A7AFDF7E4BD96ED000A0B9325F07E
:10708800C7FC1B4A1B49D2F8EC20DFF86CE081FBF7
:107098000231D217C2EBA11207EE902AF8EEE77A76
:1070A800AEF80000FDEEE77A0B9B17EE902AAEF8DB
:1070B8000220FCF7FCBD00BF48270020B440002098
:1070C80035FA8E3CDB0FC93F00000000200000208D
:1070D800DB0F4940DB0FC940E4CB1641DB0F49C049
:1070E800E4CB16C192E741B99730083C15A82ABEEF
:1070F80090070020D34D6210305C002025EE866A90
:10710800A5EE076AB0EE675AA6EE265ABDEEC56A26
:1071180016EE103A994200F37F817345A8BF734673
:1071280006EE103AB8EEC66ABAF1000F00F02F83E7
:10713800E64B012A83ED006A3CF447AB90ED046A04
:107148009DED115A25EE866AA5EE076AB0EE675ADC
:10715800A6EE265ABDEEC56A16EE107AB94200F3BD
:1071680059817745A8BF774606EE107AB8EEC66A09
:10717800BAF1000F00F00C84022A83ED016A3CF496
:1071880024AB90ED086A9DED125A25EE866AA5EEAD
:10719800076AB0EE675AA6EE265ABDEEC56A16EE25
:1071A800107AB94200F340817745A8BF774606EECA
:1071B800107AB8EEC66ABAF1000F00F0DC82032A32
:1071C80083ED026A3CF401AB90ED0C6A9DED135A15
:1071D80025EE866AA5EE076AB0EE675AA6EE265A2D
:1071E800BDEEC56A16EE107AB94200F31B817745E9
:1071F800A8BF774606EE107AB8EEC66ABAF1000F55
:1072080000F0E882042A83ED036A3CF4DEAA90EDDC
:10721800106A9DED145A25EE866AA5EE076AB0EE4F
:10722800675AA6EE265ABDEEC56A16EE107AB9421E
:1072380000F3F6807745A8BF774606EE107AB8EED9
:10724800C66ABAF1000F00F0B982052A83ED046A14
:107258003CF4BBAA90ED146A9DED155A25EE866A9A
:10726800A5EE076AB0EE675AA6EE265ABDEEC56AC5
:1072780016EE107AB94200F3D1807745A8BF774659
:1072880006EE107AB8EEC66ABAF1000F00F08A82EC
:10729800062A83ED056A3CF498AA90ED186A9DEDDC
:1072A800165A25EE866AA5EE076AB0EE675AA6EE6C
:1072B800265ABDEEC56A16EE107AB9427EDC7745CD
:1072C800A8BF774606EE107AB8EEC66ABAF1000F84
:1072D80000F09A82072A83ED066A3CF476AA90EDBC
:1072E8001C6A9DED175A65EE865AE5EE075AE5EEDB
:1072F800A67AFDEEE77A17EE902A8A4203DB7245FA
:10730800A8BF7246114607EE901AF8EEE77ABAF16E
:10731800000F7FF424AEBCF1000F7FF420AE0D9A6D
:107328000E998A42B8BFF0EE647A18E6099816F00A
:1073380061FCFEF7ABBE9FED758AFFF721B99FEDA3
:10734800738AFFF744B938EE678A84F88901FDEE3D
:10735800C87AC7F5FA62CDED077ABDF91C301B0370
:1073680081FB0301DB1712B2C3EBA11302FB03F38A
:1073780043F30F333B4407EE903AB8EEE78A86EDC5
:10738800038AFCF704BB524B1B6813F0805A7EF447
:1073980053AFFEF74BBF9FED4F0ADFF8488125EE4C
:1073A800800A25F035FBD4F81461A8F80600FDF72B
:1073B8001BB94949494A8846FEF788BA0F4681E70A
:1073C80003F0DEFF059BDFF81C8193F800E0069BC5
:1073D8003A78D4F81461C01AA8F80400FEF7EBBB99
:1073E80003F0CEFF059BDFF8FC8093F800E0069BD6
:1073F800C01AA8F80200FEF725BC03F0C1FF059BE0
:10740800DFF8E08093F800E0069BC01AA8F80200B5
:10741800FEF7A5BA0F46A7E60B4681E60F462FE70B
:107428000F460AE70F46E5E60F46C0E610AB03EB4A
:107438008202BDEEE46ACDF82CE09646284923483E
:107448000C94524616EE109A0F96F24605E05345F4
:10745800A0EC016A01F1100134D091ED006AB3EC9F
:10746800014A25EE866AA7EE046AB0EE674AA6EEE0
:10747800864AB0EE446A37B1B4EE445AF1EE10FAD7
:10748800C8BFB0EE646ABDEEC64A06EE109A14EEA6
:10749800104AA14507DC14EE104A0B9EB442A8BF5F
:1074A800344606EE104AB8EEC66A002ACFD1BCF1BF
:1074B800000FCCD10D9CA6460E9CA645B8BFB0EED9
:1074C800646AC4E70C9C0F9EFCF77FB9B4400020A7
:1074D800544200200000C842E8460020BC1F00209B
:1074E80048270020305C0020E4CB1641DB0F49C060
:1074F800DB0FC940E4CB16C1DB0FC93FDB0F4940A6
:1075080092E741B99730083C15A82ABE0000000050
:10751800F4EEC77AF1EE10FA40F303815FED0C5AEE
:107528001FED0F6A01E0F0EE476AF4EEC66AF1EE6D
:1075380010FA36EEE57AF6DC5FED146AB4EEE67A18
:10754800F1EE10FA40F1F7805FED175A1FED176A58
:1075580001E0B0EE667AB4EEC67AF1EE10FA77EE94
:10756800256AF6D41FED1C7AF4EEC76AF1EE10FA1C
:1075780040F3C1801FED1F7A77EE666A66EEA65A61
:107588001FED215A1FED216A1FED217AA5EE856AAC
:1075980026EEA55AA5EE867AE5EE076A15E55FEDB3
:1075A800257A65E5D64800F18003FEF7EBBA9FED32
:1075B800D57AF4EEC77AF1EE10FA44BF9FEDD27A8D
:1075C80077EE677A44E59FEDD17AF4EEC76AF1EE7B
:1075D80010FA40F32881DFEDCE5A9FEDCE6A01E024
:1075E800F0EE476AF4EEC66AF1EE10FA36EEE57A86
:1075F800F6DCDFEDC56AB4EEE67AF1EE10FA40F19A
:107608000F81DFEDC35A9FEDC46A01E0B0EE667AE0
:10761800B4EEC67AF1EE10FA77EE256AF6D49FED4D
:10762800BF7AF4EEC76AF1EE10FA05DD9FEDB77A7E
:1076380077EE666AFFF706BA9FEDB27AF4EEC76A8C
:10764800F1EE10FA44BF9FEDB07A77EE666AFFF765
:10765800F9B9A8F80600A5F8B440FBF76BBA802082
:107668001BF03CFA08B10BF03BFE17F079FBFDF775
:107678003CBEFDEEE77A17EE902A4A45FFF66BAC62
:1076880065E4BDEEC66A16EE101A4945BFF63FAC72
:1076980049463FE4BDEEC66A16EE101A4945BFF6E4
:1076A80012AC494612E4BDEEC66A16EE101A4945F8
:1076B800BFF6E5AB4946FFF7E5BBBDEEC66A16EE79
:1076C800101A4945BFF6B7AB4946FFF7B7BBBDEE41
:1076D800C66A16EE101A4945BFF689AB4946FFF748
:1076E80089BBBDEEC66A16EE101A4945BFF65BABFC
:1076F8004946FFF75BBB9FED837AF4EEC76AF1EE6C
:1077080010FA44BF9FED807A77EE666A36E714EE8A
:10771800901AFFF726BBB0EE677A77E4F0EE477A67
:107728008AE4B0EE667A07E794F86831002B7BF4B8
:1077380070ACFBF75BBCF0EE476A13E7784F38682C
:1077480022F07EFA774B1B780022022B3A607DF4F8
:10775800CAAD0BF0DDFDFDF7C6BDFB5C002B7DF46B
:10776800C4ADFEF740BC80201BF0B8F900287CF4BB
:107778005FACFEF765BCBCF1000F7FF420AD0D9F38
:10778800B9460E9FB945B8BFB0EE646A17E5BCF1BB
:10779800000F7FF4CDAC0D9B0E9FBB42B8BFB0EE7F
:1077A800646AC5E4BCF1000F7FF472AD0D9FB94661
:1077B8000E9FB945B8BFB0EE646A69E5BCF1000F29
:1077C8007FF443AD0D9FB9460E9FB945B8BFB0EEE3
:1077D800646A3AE5BCF1000F7FF414AD0D9FB94619
:1077E8000E9FB945B8BFB0EE646A0BE545201EF0A0
:1077F800A5FDFF201EF0A2FD4B481EF08BFD28467C
:107808001EF09CFDFDF79ABDBCF1000F7FF462AD40
:107818000D9FB9460E9FB945B8BFB0EE646A59E5E9
:10782800F0EE476AFBE6B0EE667AE2E63F4A404B86
:1078380010681B6898473F4BDBED007A93ED007AA0
:107848003D4BD8ED006A83ED020A3C4B67EE277A80
:10785800334427EE8C7AD3ED007A394B67EE277ADA
:10786800F0EE665AEDEE275A93ED006AB1EE467ACD
:10787800F4EEC75AF1EE10FA08D4F4EEC65AF1EE57
:1078880010FA8CBFB0EE467AB0EE657A2D4B1B78B5
:10789800012B02D0192B7BF42FABDFED2B7AB4EE42
:1078A800E7DAF1EE10FACCBF01230023FBF72FBB78
:1078B800DFED267AF4EEE7DAF1EE10FA78DCDFEDA8
:1078C800247AF4EEE7DAF1EE10FA71D4214BD3ED15
:1078D800007AB1EE677AB4EEC7DAF1EE10FA64D442
:1078E800B4EEE7DAF1EE10FA88BFB0EE67DA1A4BB9
:1078F800C8ED00BA1B689A427BF7FBA9FBF75FBA91
:10790800BC1F0020DB0FC9BFDB0F49C0DB0F49409C
:10791800DB0FC940E4CB1641E4CB16C1DB0FC93FEE
:10792800B0530020B04200204C030308FC30002074
:107938001031002020000020544000202031002079
:1079480088310020E42E00200000964200C0F84450
:1079580000C0F8C48431002068310020132B05D101
:10796800B0EE480A25F054F8AAF80000B0EE480A2C
:10797800D5F81432104898472378132BB0EE408A74
:107988007DF419A825F044F8AAF80200FDF713B809
:10799800BCF1000F7FF4F0AB0D9FB9460E9FB945BF
:1079A800B8BFB0EE646AFFF7E7BBB0EE47DA9EE710
:1079B8009FED02DA9BE700BFB456002000000000EC
:1079C8002DE9F04F2DED028B93B0064615F0FAFB2A
:1079D8009C4B1D7825B113B0BDEC028BBDE8F08F30
:1079E800DFF8B4B2DBF800305A05F4D5964F3A68A0
:1079F800002A00F02481954CD4F8103103F5F433B3
:107A080048339E42C0F01B81DFF8909294F81431FD
:107A1800D9F80010C4F81061013384F814318B07C9
:107A280001F1F88011F0140F41F0B38094F814318B
:107A3800580700F0F287282BDFF864A201F0B08322
:107A48005E209047824B1B78002B69D07F4C814A7F
:107A5800D4F82031F31A934200F26D87DFF844928C
:107A680099F80080B8F1000F31D17B4B186803F00A
:107A78007FFEC0B201280ED90228784F41F0058454
:107A88003B78002B41F09E85D4F82831F31AB3F5E2
:107A98007A6F81F06C8672480268002A40D099F8A3
:107AA8000030BBB96F4B1B689B781E3B012B6A4BA0
:107AB8004FF00201186841F2B785043021F05CFFED
:107AC8000122002389F8002084F8343126E0644834
:107AD80002682AB3D4F8303140F6B731F31A8B4232
:107AE8001ED994F82C31002B01F0CB83013BDBB27B
:107AF80084F82C31002B01F0268312F8011B94F82E
:107B08003471026094F835315348CA19013300685A
:107B180084F8342184F8353103F02EFEC4F830613E
:107B2800514BDAF800801B7843B1504F386828B1C0
:107B38004F4B1B78013B012B41F2A2804D4B1B7828
:107B480063B14D4F3B684BB1404CDAF80090D4F824
:107B58004C31A9EB0303632B00F24E86DFF8488112
:107B680098F80090B9F1020F01F0C3823B4F97F8E3
:107B78007430032B00F03C87404B1B7873B1404DA9
:107B88002B685BB1314C03F0FBFBD4F85831029001
:107B980044F61F62C31A934200F2D880394B1B780F
:107BA800002B40F08380384B1B7843B1274CD4F826
:107BB800A83203F5C333A0339E4280F07D86334B51
:107BC8001B78002B3FF407AF204E314C314D06F2A5
:107BD800C927206803F0CCFD00283FF4FCAE2068DC
:107BE80003F0C2FD2B7880465A1E33B120682A70F4
:107BF80003F0BEFD0028F2D1EDE603223946781ED7
:107C080025F0A9FE96F8C83296F8C92286F8CB82E4
:107C180083F47F4383F0FF039B1A1FFA88F89BB213
:107C2800B8EB132FD5D196F8CA22DBB29A42D0D13D
:107C3800781E21F01FFC2B7818442870C9E7DFF85C
:107C480060A0FFE63D510020185E0020FC210020C6
:107C58003E3E00203F0D0300085E00203800002053
:107C6800105E00200C5E0020403E0020B45B002027
:107C7800483E0020503E0020684D0020583E00201D
:107C88005C3E00209C3E0020B13E0020623E002069
:107C9800683E00206C3E002030570020A83E00209F
:107CA8009C590020145E0020BA3400201F4C227812
:107CB800002A40F0E2851E4F3C7854BB1D4D2A78BF
:107CC800002A41F00A841C4C1C4DD4F8A0122878D4
:107CD8001B4B93FBF0F30B449E42FFF464AF19492E
:107CE80094F8A432C4F8A062CF5CF80701F1A1852A
:107CF800B90701F15A857A0701F1EA8494F8A432A8
:107D08002978013393FBF1F201FB123384F8A43292
:107D180049E70D4D286E002841F07E828146064BCA
:107D280087F80090C3F8A0623DE700BF303E00200E
:107D3800A53E0020A43E0020FC210020B03E0020EB
:107D4800A0860100AC3E0020B83E002094F85E31C9
:107D5800002B41F00082DA4B1B6803F00802002A6E
:107D680048F603414AF60B404BF60F4249F60747DF
:107D780004BF02460F4613F0040F4FF0190118BF55
:107D880017469A0684F85E1103D547F4804747F0F2
:107D98002007CC4B5A79C7F30909002A41F09C8582
:107DA8009B79002B41F09185984664204FF0FF3372
:107DB8004FF0000C0A970B97ADF834C0CDF83AC0D5
:107DC800CDF83EC0CDF842C0CDF83090ADF8368041
:107DD800ADF838308DF846000AAF0FCFDFF8FCE277
:107DE80084F805C0AEE80F0097E80F00AEE807007A
:107DF8002EF8023B71464FF0010C1B0CFE271F208A
:107E0800C82201F81E39A770A27184F807C0E07073
:107E180094F86E01207180F0F10383EA0313DAB25B
:107E2800130983F0E70343EA022383EAC2031BB280
:107E380083EA0312D2B2C3F3072383EA121343EA95
:107E4800022383EAC2031BB283F0C80282EA021249
:107E5800D2B2C3F3072383EA121343EA022383EA65
:107E6800C2031BB283EA0C0787EA0717FFB2C3F302
:107E7800072282EA171242EA072200EB0C0382EA81
:107E8800C7070EEB0C0084F86E31278011F8013B10
:107E98007B4083EA0313DBB21A0982EA172242EA1B
:107EA800032282EAC3031BB29FB281422780EDD12D
:107EB80083F07C0383EA0313DBB24FEA131E8EEAD6
:107EC800172E8EEA032E8EEAC30E0FFA8EFE1FFAC5
:107ED8008EF3DFF80CC223804FEA13295FFA8EFE77
:107EE80004F1220384F8289084F827E00CF5CB7875
:107EF8000393DCF80C30DCF80000DCF80410DCF844
:107F0800082047460FC7039B0CF1100C9C45B84648
:107F1800EFD1DCF8000038606B4F9CF8043088F82B
:107F2800043007F1270884F8BDE184F8BE9117F8FA
:107F3800011F286803F020FCB845F8D194F85F3198
:107F4800002B41F00D816149DAF8002009780A20F8
:107F580084F85F01002901F06C825D4F012938889F
:107F6800069041F225860229B7F802E001F0B085B3
:107F7800B8880590032901F01186F888049004292F
:107F880001F006860529388901F0FD850629B7F82C
:107F98000A9001F0F4850729B7F80C8001F0EC8508
:107FA800FB89039394F86E110A920B4683F0300212
:107FB80082EA0212D2B217094649079387F07A0774
:107FC80047EA02270988237187EAC202424FC1EBB8
:107FD800012187FB01370F4412B2C917C1EB672390
:107FE800069F8DF83D3082EA0211C9B2C2F307221A
:107FF8004FF0000C82EA111267F30F0C059F0692EE
:108008006EF31F4C049ACDF82CC04FF0000E67F3A6
:108018000F0E002762F31F4E60F30F07039ACDF887
:1080280030E0002068F30F0062F31F40069A0E90BC
:1080380069F31F474FF000090D978DF83C9042EA0D
:1080480001220DF1280C82EAC107BCE80F003FB2FB
:1080580087F0C80888EA0818DFF880E084F80590F7
:108068005FFA88F8C7F30727AEE80F0087EA181702
:1080780047EA08239CE8030083EAC8031BB283F09D
:1080880023024EF8040B82EA0212D2B2C3F307238A
:10809800079F83EA1213704643EA022383EAC20267
:1080A80007F1010C20F814194FF023081621FE27B8
:1080B800C82384F86EC10EF1020E2280E17011E02F
:1080C800A83E00206C3D002093230020DC510020B6
:1080D800AC5F0020603D00200308208004220020BF
:1080E800FE21002084F80780A770A371114610F8BC
:1080F800013B4B4083EA0313DBB21A0982EA1122DF
:1081080042EA032282EAC3031BB299B27045218076
:10811800EDD183F0F40383EA0313DBB24FEA131EB5
:108128008EEA112E8EEA032E8EEAC30E0FFA8EFE09
:108138001FFA8EF8E64FA4F800804FEA182C5FFA71
:108148008EFE84F81EE084F81FC07968BA68386823
:10815800FB6807F5CB78A8E80F0038697969BA6930
:1081680004F29717A8E8070004F2B51884F8B5C117
:1081780084F8B4E117F8011F286803F0FDFAB84540
:10818800F8D194F86671002F40F0F487D14B94F839
:108198006EE1B3F90010B3F90220B3F904309FED92
:1081A800CE6A677107EE103ADAF800300A938EF05B
:1081B8006A0383EA031306EE901AD9B20B0983F017
:1081C800D50343EA012383EAC1031BB283EA0311FF
:1081D8005242C9B207EE902AC3F3072383EA111368
:1081E80043EA0123F8EEE77AF8EEE66AB8EEC77AD2
:1081F80083EAC1031BB267EE867A66EE866A27EECB
:10820800067A002083F0C808CDED0C7ACDED0B6A14
:108218008DED0D7A0E900F90109088EA081C0DF1E4
:1082280028095FFA8CFCC3F30728B9E80F0088EA2D
:108238001C1848EA0C2888EACC08DFF8B8C20FFAFC
:1082480088F8ACE80F0088F01E0799E8070087EA6D
:108258000717FFB2C8F3072383EA171343EA072374
:108268008CE8070083EAC7071C20C8214FF00509DE
:108278004FF01E08FE230EF10102E070A17184F890
:10828800669184F80780A370ACF1100184F804E0CB
:108298000CF10C00278084F86E2111F8013B7B401B
:1082A80083EA0313DBB21A0982EA172242EA03229D
:1082B80082EAC3031BB29FB281422780EDD183F0CB
:1082C800270383EA0313DBB24FEA131E8EEA172E45
:1082D8008EEA032E8EEAC30E0FFA8EFE1FFA8EF96F
:1082E800DFF8ECC1A4F800905FFA8EFE4FEA192976
:1082F80084F8259084F824E00CF5CB7804F1220A60
:10830800DCF80000DCF80410DCF80820DCF80C309D
:1083180047460FC70CF1100CD445B846F0D16F4F43
:10832800BCF80030A8F8003007F1240884F8BAE156
:1083380084F8BB9117F8011F286803F01DFAB845A7
:10834800F8D194F867310393002B40F00E87644B03
:108358001B68052213F0140F84F8672141F05E8032
:10836800DFED607A94F86E815A4B5F4AB3F90410D6
:10837800B2F906205D4F5E48CDED0C7A88F02203F5
:1083880083EA03135FFA83FE4FEA1E1383F059034F
:1083980043EA0E2383EACE03B2F5FA6F1BB2A8BFF5
:1083A8004FF4FA6283EA031E5FFA8EFEB2F57A7F13
:1083B800C3F3072383EA1E13B8BF4FF47A724FF052
:1083C800640C43EA0E23A2F57A720CFB02F283EAEC
:1083D800CE0387FB02C780FB01C00FFA83FED217CA
:1083E800C9174FF00009C2EBA712C1EBA0018EF02C
:1083F800C807ADF83A20ADF83810CDF82890CDF878
:108408002C90CDF834900DF1280C87EA0717BCE8BA
:108418000F00FFB2CEF3072E8EEA171E4EEA072E84
:108428008EEAC707DFF8CCE0DCF800C084F80480E7
:10843800AEE80F003FB287F04A0383EA0313DBB2CA
:10844800C7F3072181EA1311724641EA032108F1B3
:10845800010881EAC303142042F810C9FE274FF02F
:108468004A0C002184F86E814FF0C808E070238020
:108478000EF1040E84F807C0A770617184F80680B5
:10848800184612F8011B414081EA0111C9B20B09D3
:1084980083EA102343EA012383EAC10109B288B2BF
:1084A80072452080EDD181F0140181EA0111C9B231
:1084B8004FEA111E8EEA102E8EEA012E8EEAC10EA8
:1084C8000FFA8EFE1FFA8EF7DFF80480278013E07C
:1084D800FE210020D451002088C3E43A93230020D1
:1084E800A83E002000000000AC5F0020D34D6210C1
:1084F80067666666042200204FEA172A5FFA8EFE36
:1085080084F81DA084F81CE0D8F80410D8F80000FE
:10851800D8F80820D8F80C30B8F8189008F5CB7CB3
:10852800ACE80F00D8F81000D8F81410ACE8030035
:1085380004F29717ACF8009084F8B3A1B94684F810
:10854800B2E104F2B31A19F8011F286803F014F90C
:10855800CA45F8D1CD4BCE4A1B781278013B12F0B0
:108568000100DBB214BFC0214021172B04D8C94A2F
:10857800134493F830300393C74B1A8893071ABFF4
:10858800002341F01001012312F4027F18BF0223D7
:1085980012F0100F18BF062312F0200F18BF102377
:1085A800002841F0DA804FF0030C94F86EA10A938A
:1085B8008AF0460383EA0313DAB2130983F09203BD
:1085C80043EA022383EAC2031BB283EA0310C0B260
:1085D800C3F3072282EA101242EA002282EAC002AA
:1085E80012B282F0C80E8EEA0E1E5FFA8EFEC2F339
:1085F800072200239DF80C908DF82C9082EA1E1219
:1086080003208DF82FC08DF82D3042EA0E2C8DF8FE
:108618002E108DF830000AAA07CA8CEACE0E0FFA7F
:108628008EFEDFF88C92E3718EEA0E1CA9E8030037
:108638005FFA8CFCCEF3072E8EEA1C1E4EEA0C2144
:1086480081EACC0C94F808E089F800200FFA8CFC39
:108658008EEA0C0E8EEA0E1E5FFA8EFECCF307220F
:1086680082EA1E1242EA0E22607AA17A94F80BC0BE
:10867800637182EACE0212B2504080EA001E5FFAAD
:108688008EFEC2F3072080EA1E1040EA0E2080EA20
:10869800CE0000B2414081EA0111C9B2C0F30722FD
:1086A80082EA111242EA012282EAC10212B28CEA7B
:1086B800020C8CEA0C1C5FFA8CFCC2F3072282EADB
:1086C8001C1242EA0C2294F80CE0607BA17B84F82F
:1086D80004A082EACC0212B28EEA020E8EEA0E1EC4
:1086E8005FFA8EFEC2F3072282EA1E1242EA0E22C7
:1086F80082EACE0212B2504080EA0010C0B2C2F341
:10870800072282EA101242EA002282EAC00212B26A
:10871800514081EA0111C9B2C2F3072282EA11125B
:1087280042EA012282EAC102E17B207C039013B273
:1087380081EA030282EA0212D2B2C3F3072383EA70
:10874800121343EA022383EAC2031BB202465A40C9
:1087580082EA0212D2B2C3F3072383EA121343EA6E
:10876800022383EAC2031BB283F0320282EA0212B6
:10877800D2B2C3F3072383EA121343EA022383EA3C
:10878800C2031BB29AB24FF0FE0C0AF101014FF07E
:10879800090EC820DBB284F802C04FEA122C84F814
:1087A80003E0A07184F86E11228084F812C063740B
:1087B800D8F80820D8F80000D8F80410B8F80CA0A9
:1087C80009F5C47EAEE807009DF80C208EF802205B
:1087D800AEF800A009F5CC7884F8A8C184F8A731D0
:1087E80017F8011F286802F0C7FFB845F8D1029BA7
:1087F800C4F85831FFF7D2B9412021F06BF8274B64
:10880800DFF8B080B3F9023088FB0320DB17C3EB35
:10881800A00080B221F044F8204BB3F9003088FB67
:108828000320DB17C3EBA00080B221F039F81B4B03
:10883800B3F9043088FB0320DB17C3EBA00080B238
:1088480021F02EF8164B3868197802F095FF94F845
:10885800503113F0010800F04585124AC4F84C91D4
:108868000133DBB2A2FB0312D20802EB8202A3EBB4
:10887800420384F85031FFF771B90B4B0B49186864
:1088880002F04AFF00232370FFF715BACC420020FC
:10889800FC4800203CDF0208623D0020D451002043
:1088A80036510020CDCCCCCCA03E0020F03D00209D
:1088B800042200206766666694F8AC32C14AC4F8A0
:1088C800A86202EB8302926C42B312AD04F2B323A6
:1088D800BD4E45F8203D002104F2C52331800B939D
:1088E80080211523A52784F8B232284684F8B112CE
:1088F80084F8B072904728463188F8F7E3FC0A9D5F
:10890800B24804F52C716D1A152DA8BF15252A46F5
:1089180023F052FFAE4A94F8AC321570AD4A0133D9
:1089280082FB0312A2EBE37202EB42029B1A84F869
:10893800AC32FFF744B9A84AA84B92F80BE0DAF832
:108948000000D4F824211B88A549801A4FF47A72B4
:10895800DFB202FB0EF21B0A8F770F7590424FF0C1
:108968000007CB774B758F700F7180F07A849D4B21
:108978009D4F1B689D4ADFF890E210689268C4F822
:10898800206187FB038CDB17C3EB6C13D4F818C189
:1089980087FB0C878EFB00988EFB029ED217C2EBDA
:1089A800AE0203F5FA734FEAEC7E9BB2CEEB671E7C
:1089B800C0170CF5EA47C0EBA80030378B761B0AC6
:1089C8000EF1780E3F120CF1300CCB764FEA2028CE
:1089D8001312087781F81D8081F8202081F8213052
:1089E80081F824E081F8237081F822C0FFF736B8B7
:1089F8007F4B0293186802F0B3FE00283FF4BCA82E
:108A0800029B0121186802F0A7FE0222002387F8C2
:108A1800742088F80030FFF7AFB85E2090473B68B5
:108A280002209847734B704A9B6A323382FB0328B3
:108A3800DB17C3EB68185FFA88F020F0EFFFC8F384
:108A4800072020F0EBFF3B685E2098473B68032037
:108A58009847694B1B78D90740F1918322F04AF86F
:108A6800664B9FED677AD3ED037A67EE877AFCEE63
:108A7800E77ACDED027ABDF80830002800F0A88525
:108A8800D8B24FEA132820F0C9FF404620F0C6FFAD
:108A98005C4B1B78042B77D0DFF870A1B4F81C115D
:108AA8009AF80020DFF8349191FBF2F302FB1313DC
:108AB8009BB2B9F80010A4F81C314FEA03181FFA4A
:108AC80088F8642303FB01235200B3FBF2F348EA5E
:108AD8000328C3F303225E203B681FFA88F848EA9C
:108AE800020898473B68062098475FFA88F020F00C
:108AF80095FF4FEA182020F091FF374AB4F81C314F
:108B0800517AB9F8009001330129A4F81C3101F019
:108B18000980537B09EB89091FFA89F9002B40F07A
:108B280016863B685E2098473B683A2098472E4B4C
:108B3800A3FB09384FEA58181FFA88FA5FFA8AF037
:108B480020F06CFF4FEA1A2020F068FF3B685E2097
:108B580098473B683B209847642303FB18939BB2D4
:108B68002948053380FB0320DB17C3EBA000C0B204
:108B780020F054FF002020F051FFDFF8948098F88F
:108B88000630002B40F0728594F814313A68FEF7ED
:108B980052BF5E2090473B6830209847D4F8188130
:108BA8005FFA88F020F03AFFC8F3072020F036FF7C
:108BB80094F8143113F0030800F04E843A68FEF775
:108BC80037BF00BF3CDF0208AE3D002088440020CC
:108BD8009D440020565555553C5C0020C85B00203C
:108BE800703E0020782100201F85EB51BC5B0020DF
:108BF8001835002078400020FC4800204C5C0020FC
:108C0800CDCC4C3E663D0020676666664A5C002017
:108C18006C3D0020DFF838839FEDC48A03944FF041
:108C2800240A5E20904750463B689847C04BF8ECB2
:108C3800016A9B8A07EE103AF8EEE66AB8EEC77A40
:108C48000AF1010AC6EE877A5FFA8AFA67EE887A2D
:108C5800FDEEE77ACDED027ABDF90840E0B220F0EA
:108C6800DDFEC4F3072020F0D9FEBAF1270F01D0AA
:108C78003A68D6E7039CD9F800103A68FEF7D2BEE6
:108C8800AC4CDFF8D0920AE01B2B00F046820D2B8B
:108C980000F00D824FF0010389F80130386802F0C6
:108CA80067FD00283BD0386802F05EFD83B27E2B5A
:108CB800DAF800202AD099F801100029EED194F8AA
:108CC8003621002AE0D07D2B00F0068294F844E19A
:108CD800BEF1000F04D080F02003DBB284F8441109
:108CE800511CC9B22244092984F8361182F8383156
:108CF80000F0E6810829D1D8B4F84221134403EBE7
:108D0800132303F0FF03A4F84231C7E74FF0000331
:108D180084F8363184F8373189F80130BEE794F8A1
:108D2800453133B194F8393184F84501302B00F0DE
:108D3800958494F83721804BDFF81CC2DFF81CE2D9
:108D48000127104600283EF4F9AEDAF80020A2EB1D
:108D58000802012A00F2A68194F84691B9F1000FA1
:108D680040F0E68194F8471133F8112012B984F8DD
:108D78004771E7E70131B2F5826F84F8471100F0D7
:108D8800BC801FD9B2F5E26F00F09B8035D9B2F5EF
:108D9800046F00F0A580B2F5116F00F01B81B2F5E9
:108DA800E46FCFD11046624A176C918A642303FBA3
:108DB80007F393FBF1F120F0C5FD002384F8373168
:108DC800FEF7BCBEB2F5007F00F01E812DD8B2F5CB
:108DD800807F00F03D81B2F5887FB3D1DCF80020B8
:108DE8005207AFD5D4F818114FF4887020F0AAFDB7
:108DF800002384F83731FEF7A1BEB2F5C06F00F04A
:108E08001781B2F5E06F9DD1494A906B918A64232E
:108E180003FB00F34FF4E06093FBF1F120F092FDC7
:108E2800002384F83731FEF789BEB2F5047F00F0DD
:108E38001F81B2F5806F85D194F848310133DBB2D8
:108E4800032B00F2508142F2107184F8483101FB83
:108E580003F13A4B1B68002B40F043810131384B3A
:108E68001B78DF07374B1B8848BF0431D80748BF3A
:108E78000A319A0748BF14311F0648BF2831D80560
:108E880048BF28315A0748BF64311F0748BFC83157
:108E9800980548BF01F5C8719A0648BF01F57A716F
:108EA800DF0648BF01F5FA61580648BF01F57A6147
:108EB8004FF4806020F046FD002384F83731FEF738
:108EC8003DBE10461A4AD76B918A642303FB07F309
:108ED80093FBF1F120F036FD84F83791FEF72EBEB2
:108EE800194BB3F9041001EB81011046490020F039
:108EF80029FD84F83791FEF721BEDCF8002012F036
:108F080020097FF41FAFDBF80010090600F19083F9
:108F18000E4A127B002A3FF415AF94F84911032931
:108F280000F21086DFE801F04C42331C00007A445E
:108F38008C510020FC2100203CDF0208A03D0020CD
:108F4800FC480020623D0020D45100203C5C0020F9
:108F5800C451002038000020A83E00206C3D0020AD
:108F6800CD4B1B6859799A79DB7901F1407101EB96
:108F7800022101EB0341002384F849314FF4826058
:108F880020F0E0FC002384F83731FEF7D7BDC34B4F
:108F98001A68137A507992781B0403EB0023134460
:108FA8004A1C84F8492103EB0161E7E7BB4B1A68C7
:108FB800D379107952781B0403EB00231344EFE7AD
:108FC800B64B1A689379D07812781B0403EB002308
:108FD8001344E5E79EF80520002A3FF4B3AEB04AF3
:108FE800117800293FF4AEAEAE4B1B8803EB830328
:108FF8005B004FF4116093FBF1F120F0A3FC002318
:1090080084F83731FEF79ABD9EF8061000293FF420
:1090180099AEA54BA5491B68104681FB0321DB17B8
:10902800C3EBA10120F08EFC84F83791FEF786BDD2
:109038009EF80620002A3FF485AE9B4B4FF4C06093
:10904800996820F07FFC002384F83731FEF776BD5D
:10905800DCF8002051077FF575AE954B4FF4807012
:10906800196820F06FFC002384F83731FEF766BDDD
:109078009EF80520002A3FF465AE894A1178002938
:109088003FF460AE8B4B5B7B002B00F05D83854B20
:109098001B8893FBF1F101EB810149004FF4047047
:1090A80020F050FC002384F83731FEF747BD4FF01D
:1090B800010184F8361184F83831A4F84221EDE52D
:1090C800B4F84221C2F1FF0293427FF4E3AD4FF0BE
:1090D800010384F84531DDE54FF0010384F844319C
:1090E800DCE50231BBE6012384F8483142F2107115
:1090F800AFE602F045F9704B1A6840F6B833821AA9
:109108009A4200F280816D4B1B793A2B00F01C8447
:10911800002388F80030FEF72FBD386802F028FBDE
:1091280000287FF4B7AD4FF0010384F83731B5E577
:109138006349062020F024FA002384F8460184F8C5
:109148003731FEF7FBBC94F8341194F835315D489B
:109158004A1CFEF7DBBC013B84F85E31FEF7EEBE2D
:10916800013B84F85F31FFF70CB8013B84F86731A5
:10917800FFF73DBB013F84F86671FFF7E2B8524A3A
:10918800524BB2F80880A3FB08384FEA98085FFAF8
:1091980088F020F043FC4FEA182020F03FFC77E4E9
:1091A800DAF8003002934FF000085E2084F814814A
:1091B80090473B68DFF8249117209847404620F0F5
:1091C8002DFC029C424B2246A3FB02239B0BA9FBCE
:1091D80003125209C2EB0212A3EB8203D8B220F0A9
:1091E8001DFC3B685E2098473B6818209847394B20
:1091F8002246A3FB02239B09A9FB03125209C2EBD7
:109208000212A3EB8203D8B220F008FC404620F0FB
:1092180005FC3A68FEF714BC0024DFF8C480A146B8
:109228004FF0500A02E0DBB283F3118815F804B05E
:10923800601C5946284420F047FA002840F0038172
:109248000BF101031C44EFF311838AF312882A6E91
:109258009442E8DB0022DBB22A6683F31188FEF72A
:109268005EBD1D4BDAF800201B78C4F82421013BB1
:10927800012B3FF67CAB102202238A700B71FFF79B
:1092880076BB20F0ADFBFEF749BC20F099FB01232B
:109298003B70FEF700BC00BFD45F00206451002083
:1092A8004A5C0020C85B0020BC5B002067666666DD
:1092B800782100203C5C0020C0340020A834002025
:1092C80045990208085E00206C3D0020CDCCCCCC2E
:1092D80073B2E745D34D6210663D002089888888BF
:1092E8004DD10108BE4B1B88DA0515D4D80600F10C
:1092F800F783990600F112845A0600F131841807A1
:1093080000F13284D90700F1338413F0020F0CBF47
:109318004FF004084FF00C08B24BB34A1B78D278D0
:1093280003F001030AB143F002035320039320F032
:10933800D1FAAE4A128802EB820202EB8202900056
:1093480080B220F0ADFA002020F0AAFAA84AA94974
:1093580012883868C2EBC212520081FB02311144F4
:10936800D217C2EB6122D3B21946029302F004FA73
:10937800039BA14A3868127848EA0308029B5340C5
:109388009D4A0021137002F0F7F94146386802F04F
:10939800F3F9994B984A1B78386888EA0303DBB2DB
:1093A8001946137002F0E8F994F85031002B7FF455
:1093B80054AA4F2020F08EFA19F0F0FB19F0EEFBBA
:1093C80019F0ECFB0121386802F0D6F98B4A8A4B78
:1093D80092F800801B78884A386808F0010883F002
:1093E80001034146137002F0C7F9834B824A1B7888
:1093F800386888EA03031946137002F0BDF994F837
:109408005031FFF72ABA7E4AB2F8523100210133AF
:10941800A2F8523188F80010FEF7AEBB794B9FEDE9
:109428007A7AD3ED007AF8EEE77A67EE877AFEF774
:1094380099BF884689460846049105918E4606914B
:109448000391FEF7AFBD41463A2020F099F840EA73
:1094580009095FFA89F9F3E66C49D4F81021694BD8
:109468008A421B6840F26C81002BB8BF5B42684A95
:109478001BB282FB03124FEAE37ACAEB621A4FF07F
:10948800640808FB1A380FFA88F80FFA8AFA5FFAA4
:1094980088F95FFA8AF2C8F30728CAF3072A3B68F3
:1094A80002925E2098473B6810209847029A10461F
:1094B80020F0B4FA504620F0B1FA3B685E20984795
:1094C8003B6821209847484620F0A8FA404620F0FB
:1094D800A5FA94F81431FFF771BB4E494E4B00932F
:1094E800A1F13F074D4B4E4A099101F8404C0AA89B
:1094F8004C490897F7F7BEFF089F7B1C08933C7000
:10950800089B2922591C08911A70089BEA22591CA9
:1095180008911A70089BC822591C08910AA81A7049
:1095280022F092F900F101080AA94246089823F0AE
:1095380043F9089A02EB08030133089302F808403C
:10954800089B5A1C08921C70089B5A1C08921C7095
:10955800089B5A1C08921C70089B5A1C08921C7085
:10956800089B5A1C08921C70089B5A1C08921C7075
:10957800089B5A1C08921C70089B5A1C08921C7065
:10958800089B5A1C08921C70089B5A1C08921C7055
:10959800089B5A1C08921C70089B5A1C08921C7045
:1095A800089B0122991812A808911A7050F8283DB2
:1095B800DB1B3B7013F0ACFD114B2C70C3F8A062A1
:1095C800FEF7F1BAC4F8286187F80080FEF763BA9D
:1095D800DBF80020D2067FF553AA8046FFF753BA7E
:1095E800623D0020FC4800207C3D0020C85B002034
:1095F800603D002003082080365100207848002074
:10960800FC210020782100200AD7233C3F4B4C0046
:109618001F85EB51F03D00205D51002050040308E8
:10962800580403086404030802F096F8FEF748BAE1
:109638001023042218460AA98DF82A908DF82B9039
:109648008DF82C908DF82D908DF828308DF82920E4
:1096580020F058F984F83791FEF770BA0621AA4825
:1096680020F032F884F84601FFF763BB3B68DFF867
:10967800CC92DFF8C0A25E2098473B682820984724
:10968800D9F800308AFB032ADB17C3EBAA0A5FFA72
:109698008AF020F0C3F9CAF3072020F0BFF93B682D
:1096A8005E2098473B6804209847B8F80830002B9C
:1096B80040F01982D9F8083083F310085FFA88F06F
:1096C80020F0ACF9C8F3072020F0A8F9FFF75CBA3E
:1096D8008E4B8F4A0B93A3F140081268002103F8C0
:1096E800401C212388F80230D30040F10B828949BD
:1096F8000327894B1B88580500F10182DA0700F11E
:109708002C8203F00203854A002B1CBF0327114655
:10971800DFF82C923A46484623F04EF807EB090347
:1097280012A80133A9F1020140F8203D00225B1A7A
:1097380007F8092088F8013013F0EAFCFEF7DEBAD2
:10974800C146C2464246AAE6754B1988A3E49AF870
:10975800003099FBF3F9FFF7E4B9724AD278002A8E
:109768000CBF4FF0040C4FF0050CFEF71EBF6E4AFD
:10977800012310683B7001F0F7FF6B4B0746186830
:1097880001F0F2FF7F067EF486A98E287EF483A975
:1097980099F80030002B7EF49AA9644B644A1A6049
:1097A8002D2384F82C31FEF77DB9584A5C4B0B9277
:1097B8000DF14808A2F13D0048F8200D1988DFF89E
:1097C8007C91A2F1400300204FF00A0E02F8400CF1
:1097D800082283F801E040469A70F7F74DFDD9F862
:1097E80000305449DA1781FB0313C2EBA30399B283
:1097F8004046F7F741FD09F0FDFAD9F808900A9BB1
:109808004FEA1942591C0A911A700A9B4FEA192209
:10981800591C0A911A700A9B5A1C0A9283F80090E4
:109828000A9B5A1C0A921870404613F071FCFEF706
:1098380062BADFF810919FED408AB9F902303348D7
:109848000B9007EE903AF8EEE77A0DF1480867EECC
:10985800887AA0F13D01FDEEE77A48F8201D00F86E
:10986800402C0822CDED027A00F83F2C1E2200F889
:109878003E2CBDF808104046F7F7FEFCB9F9003059
:1098880007EE903AF8EEE77A404667EE887AFDEE02
:10989800E77ACDED027ABDF80810F7F7EDFCB9F9D3
:1098A800043007EE903AF8EEE77A404667EE887A99
:1098B800FDEEE77ACDED027ABDF80810F7F7DCFC8B
:1098C800404613F025FCFEF713BA1C4B9046B3F93B
:1098D80000306420FEF76CBA11499A790B8803EBC3
:1098E800830303EB83034FEA83081FFA88F8002AEF
:1098F80040F05B814FF0FF331BB2039309F07AFA13
:10990800039B40B2FEF754BA36230020F03D0020F6
:10991800544200203C040308623D00204C04030824
:10992800C85B00207C3D0020085E0020105E0020FF
:10993800703E00206766666658A08B41BC5B0020BD
:10994800B33D0020D45100209E4B029299781846CE
:1099580010F098F8029A00287FF4DAAB9A4F9B4BE4
:10996800DFF890E2FA669A481A689A4C9B689A4916
:10997800FB64994B00880291FA62DEF80010B4F893
:109988005221F861F9631868FA6500F05BFA0390F0
:1099980000287EF4ECA8904B4946186801F0DCFEDC
:1099A800884A94F85431D2780492642B4FF0040218
:1099B80087F8742040F0228194F85531072B04BFB2
:1099C8009DF80C3084F8553194F855311A4607EB58
:1099D8000219824BD9F8041003930846059207919F
:1099E80021F032FFD9F8081006915FFA80F908468D
:1099F80021F02AFFC3B209EB03027848079908321D
:109A0800C2710598059300F00F0E20F00F027348FD
:109A1800827203EBC900714B4A4683F80DE09873D4
:109A280003F10F0022F0C8FE059B06991A466C4BFD
:109A380009F10900184422F0BFFE6848C37903F110
:109A48000109CBB1013B5FFA83FC0CF1080CDFF88C
:109A5800A8E184440023073010F8011B59408B000B
:109A6800CA0883EA410302F018024B404EFA02F298
:109A780053408445DBB2EFD1594A049809F80230C3
:109A880022F0C2FD94F855310022013384F8553193
:109A980084F85421039BDDF80C909B785BB1029B02
:109AA80019F80510186801F067FE013599F80230B9
:109AB800EDB2AB42F3D894F854310322013384F861
:109AC800543187F8742088F80020029BFEF792BF73
:109AD800984699461846049305930393FEF762BA8D
:109AE8004FF0340818E409F085F91FF097FF0020BB
:109AF8001FF094FF94F814313A68FDF79CBF0327D0
:109B0800384905E6DBF80030374A384903F4800362
:109B1800002B16BF114604270327EAE54FF0240857
:109B2800FFF7FABB3B685E2098473B6839209847A7
:109B38005FFA89F01FF072FF4FEA19201FF06EFFDD
:109B4800FFF71BB84B1CDBB2042B84F849314FEAF2
:109B580001617FF413AAFFF70EBA25490427D7E558
:109B68004FF01008FFF7D8BB4FF02008FFF7D4BB21
:109B78004FF00808FFF7D0BB0393FEF713BA9846D7
:109B88000393FEF70FBA984699460393FEF70ABA6D
:109B98009846994618460393FEF704BA984699469C
:109BA800184604930393FEF7FDB9084B1B68A3E618
:109BB800984699461846049305939E460393FEF7E4
:109BC800F1B900BFA834002038000020BC5B002099
:109BD800C85B0020FC21002018350020404D0020E3
:109BE800464D0020400403083C04030834040308DD
:109BF80044040308782100200007090E97F875909F
:109C08004549059519F00F0F04BF09F101095FFADD
:109C180089F9B9F1070F28BF4FF001094FEA091C6C
:109C280007EB0C03187C3D4B03930A18002392F8AA
:109C380024103A4A93725FFA8CF31A46384B9646C8
:109C480007EB0C024EEA000001291870D26803F1F4
:109C580001000CD90239C9B28D1C1D44034603F812
:109C6800012BAB424FEA1222F9D101310844BC441E
:109C780022F0600309F101099CF811205FFA89F9C3
:109C88001343B9F1080F037000F1010340D04FEA04
:109C9800091C07EB0C01224A087C1F4901449A1A47
:109CA80091F8241055180EF1100E132D5FFA8EFE40
:109CB800C6DD059D0398DFF870E0D2B2931DDBB2D4
:109CC80043F04001C17103F1010CCBB10532D3B2AD
:109CD8000833C31805930EF10100002310F8011B87
:109CE80059408B0083EA4103CA084B400D4902F0F2
:109CF800180241FA02F25340059A8242DBB2EDD1D2
:109D080004980CF80E3087F8759022F07DFCC1E6B7
:109D1800034A059D9A1ACDE73CDF0208404D002012
:109D28004D4D00200007090E464D0020436A826908
:109D3800D154436A0169426B01338B4228BF002327
:109D48004362002A2FD0EFF31181502383F3128846
:109D5800436B1A68D2072CD470B45E686EB9456A32
:109D6800826A954217D084691444DC600ED9AA1A15
:109D78005A608562002280F850201A6842F0010279
:109D8800C9B21A6081F3118870BC70470469A21ABD
:109D98005A608662EEE7012380F85030C9B281F339
:109DA800118870BC7047C26C136843F0800313605D
:109DB8007047C9B281F31188704700BF026B10B4B5
:109DC80062B1036CC2684469D11A013B615C5DF8F9
:109DD800044B08BF13460364C8B27047016A43695D
:109DE800C4685B5C0131A14228BF114601625DF87D
:109DF800044BD8B2704700BF436B13B190F85000C2
:109E08007047836A406A181AB0FA80F040097047B0
:109E1800416A836A99420AD3CB1A416B026961B1DC
:109E28004968501E0B4483420AD2C01A704702691F
:109E38001144CB1A416B0029F2D1501EC01A704749
:109E480000207047036B43B1026C5B6893422FBFDD
:109E5800981AC0689B1AC0187047C269036A9A4268
:109E68002FBFD01AC0688018C01A70472B230373FD
:109E78002A23837000238375704700BF03682DE988
:109E8800F041DF691FB13B46BDE8F0411847002AA1
:109E9800164611DD04460D460E4400E023689B6813
:109EA800204698470028F9D0236815F8011B1B683D
:109EB80020469847AE42F1D1BDE8F08100233F2209
:109EC800027043708370C3707047152303701623A4
:109ED800C370172383712D2343702E2303712F23FF
:109EE800C37170472DE9F0470569C3681D4028D044
:109EF8000F4606464FF000484FF00009B5FA85F3C3
:109F080028FA03F2D2431B3B32611540042B16D8C2
:109F1800DFE803F03129211903007B6A002B32D0D6
:109F280003F1FF3A1FFA8AFAC7F824903C6A34B161
:109F380023682046514698476468002CF8D1002DC4
:109F4800DCD1BDE8F0873868716B036889B298473F
:109F5800002DD3D1F5E77868B16B036889B29847CB
:109F6800002DCBD1EDE7B868F16B036889B298474B
:109F7800002DC3D1E5E7F868316C036889B29847CA
:109F8800002DBBD1DDE7F36A1FFA83FACEE700BFE5
:109F980030B50446C06C61710368A26823F0010300
:109FA800036087B0A379009213F004023DD04FF408
:109FB800805213F00203019244D102934FF480635C
:109FC8000022039311F00103059237D1049308236B
:109FD8008D07694648BF04931AF078FE6079E36CF0
:109FE800A17900F00202002A15BF4FF440324FF465
:109FF80080324FF40034002410F0010F586808BF75
:10A008002246CC074CBF024320EA02025A609A68F3
:10A0180009074CBF42F0080222F008029A601A6849
:10A0280042F001021A6007B030BD13F0020301923A
:10A038000BD04FF4005513460295C1E7042304934F
:10A048000C23C5E74FF40053B7E70293B8E700BF06
:10A0580010B50446C06CA160036823F001030360D7
:10A06800A37986B013F00402009141D04FF48052D6
:10A0780013F00203019244D102934FF48063627992
:10A088000393D1074FF000030493059345BF0423BE
:10A09800049308230C236946920748BF04931AF0D7
:10A0A80015FE6079E36CA17900F00202002A15BF61
:10A0B8004FF440324FF480324FF40034002410F053
:10A0C800010F586808BF2246CC074CBF024320EA5C
:10A0D80002025A609A6809074CBF42F0080222F04F
:10A0E80008029A601A6842F001021A6006B010BDB0
:10A0F80013F00203019207D04FF400511346029166
:10A10800BDE74FF40053B7E70293B8E7F0B50C2961
:10A118002BD8DFE801F06F2A2A2A4C2A2A2A2B2A70
:10A128002A2A0700046AB2F80CE097881668674D77
:10A1380024F480540462036A4468C16923F4005318
:10A1480043EA0E3321F4E641A84243EA073341EAE1
:10A15800062100F0B58005F50065A84200F0B08042
:10A1680092684460C16102640362F0BD046A968922
:10A178009588D2F800E0554F24F480740462036A8D
:10A188004468C16923F4007343EA062321F073018C
:10A19800B84243EA052341EA0E017ED04C4DA8425D
:10A1A8007BD092684460C161C2630362F0BD046AF7
:10A1B80096899588D2F800E0444F24F01004046290
:10A1C800036A4468816923F0200321F0807143EA1F
:10A1D800061321F4E641B84243EA051341EA0E2189
:10A1E80048D03B4DA84245D0926844608161826363
:10A1F8000362F0BD046A9389B2F804E01768334E2D
:10A2080024F001040462056A4468816943EA0E0384
:10A2180021F4803125F002059BB221F07301B04290
:10A2280043EA050341EA070114D0294DA84211D099
:10A2380005F54065A8420DD005F58065A84209D00E
:10A2480005F58065A84205D0926844608161426343
:10A258000362F0BDD689158A578A23F00803334371
:10A268003D43D68824F4407423F00403ADB233434D
:10A278002C43E9E7D589178AD68823F0800343EA77
:10A28800051324F44064558A23F0400344EA870404
:10A2980043EA061344EA8504A6E7D589178AD688CF
:10A2A80023F4006343EA052324F44054558A23F435
:10A2B800806344EA071443EA062344EA051470E776
:10A2C800158A24F4804444EA851449E7002C0140A7
:10A2D800003401402DE9F04FC822002183B07948AD
:10A2E800794CDFF80892794D794E7A4FDFF8008281
:10A2F80023F04BFB78487949DFF8F8E1DFF8F8C13B
:10A3080000221359834200F0C280B3F1804F00F05D
:10A31800CA80AB4200F0C980B34200F0C880BB429B
:10A3280000F0C780734500F0C680634500F0C58023
:10A33800434500F0C480DFF8C4A153457AD00AF53C
:10A34800806A534508BF092375D01432782AD8D1BA
:10A358005D4C634D634E614F04F1780802E014349C
:10A36800A04564D0A379002BF9D023794FEA1319BB
:10A3780009F1FF39B9F1050F03F00F03EFD835F8EC
:10A38800190040FA03F2D207E9D54FF0010A0AFA98
:10A3980003F3013B184021F051FF16F809305249E8
:10A3A800184411EBC002DAD051F83000DFF850E160
:10A3B800217A00F138439B0A1EF8033003F01F0E80
:10A3C8005B09022B0AFA0EFA63D0032B66D0012B25
:10A3D80058D093880093B3FA83F3C3F11F039BB259
:10A3E800DA0800EB820203F00703D2F820E09B00B2
:10A3F8004FF00F0C0CFA03FC2EEA0C0EC2F820E00A
:10A40800D2F820E001FA03F343EA0E031362694627
:10A418000023022214348DF804208DF805308DF8BD
:10A4280006308DF8073016F0EFFDA0459AD103B03D
:10A43800BDE8F08F082309EBC3034FF0010B93F835
:10A4480004A00AF01F034FEA5A1ABAF1020F0BFAD6
:10A4580003F311D0BAF1030F08D0DA457FF475AFD2
:10A46800D1F814A043EA0A034B616EE7D1F81CA0A7
:10A4780043EA0A03CB6168E7D1F818A043EA0A0364
:10A488008B6162E77B694AEA03037B61A1E70023EA
:10A49800D1E7BB694AEA0303BB619AE7FB694AEA69
:10A4A8000303FB6195E70123C5E70223C3E7032301
:10A4B800C1E70423BFE70523BDE70623BBE707235E
:10A4C800B9E700BF603B00203001030800040040EA
:10A4D8000008004000100040002C0140001002401D
:10A4E800C8010308C0010308245A0020D400030847
:10A4F8000040014000140040003401400044014085
:10A5080028010308002867D003682DE9F04F03F1FC
:10A5180038445C4EA40A0125345D04F01F06640922
:10A52800022C05FA06F558D0032C00F0A580012C62
:10A5380058D08088B0FA80F4C4F11F04A4B2E508AA
:10A5480003EB850504F007042E6AA4000F27A74033
:10A5580026EA07062E622E6A01F00307A2407C1E37
:10A568003243012CC1F3810CC1F300182A62C1F3F4
:10A5780041113CD9C60700F18980850700F1958013
:10A58800440700F1A380020700F1B180C60600F17C
:10A59800BF80850600F1CD80440600F1DB8002060D
:10A5A80000F1E980C60500F1F780850500F1058115
:10A5B800440500F11381020500F12181C60400F170
:10A5C8002F81850400F13D81440400F14B81020490
:10A5D80000F15981BDE8F08F70472B4CA6693543CF
:10A5E800A561A6E7284C666935436561A1E70024A3
:10A5F80022464FF0010E4FF0030904E00132102A01
:10A6080004F10204E6D00EFA02F636EA0005F5D1A6
:10A61800D3F808A009FA04F5ED430AEA050AC3F8D5
:10A6280008A0D3F808B00CFA04FA4AEA0B0AC3F8EF
:10A6380008A0B3F804A01FFA8AFA2AEA06069E8040
:10A64800B3F804A008FA02F646EA0A06B6B29E80F3
:10A658001E682E401E60D3F800A007FA04F646EAEA
:10A668000A061E60D3F80CA001FA04F605EA0A0AE5
:10A6780046EA0A05DD60C1E7034CE6693543E56152
:10A6880057E700BF28010308001002401A6822F0AB
:10A6980003021A601A683A431A60DA6822F0030261
:10A6A8000A438507DA607FF56BAF1A6822F00C025F
:10A6B8001A601A6842EA87021A60DA6822F00C0205
:10A6C80042EA81024407DA607FF55DAF1A6822F03A
:10A6D80030021A601A6842EA07121A60DA6822F031
:10A6E800300242EA0112DA6002077FF54FAF1A68BA
:10A6F80022F0C0021A601A6842EA87121A60DA6801
:10A7080022F0C00242EA8112C606DA607FF541AF44
:10A718001A6822F440721A601A6842EA07221A601C
:10A72800DA6822F4407242EA01228506DA607FF58F
:10A7380033AF1A6822F440621A601A6842EA872224
:10A748001A60DA6822F4406242EA81224406DA603A
:10A758007FF525AF1A6822F440521A601A6842EA57
:10A7680007321A60DA6822F4405242EA0132DA60AB
:10A7780002067FF517AF1A6822F440421A601A6879
:10A7880042EA87321A60DA6822F4404242EA8132A9
:10A79800C605DA607FF509AF1A6822F440321A60FC
:10A7A8001A6842EA07421A60DA6822F4403242EA3A
:10A7B80001428505DA607FF5FBAE1A6822F4402273
:10A7C8001A601A6842EA87421A60DA6822F440225C
:10A7D80042EA81424405DA607FF5EDAE1A6822F458
:10A7E80040121A601A6842EA07521A60DA6822F4BC
:10A7F800401242EA0152DA6002057FF5DFAE1A68BC
:10A8080022F440021A601A6842EA87521A60DA682B
:10A8180022F4400242EA8152C604DA607FF5D1AEE2
:10A828001A6822F040721A601A6842EA07621A60CF
:10A83800DA6822F0407242EA01628504DA607FF544
:10A84800C3AE1A6822F040621A601A6842EA876248
:10A858001A60DA6822F0406242EA81624404DA60EF
:10A868007FF5B5AE1A6822F040521A601A6842EABB
:10A8780007721A60DA6822F0405242EA0172DA601E
:10A8880002047FF5A7AE1A6822F040421A601A68DF
:10A8980042EA87771F60DA6822F0404242EA817113
:10A8A800D960BDE8F08F00BF03682DE9F04F03F1D0
:10A8B8003845644EAD0A0124755D05F01F066D0923
:10A8C800022D04FA06F400F0A280032D00F0A48003
:10A8D800012D52D08088B0FA80F4C4F11F04A4B2CC
:10A8E800E50803EB850504F007042E6AA4000F278A
:10A8F800A74026EA07062E622E6A01F0030702FA2D
:10A9080004F47A1E3443012AC1F3810CC1F3001800
:10A918002C62C1F3411135D9C60700F1978085072C
:10A9280000F1A380440700F1B180020700F1BF8065
:10A93800C60600F1CD80850600F1DB80440600F1F3
:10A94800E980020600F1F780C60500F1058185055A
:10A9580000F11381440500F12181020500F12F81E6
:10A96800C60400F13D81850400F14B81440400F1E7
:10A978005981020455D4BDE8F08F334D6E693443D4
:10A988006C61A7E7002422464FF0010E4FF003093F
:10A9980004E00132102A04F10204ECD00EFA02F6A7
:10A9A80036EA0005F5D1D3F808A009FA04F5ED4315
:10A9B8000AEA050AC3F808A0D3F808B00CFA04FAA2
:10A9C8004AEA0B0AC3F808A0B3F804A01FFA8AFAE7
:10A9D8002AEA06069E80B3F804A008FA02F646EAB8
:10A9E8000A06B6B29E801E682E401E60D3F800A0EC
:10A9F80007FA04F646EA0A061E60D3F80CA001FA24
:10AA080004F605EA0A0A46EA0A05DD60C1E70E4DC2
:10AA1800AE693443AC615DE70B4DEE693443EC61DC
:10AA280058E71A6822F040421A601A6842EA8777A3
:10AA38001F60DA6822F0404242EA8171D960BDE8BD
:10AA4800F08F00BF28010308001002401A6822F0A6
:10AA580003021A601A683A431A60DA6822F003029D
:10AA68000A438507DA607FF55DAF1A6822F00C02A9
:10AA78001A601A6842EA87021A60DA6822F00C0241
:10AA880042EA81024407DA607FF54FAF1A6822F084
:10AA980030021A601A6842EA07121A60DA6822F06D
:10AAA800300242EA0112DA6002077FF541AF1A6804
:10AAB80022F0C0021A601A6842EA87121A60DA683D
:10AAC80022F0C00242EA8112C606DA607FF533AF8F
:10AAD8001A6822F440721A601A6842EA07221A6059
:10AAE800DA6822F4407242EA01228506DA607FF5CC
:10AAF80025AF1A6822F440621A601A6842EA87226F
:10AB08001A60DA6822F4406242EA81224406DA6076
:10AB18007FF517AF1A6822F440521A601A6842EAA1
:10AB280007321A60DA6822F4405242EA0132DA60E7
:10AB380002067FF509AF1A6822F440421A601A68C3
:10AB480042EA87321A60DA6822F4404242EA8132E5
:10AB5800C605DA607FF5FBAE1A6822F440321A6047
:10AB68001A6842EA07421A60DA6822F4403242EA76
:10AB780001428505DA607FF5EDAE1A6822F44022BD
:10AB88001A601A6842EA87421A60DA6822F4402298
:10AB980042EA81424405DA607FF5DFAE1A6822F4A2
:10ABA80040121A601A6842EA07521A60DA6822F4F8
:10ABB800401242EA0152DA6002057FF5D1AE1A6806
:10ABC80022F440021A601A6842EA87521A60DA6868
:10ABD80022F4400242EA8152C604DA607FF5C3AE2D
:10ABE8001A6822F040721A601A6842EA07621A600C
:10ABF800DA6822F0407242EA01628504DA607FF581
:10AC0800B5AE1A6822F040621A601A6842EA876292
:10AC18001A60DA6822F0406242EA81624404DA602B
:10AC28007FF5A7AE1A6822F040521A601A6842EA05
:10AC380007721A60DA6822F0405242EA0172DA605A
:10AC480097E600BF10B50409013C052C17D80D4B39
:10AC580033F8142000F00F0042FA00F313F0010358
:10AC68000DD0012303FA00F00138104021F0E6FA74
:10AC7800054A064B125D104403EBC00010BD0020CE
:10AC880010BD00BFC8010308C0010308245A0020F2
:10AC980001490248FFF726B9003C00200040014066
:10ACA80001490248FFF71EB9D83B00200034014093
:10ACB80001490248FFF716B9D83B0020003401408B
:10ACC80001490248FFF70EB9B03B002000040040DC
:10ACD80002494FF08040FFF705B900BF883B0020CC
:10ACE80001490248FFF7FEB8603B0020002C0140F4
:10ACF80001490248FFF7F6B8603B0020002C0140EC
:10AD08002DE9F04104684A4DA30AAB4272D009D834
:10AD1800B3F5801F6AD04A3DAB425AD14FF0700E4E
:10AD2800022608E0434DAB4268D00335AB4252D10E
:10AD38004FF0C00E042647794FEA970C002961D0DE
:10AD4800B000634685190227D4F80C809F400CEBAD
:10AD58004503BFB2384D03F1040C47EA080745F82C
:10AD6800231045F82C20E760EFF31181502282F37D
:10AD78001288821905EBC202136973B31362043394
:10AD8800821905EBC202576917B11F605369043372
:10AD9800821905EBC202976917B11F6093690433E2
:10ADA800821905EBC202D76917B11F60D369043352
:10ADB8000027CAB21F6082F31188304405EBC00037
:10ADC800036A6BB9E3684FF6FE721340E360BDE8AF
:10ADD800F081BDE8F081BDE8F08105EB0E03CFE717
:10ADE800E36843F00103E360BDE8F0814FF0480EEB
:10ADF8000126A0E74FF0200E00269CE74FF0980EA2
:10AE0800032698E7BF08022306FA03F0BB40DB439A
:10AE1800E768094D9BB23B4087190CEB470CE36090
:10AE28000CF1040345F82C1045F823209CE700BFDB
:10AE38004B0010004D001000603B00201F4B984253
:10AE48002CD0B0F1804F2BD0A3F59433984229D061
:10AE580003F58063984227D003F50063984225D014
:10AE680003F58063984223D003F59033984221D0AC
:10AE780003F5406398421FD003F58063984207D0DA
:10AE880003F58063984208BF092202D0002070476A
:10AE980008220B4B03EBC203187970470022F8E72E
:10AEA8000122F6E70222F4E70322F2E70422F0E7A0
:10AEB8000522EEE70622ECE70722EAE7002C01402C
:10AEC800D40003082DE9F04F013085B0C3B20393D5
:10AED8008E4D8F4F8F4C904E0A2302933220DFF80D
:10AEE80040921CF0ADFF4FF4FA7A4FF0100C4FF47B
:10AEF8007A70D9F80430C3F30803002B40F0C880F7
:10AF0800EFF31183002B40F0C3802968A26800BFCB
:10AF18002B689942F9D1D7F800E000FB0EF39B1A91
:10AF2800B3FBFEF300FB01314FF0010E0191D9F89C
:10AF38000430C3F30803002B40F08E80EFF3118335
:10AF4800002B40F089802B68A16800BF2A689342D3
:10AF5800F9D1D7F800B000FB0BF2521AB2FBFBF2A2
:10AF680000FB0323019A9B1AB3F57A7FDFD3BAF16A
:10AF7800010ABED1039B002B40F0C4804FF47A7ABB
:10AF8800DFF89C9150464FF0100CD9F80430C3F309
:10AF98000803002B40F09980EFF31183002B40F059
:10AFA80094802968A26800BF2B689942F9D1D7F824
:10AFB80000E000FB0EF39B1AB3FBFEF300FB01312C
:10AFC8004FF0010E0191D9F80430C3F308033BBBDD
:10AFD800EFF3118323BB2B68A16800BF2A68934253
:10AFE800F9D1D7F800B000FB0BF2521AB2FBFBF212
:10AFF80000FB0323019A9B1AB3F57A7FE3D3BAF1D6
:10B00800010AC2D1029B013B02937FF467AF434917
:10B01800434B4448444A0860DA6005B0BDE8F08F05
:10B02800EFF311888CF31288A1682368DB0344BF0F
:10B03800C6F800E0A1682B6832685FFA88F888F3E0
:10B048001188D7F800801A4400FB08F35B1AB3FB99
:10B05800F8F300FB0233CDE7EFF311888CF3128885
:10B06800A1682368DB0344BFC6F800E0A1682B6829
:10B0780032685FFA88F888F31188D7F800801A4494
:10B0880000FB08F35B1AB3FBF8F300FB023369E734
:10B09800EFF311828CF31288D4F808E02368D903FF
:10B0A80003D501233360D4F808E02B683168D2B2A5
:10B0B80082F311883A68194400FB02F3A3EB0E03EC
:10B0C800B3FBF2F300FB01312EE7EFF311828CF3AF
:10B0D8001288D4F808E02368D90303D50123336024
:10B0E800D4F808E02B683168D2B282F311883A6844
:10B0F800194400FB02F3A3EB0E03B3FBF2F300FBCE
:10B1080001315DE718461CF041FD37E79C590020E6
:10B11800A059002010E000E098590020FC9F002072
:10B1280000ED00E0EFBEADDE0400FA052DE9F04FBA
:10B13800013085B0C3B203930B4602918B4C8C4E01
:10B14800002B00F09A8032208A4D8B4FDFF82C922A
:10B158001CF076FE4FF4FA7A4FF0100C4FF47A7028
:10B16800D9F80430C3F30803002B40F0DE80EFF376
:10B178001183002B40F0D9802968A26800BF2B6892
:10B188009942F9D1D7F800E000FB0EF39B1AB3FB04
:10B19800FEF300FB01314FF0010E0191D9F80430A4
:10B1A800C3F30803002B40F08780EFF31183002BD3
:10B1B80040F082802B68A16800BF2A689342F9D1C9
:10B1C800D7F800B000FB0BF2521AB2FBFBF200FBFF
:10B1D8000323019A9B1AB3F57A7FDFD3BAF1010AE8
:10B1E800BED1039B002B40F0BD804FF47A7ADFF884
:10B1F8008C9150464FF0100CD9F80430C3F3080373
:10B20800002B75D1EFF31183002B71D12968A26847
:10B2180000BF2B689942F9D1D7F800E000FB0EF384
:10B228009B1AB3FBFEF300FB01314FF0010E0191B5
:10B23800D9F80430C3F3080313BBEFF31183FBB948
:10B248002B68A16800BF2A689342F9D1D7F800B0EB
:10B2580000FB0BF2521AB2FBFBF200FB0323019A2C
:10B268009B1AB3F57A7FE3D3BAF1010AC4D1029BE2
:10B27800013B0293002B7FF466AF05B0BDE8F08F69
:10B28800EFF311888CF31288A1682368DB0344BFAD
:10B29800C6F800E0A1682B6832685FFA88F888F37E
:10B2A8001188D7F800801A4400FB08F35B1AB3FB37
:10B2B800F8F300FB0233D2E7EFF311888CF312881E
:10B2C800A1682368DB0344BFC6F800E0A1682B68C7
:10B2D80032685FFA88F888F31188D7F800801A4432
:10B2E80000FB08F35B1AB3FBF8F300FB023370E7CB
:10B2F800EFF311828CF31288D4F808E02368D9039D
:10B3080003D501233360D4F808E02B683168D2B242
:10B3180082F311883A68194400FB02F3A3EB0E0389
:10B32800B3FBF2F300FB01317FE7EFF311828CF3FB
:10B338001288D4F808E02368D90303D501233360C1
:10B34800D4F808E02B683168D2B282F311883A68E1
:10B35800194400FB02F3A3EB0E03B3FBF2F300FB6B
:10B36800013118E718461CF011FC3EE710E000E038
:10B37800985900209C590020A059002000ED00E0B9
:10B38800204B5B68C3F3080330B4BBB9EFF31183F8
:10B39800A3B91D4B1D4C1868A16800BF1A689042DC
:10B3A800F9D11B4B1C684FF47A7202FB04F3591A4B
:10B3B800B1FBF4F130BC02FB00107047EFF31182CF
:10B3C800102383F3128811498C680B6813F4803FAB
:10B3D800104B02D0012018608C680B49D2B20D685E
:10B3E800186882F311880A4B19684FF47A72284456
:10B3F80002FB01F31B1B30BCB3FBF1F302FB003073
:10B40800704700BF00ED00E09C59002010E000E00C
:10B41800A0590020985900202DE9F84F8046FFF7E1
:10B42800AFFF254E2549DFF8A0E0254A254D844683
:10B4380010274FF47A740120DEF80430C3F30803B0
:10B44800D3B9EFF31183BBB90B68D2F808A000BFDA
:10B45800D1F800904B45F7D1D6F800B004FB0BF9B2
:10B46800A9EB0A09B9FBFBF904FB0393A3EB0C0353
:10B478004345E1D3BDE8F88FEFF3118A87F31288CB
:10B48800D2F808B01368DB0344BF2860D2F808B0CC
:10B498000B68D5F800905FFA8AFA8AF31188D6F813
:10B4A80000A0994404FB0AF3A3EB0B03B3FBFAF3E4
:10B4B80004FB0933DAE700BFA05900209C5900209B
:10B4C80010E000E09859002000ED00E02DE9F04F71
:10B4D800DFF830C1474A4849484E494D8046102751
:10B4E80018F1FF38C0F08480DCF80430C3F3080397
:10B4F800002B5CD1EFF31183002B58D10B689468B3
:10B5080000BF08688342F9D1D6F800904FF47A70EA
:10B5180000FB09FEAEEB040EBEFBF9FE00FB03EEDA
:10B52800DCF80430C3F308034FF47A740120FBB944
:10B53800EFF31183E3B90B68D2F808A000BFD1F884
:10B5480000904B45F7D1D6F800B004FB0BF9A9EBF6
:10B558000A09B9FBFBF904FB0393A3EB0E03B3F54C
:10B568007A7FBDD2DCF80430C3F30803002BDFD0A8
:10B57800EFF3118A87F31288D2F808B01368DB0357
:10B5880044BF2860D2F808B00B68D5F800905FFA7D
:10B598008AFA8AF31188D6F800A0994404FB0AF3C2
:10B5A800A3EB0B03B3FBFAF304FB0933D5E7EFF383
:10B5B800118487F31288D2F808901368D80303D54A
:10B5C80001232B60D2F808900B682868E4B284F352
:10B5D8001188D6F800A04FF47A7400EB030E04FB30
:10B5E8000AF3A3EB0903B3FBFAF304FB0E3E97E758
:10B5F800BDE8F08F10E000E09C590020A059002021
:10B608009859002000ED00E030B4EFF311831022C8
:10B6180082F312880649074C0A6807480132002558
:10B628000A602560DBB2026883F3118830BC70477A
:10B638009C5900209859002010E000E01D4B70B57F
:10B648009C68E36C226BDD69C2B1636B2BB12B077D
:10B6580002D5E36C08221A6270BD2A06F7D5A26AE1
:10B66800616A8A421FD0511CA069A162825C20696C
:10B67800E66C81423285EAD3A362E8E7A906E4D5FD
:10B68800E26A1AB1988C80B29047DEE7E1699B8C38
:10B698006069DBB24E1CE6614354E169E368994294
:10B6A80028BFE261D1E7E26C136823F080031360DE
:10B6B800CDE700BF7C2B002070B4EFF31186502338
:10B6C80083F31288436B1A68D20720D45D686DB97A
:10B6D800446A826A944217D081691144D9600ED9AC
:10B6E800A21A5A608462002280F850201A6842F038
:10B6F8000102F1B21A6081F3118870BC70470169C8
:10B708008A1A5A608562EEE7012380F85030F1B258
:10B7180081F3118870BC704703682DE9F041DF6937
:10B728001FB13B46BDE8F0411847002A164611DD17
:10B7380004460D460E4400E023689B68204698475F
:10B748000028F9D0236815F8011B1B682046984784
:10B75800AE42F1D1BDE8F08103689B69184700BF8C
:10B7680003685B69184700BF0368DB68184700BFB8
:10B7780003685B68184700BF03681B68184700BF69
:10B78800054B53F8203033B11A689B88918A0B42D5
:10B7980018BF1B04936170478C590020036803F19C
:10B7A80038422DE9F04F920A584DAA5C02F01F0565
:10B7B80052090124022A04FA05F400F08C80032AB5
:10B7C80000F08E80012A3CD001F003077A1E012A7E
:10B7D800C1F3810CC1F300188088C1F3411135D938
:10B7E800C60700F19780850700F1A380440700F1A0
:10B7F800B180020700F1BF80C60600F1CD80850642
:10B8080000F1DB80440600F1E980020600F1F780D0
:10B81800C60500F10581850500F11381440500F195
:10B828002181020500F12F81C60400F13D818504C4
:10B8380000F14B81440400F15981020455D4BDE85C
:10B84800F08F334A55692C435461BDE700242246E2
:10B858004FF0010E4FF0030904E00132102A04F101
:10B868000204ECD00EFA02F636EA0005F5D1D3F858
:10B8780008A009FA04F5ED430AEA050AC3F808A086
:10B88800D3F808B00CFA04FA4AEA0B0AC3F808A07D
:10B89800B3F804A01FFA8AFA2AEA06069E80B3F8CB
:10B8A80004A008FA02F646EA0A06B6B29E801E68A6
:10B8B8002E401E60D3F800A007FA04F646EA0A06EE
:10B8C8001E60D3F80CA001FA04F605EA0A0A46EA53
:10B8D8000A05DD60C1E70E4A95692C43946173E758
:10B8E8000B4AD5692C43D4616EE71A6822F04042AE
:10B8F8001A601A6842EA87771F60DA6822F04042C5
:10B9080042EA8171D960BDE8F08F00BF28010308C1
:10B91800001002401A6822F003021A601A683A43BB
:10B928001A60DA6822F003020A438507DA607FF5B5
:10B938005DAF1A6822F00C021A601A6842EA8702A0
:10B948001A60DA6822F00C0242EA81024407DA60DF
:10B958007FF54FAF1A6822F030021A601A6842EA7F
:10B9680007121A60DA6822F0300242EA0112DA603D
:10B9780002077FF541AF1A6822F0C0021A601A6800
:10B9880042EA87121A60DA6822F0C00242EA81129B
:10B99800C606DA607FF533AF1A6822F440721A607F
:10B9A8001A6842EA07221A60DA6822F4407242EA08
:10B9B80001228506DA607FF525AF1A6822F4406215
:10B9C8001A601A6842EA87221A60DA6822F440622A
:10B9D80042EA81224406DA607FF517AF1A6822F43A
:10B9E80040521A601A6842EA07321A60DA6822F48A
:10B9F800405242EA0132DA6002067FF509AF1A685E
:10BA080022F440421A601A6842EA87321A60DA68F9
:10BA180022F4404242EA8132C605DA607FF5FBAE85
:10BA28001A6822F440321A601A6842EA07421A6019
:10BA3800DA6822F4403242EA01428505DA607FF58D
:10BA4800EDAE1A6822F440221A601A6842EA874268
:10BA58001A60DA6822F4402242EA81424405DA6038
:10BA68007FF5DFAE1A6822F440121A601A6842EABB
:10BA780007521A60DA6822F4401242EA0152DA6088
:10BA880002057FF5D1AE1A6822F440021A601A68DE
:10BA980042EA87521A60DA6822F4400242EA815286
:10BAA800C604DA607FF5C3AE1A6822F040721A60E5
:10BAB8001A6842EA07621A60DA6822F0407242EABB
:10BAC80001628504DA607FF5B5AE1A6822F040623B
:10BAD8001A601A6842EA87621A60DA6822F04062DD
:10BAE80042EA81624404DA607FF5A7AE1A6822F060
:10BAF80040521A601A6842EA07721A60DA6822F03D
:10BB0800405242EA0172DA6097E600BF2DE9F04F31
:10BB18004A484B4B4B4C4FF090414FF0010A4FF0C5
:10BB280002094FF004084FF0080C4FF0100E2027C0
:10BB38004026802530F8022B12F0010F03D019603F
:10BB4800A3F804A0083312F0020F03D01960A3F879
:10BB58000490083312F0040F03D01960A3F804808E
:10BB6800083312F0080F03D01960A3F804C0083393
:10BB780012F0100F03D01960A3F804E0083312F094
:10BB8800200F02D019609F80083312F0400F02D0B6
:10BB980019609E80083312F0800F02D019609D80D2
:10BBA800083312F4807F05D04FF4807B1960A3F826
:10BBB80004B0083312F4007F05D04FF4007B1960FD
:10BBC800A3F804B0083312F4806F05D04FF4806BEB
:10BBD8001960A3F804B0083312F4006F05D04FF4CD
:10BBE800006B1960A3F804B0083312F4805F05D025
:10BBF8004FF4805B1960A3F804B0083312F4005FB7
:10BC080005D04FF4005B1960A3F804B0083312F4B0
:10BC1800804F05D04FF4804B1960A3F804B0083367
:10BC2800D20B04D04FF4004219609A80083301F512
:10BC38008061A1427FF47EAFBDE8F08FC8010308A0
:10BC4800245A002000180048002852D0036803F145
:10BC580038422DE9F04F920A504DAA5C02F01F05B8
:10BC680052090124022A04FA05F443D0032A00F0F9
:10BC78009080012A43D001F003077A1E012AC1F3FC
:10BC8800810CC1F300188088C1F341113CD9C60763
:10BC980000F18880850700F19480440700F1A280B4
:10BCA800020700F1B080C60600F1BE80850600F1EB
:10BCB800CC80440600F1DA80020600F1E880C6056F
:10BCC80000F1F680850500F10481440500F1128138
:10BCD800020500F12081C60400F12E81850400F1DF
:10BCE8003C81440400F14A81020400F15881BDE816
:10BCF800F08F70472A4A95692C439461BBE7284A1C
:10BD080055692C435461B6E7002422464FF0010ED2
:10BD18004FF0030904E00132102A04F10204E6D0CE
:10BD28000EFA02F636EA0005F5D1D3F808A009FAAA
:10BD380004F5ED430AEA050AC3F808A0D3F808B0E9
:10BD48000CFA04FA4AEA0B0AC3F808A0B3F804A0EC
:10BD58001FFA8AFA2AEA06069E80B3F804A008FAAF
:10BD680002F646EA0A06B6B29E801E682E401E609B
:10BD7800D3F800A007FA04F646EA0A061E60D3F8CC
:10BD88000CA001FA04F605EA0A0A46EA0A05DD608B
:10BD9800C1E7034AD5692C43D4616CE7280103083D
:10BDA800001002401A6822F003021A601A683A4327
:10BDB8001A60DA6822F003020A438507DA607FF521
:10BDC8006CAF1A6822F00C021A601A6842EA8702FD
:10BDD8001A60DA6822F00C0242EA81024407DA604B
:10BDE8007FF55EAF1A6822F030021A601A6842EADC
:10BDF80007121A60DA6822F0300242EA0112DA60A9
:10BE080002077FF550AF1A6822F0C0021A601A685C
:10BE180042EA87121A60DA6822F0C00242EA811206
:10BE2800C606DA607FF542AF1A6822F440721A60DB
:10BE38001A6842EA07221A60DA6822F4407242EA73
:10BE480001228506DA607FF534AF1A6822F4406271
:10BE58001A601A6842EA87221A60DA6822F4406295
:10BE680042EA81224406DA607FF526AF1A6822F496
:10BE780040521A601A6842EA07321A60DA6822F4F5
:10BE8800405242EA0132DA6002067FF518AF1A68BA
:10BE980022F440421A601A6842EA87321A60DA6865
:10BEA80022F4404242EA8132C605DA607FF50AAFE1
:10BEB8001A6822F440321A601A6842EA07421A6085
:10BEC800DA6822F4403242EA01428505DA607FF5F9
:10BED800FCAE1A6822F440221A601A6842EA8742C5
:10BEE8001A60DA6822F4402242EA81424405DA60A4
:10BEF8007FF5EEAE1A6822F440121A601A6842EA18
:10BF080007521A60DA6822F4401242EA0152DA60F3
:10BF180002057FF5E0AE1A6822F440021A601A683A
:10BF280042EA87521A60DA6822F4400242EA8152F1
:10BF3800C604DA607FF5D2AE1A6822F040721A6041
:10BF48001A6842EA07621A60DA6822F0407242EA26
:10BF580001628504DA607FF5C4AE1A6822F0406297
:10BF68001A601A6842EA87621A60DA6822F0406248
:10BF780042EA81624404DA607FF5B6AE1A6822F0BC
:10BF880040521A601A6842EA07721A60DA6822F0A8
:10BF9800405242EA0172DA6002047FF5A8AE1A68DC
:10BFA80022F040421A601A6842EA87771F60DA680E
:10BFB80022F0404242EA8171D960BDE8F08F00BFAB
:10BFC80010B1036882881A85704700BF10B10368F2
:10BFD80082889A61704700BF38B100298388026857
:10BFE80014BF002110218B409361704710B40A4B95
:10BFF8000A4A1C7801238340234052F8200029B9BB
:10C00800B3FA83F149095DF8044BE5E7191C18BF39
:10C0180001215DF8044BDFE7885900208C59002086
:10C0280030B1036882881B8A1A4214BF012000209D
:10C03800704700BF2DE9F0410B4E346873691C400E
:10C048000FD0DFF828800127B4FA84F3C3F11F0367
:10C0580007FA03F558F8230003689847AC4375615D
:10C06800F2D1BDE8F08100BF00040140AC590020C6
:10C078002DE9F0410B4E346873691C400FD0DFF88E
:10C0880028800127B4FA84F3C3F11F0307FA03F5E4
:10C0980058F8230003689847AC437561F2D1BDE8AE
:10C0A800F08100BF00040140AC5900202DE9F041A7
:10C0B8000B4E346873691C400FD0DFF828800127C5
:10C0C800B4FA84F3C3F11F0307FA03F558F8230001
:10C0D80003689847AC437561F2D1BDE8F08100BFB1
:10C0E80000040140AC5900202DE9F0410B4E3468A2
:10C0F80073691C400FD0DFF828800127B4FA84F355
:10C10800C3F11F0307FA03F558F82300036898479B
:10C11800AC437561F2D1BDE8F08100BF0004014075
:10C12800AC5900202DE9F0410B4E346873691C406E
:10C138000FD0DFF828800127B4FA84F3C3F11F0376
:10C1480007FA03F558F8230003689847AC4375616C
:10C15800F2D1BDE8F08100BF00040140AC590020D5
:10C168002DE9F0410B4E346873691C400FD0DFF89D
:10C1780028800127B4FA84F3C3F11F0307FA03F5F3
:10C1880058F8230003689847AC437561F2D1BDE8BD
:10C19800F08100BF00040140AC5900202DE9F041B6
:10C1A8000B4E346873691C400FD0DFF828800127D4
:10C1B800B4FA84F3C3F11F0307FA03F558F8230010
:10C1C80003689847AC437561F2D1BDE8F08100BFC0
:10C1D80000040140AC590020A8B18388B3FA83F366
:10C1E800C3F11F035A1C08D0012202FA03F329B92C
:10C1F80007490A6822EA03030B607047044A11687A
:10C208000B431360704701230029F1D0F6E700BF04
:10C2180000040140084A094808B5936943F001033E
:10C2280093610021402221F0B0FB054B4FF0FF3213
:10C238001A60C3F8032008BD00100240AC59002062
:10C24800EC5900202DE9F041044618460D461646E3
:10C2580098461FF0F9FA2768E6722844A072294622
:10C268007D69434632462046AC46BDE8F04160470A
:10C27800036810B504461B689847236820469B68E6
:10C288009847A37B0133A37310BD00BF2DE9F04786
:10C29800B0F908500D81EDB2382D8CB00C4600F085
:10C2A800598106462ED9802D00F0A98077D8522DC5
:10C2B80000F0998040F24481542D00F09B816E2D4E
:10C2C80040F0FB80B64B0A681B88B64DFF2BA8BF11
:10C2D800FF23511C21601370A96881F3100189B2F2
:10C2E8002046F4F7EFFFB04B20461988F4F7EAFF31
:10C2F800296801F30F0189B220460125F4F7E2FF0E
:10C308002B4647E0042D00F0C78140F2EE80202D37
:10C3180000F0B78040F20081242D00F06381282DC1
:10C3280040F0CB800B68DFF8B882A04E591C02227F
:10C3380021601A70236806275A1C22601F70236820
:10C348000A22591C21601A70236801255A19226093
:10C358001D70B8F800102046F4F7B4FFB8F80210C2
:10C368002046F4F7AFFF23685A1922601F7023682C
:10C378005022591921601A70236800225919216026
:10C388001A7031882046F4F79DFF71882046F4F72B
:10C3980099FF2B46284663810CB0BDE8F087822DB3
:10C3A80047D0C0F03F81A02D00F03081FE2D40F035
:10C3B80084807F4D05F1080635F8021B2046F4F706
:10C3C80081FFB542F8D101252B46284663810CB080
:10C3D800BDE8F0870B680322591C21601A70236896
:10C3E800591C21601A7022680021531C0125236002
:10C3F80028462B46117063810CB0BDE8F0876D4B61
:10C408001D780B3D15F0FF05DDD06B4F00220A2685
:10C4180021683B88481C20600E702168FF2B02F1C0
:10C428000102A8BFFF23481C954220600B70EFDC77
:10C43800C9E70B68614A5B4D1178614A581C206056
:10C44800197011892046F4F73DFF554B22681B8867
:10C45800FF2B02F10101A8BFFF2321601370A96817
:10C4680081F3100189B22046F4F72CFF296801F303
:10C478000F0189B22046F4F725FF524B226819783C
:10C48800B3E70B684E4D591C6A7821601A7023680F
:10C498002A78591C21601A702368AA78591C2160CF
:10C4A8001A7029892046F4F70DFF23686A79591C08
:10C4B80021601A702268A97997E72146284603F077
:10C4C80055F9014600287FF47EAF742D00F0F68000
:10C4D800772D40F01381336872689A4240F00683E2
:10C4E800394A204618F0FCF96DE7022D00F0DE808D
:10C4F8003FF670AF012DE0D10B680022591C216076
:10C508001A7023685A1C22601D7022682521531C4A
:10C5180023602B4611703DE7052DCED10B222B4908
:10C528002046F4F79FFE082229492046F4F79AFE90
:10C538000125072227492046F4F794FE2B4629E7D0
:10C54800442DBAD1002A3FF43EAF234B1360012596
:10C558002B461FE70A68214B0125511C21601570E5
:10C568002268052150192060117022680A2150198B
:10C578002060117022680021501920601170226813
:10C588001978501920601170226859785019206064
:10C59800117022689978531923602B461170F9E6B7
:10C5A800C85B0020BC5B0020603D002054280020B0
:10C5B800305C0020F05E0020642800204A5C0020E7
:10C5C8006C3D0020663D0020513C0208D40403085D
:10C5D800E0040308EC0403085DF700089D3500201B
:10C5E8007C4200203A4B196820460125F4F752FE98
:10C5F8002B46EAE60B6800215A1C22601970226853
:10C608000125531923602B461170C3E6314B0846A8
:10C618001968F4F73FFE304B20461968F4F73AFEE4
:10C628002E4BE0E72E4B1E780A3E16F0FF063FF42D
:10C63800CAAE2C4B2C4F1E4403F101080A2314E008
:10C64800502B01F00D80002529462268501C2060DF
:10C6580020461370F4F736FE29462046F4F732FEDA
:10C6680046453FF4B0AE18F8013B0A2BE8D11F4A03
:10C678009568116805EB85054FF6FF726D009542C8
:10C68800A8BF15469142A8BF114625EAE57521EADB
:10C69800E171ADB289B2D8E720462A461449F4F7C9
:10C6A800E1FD00212046F4F70DFE9CE60422114925
:10C6B80020460125F4F7D6FD2B466BE633687268F1
:10C6C8009A4240F00F820C4A204618F009F97AE69F
:10C6D80004370020ACF7FF1FB0F7FF1FB4F7FF1FA8
:10C6E800F05E002090DF0208582800202028002053
:10C6F8005D510020CC0403088D470208292D3768B6
:10C7080000F0F881392D00F0CF87212D00F0AC879B
:10C7180072680B3DD31BEF2D00F2648201A050F824
:10C7280025F000BFA9D50008EDCB0008EDCB000827
:10C73800EDCB0008EDCB0008EDCB0008EDCB0008F1
:10C74800EDCB0008EDCB0008EDCB0008EDCB0008E1
:10C75800EDCB0008EDCB0008EDCB0008EDCB0008D1
:10C76800EDCB0008EDCB0008EDCB0008EDCB0008C1
:10C77800EDCB0008EDCB0008EDCB0008EDCB0008B1
:10C78800EDCB0008F9D50008EDCB0008DFD500088F
:10C79800EDCB000887D50008EDCB0008EDCB0008ED
:10C7A800EDCB00085FD50008EDCB000805D50008E3
:10C7B800EDCB00089FD40008EDCB000879D4000821
:10C7C800EDCB000867D40008EDCB000813D40008AF
:10C7D800EDCB000877D30008EDCB0008EDCB0008BF
:10C7E800EDCB0008EDCB0008CFC30008EDCB000867
:10C7F8004BD30008EDCB0008EDCB000831D300087F
:10C80800EDCB000889D20008EDCB0008EDCB00087D
:10C81800EDCB0008EDCB0008EDCB0008EDCB000810
:10C82800EDCB0008EDCB000849D20008EDCB00089D
:10C83800E3D20008EDCB0008EDCB000801D10008D9
:10C84800EDCB0008EDCB0008EDCB0008EDCB0008E0
:10C85800EDCB0008EDCB0008EDCB00087DD100083A
:10C86800EDCB00088DD00008EDCB000823D00008E0
:10C87800EDCB000881CF0008EDCB000859CF0008A8
:10C888003BCF00081FCF0008EDCB0008EDCB000818
:10C89800EDCB0008EDCB0008EDCB0008EDCB000890
:10C8A800EDCB0008EDCB0008EDCB0008EDCB000880
:10C8B800EDCB0008EDCB0008EDCB0008EDCB000870
:10C8C800EDCB0008EDCB0008EDCB0008EDCB000860
:10C8D800EDCB0008EDCB0008EDCB0008EDCB000850
:10C8E800EDCB0008EDCB0008EDCB0008EDCB000840
:10C8F800EDCB0008EDCB0008EDCB0008EDCB000830
:10C90800EDCB0008EDCB0008EDCB0008EDCB00081F
:10C91800EDCB0008EDCB0008EDCB0008EDCB00080F
:10C92800EDCB0008EDCB0008EDCB0008EDCB0008FF
:10C93800EDCB0008EDCB0008EDCB0008EDCB0008EF
:10C94800EDCB0008EDCB0008EDCB0008EDCB0008DF
:10C95800EDCB0008EDCB0008EDCB0008EDCB0008CF
:10C96800EDCB0008EDCB0008EDCB0008EDCB0008BF
:10C97800EDCB0008EDCB0008EDCB0008EDCB0008AF
:10C98800EDCB0008EDCB0008EDCB0008EDCB00089F
:10C99800EDCB0008EDCB0008EDCB0008EDCB00088F
:10C9A800EDCB0008EDCB0008EDCB0008EDCB00087F
:10C9B800EDCB0008EDCB0008EDCB0008EDCB00086F
:10C9C800EDCB0008EDCB0008EDCB0008EDCB00085F
:10C9D800EDCB0008F5CE0008EDCB0008EDCB000844
:10C9E800EDCB0008EDCB0008EDCB0008EDCB00083F
:10C9F800EDCB0008EDCB0008EDCB0008EDCB00082F
:10CA0800EDCB0008EDCB0008EDCB0008EDCB00081E
:10CA1800EDCB0008EDCB000899CE0008EDCB00085F
:10CA280061CE0008EDCB0008C5CD000869CD00082F
:10CA38004DCD0008EDCB000833CD0008EDCB000844
:10CA48000BCD0008EDCB0008B1CC0008EDCB0008F9
:10CA580083CC0008EDCB0008EDCB000861CC0008C2
:10CA680033CC00081FCC0008F7CB0008CFCB000858
:10CA7800ADCB0008EDCB0008EDCB0008EDCB0008EE
:10CA8800EDCB0008EDCB0008EDCB0008EDCB00089E
:10CA9800EDCB0008EDCB0008EDCB0008EDCB00088E
:10CAA800EDCB0008EDCB0008EDCB0008EDCB00087E
:10CAB800EDCB000893CB0008EDCB0008EDCB0008C8
:10CAC8003DCB0008EDCB0008EDCB0008EDCB00080E
:10CAD800EDCB0008EDCB0008EDCB0008EDCB00084E
:10CAE80027CB00085A1C32601978ECE55A1C3260D2
:10CAF8001978F5E47B1C33603B780A2B00F0E48559
:10CB0800502B40F0E2833046F4F79AFB9B4F388075
:10CB18003046F4F795FB012578802B463AE4984B8C
:10CB28001B78DB075ED4012503F014FE03F0BCFE7E
:10CB38002B462FE47B1C33603B780F2B52D8BA1C52
:10CB48003260C3EBC3038F4A7978D154F91C316042
:10CB58001344BA785A703A1D3260FA789A707A1D7E
:10CB680032603A79DA70BA1D32607A791A71FA1D30
:10CB78003260BA795A7107F108023260FA799A710B
:10CB8800012509F0FBF82B4604E43046F4F758FB7E
:10CB98007D4FF8813046F4F753FB0125B8812B46C9
:10CBA800FFF7F8BB3046F4F74BFB784F3882304636
:10CBB800F4F746FB78823046F4F742FB0125B88249
:10CBC8002B46FFF7E7BB3B467A1C326013F8020B93
:10CBD8003360FB1C79783360BA7810F059FE00286E
:10CBE8007FF4F1AB4FF0FF352B46FFF7D3BB3B4645
:10CBF8007A1C3260664A13F8021B11703360624A6D
:10CC08007B789370FB1C3360624BBA789A7001256D
:10CC18002B46FFF7BFBB604B604918684E220125C1
:10CC28001FF0CAFD2B46FFF7B5BB3A467B1C3360A5
:10CC38005B4B12F8021B197032607A785A70FA1C32
:10CC48003260BA789A703046F4F7FAFA554B0125F3
:10CC5800D8802B46FFF79EBB3046F4F7F1FA514FC8
:10CC680038803046F4F7ECFA78803046F4F7E8FA82
:10CC78000125B8802B46FFF78DBBDFF8388198F87F
:10CC88000030002B3FF49FAB474F00253046F4F7A8
:10CC9800D7FA09F0E5FD98F80030A7EC010A01354C
:10CCA8009D42F3DBFFF78FBB0D2B9BD17B1C3360C1
:10CCB8003D78072D96D8DFF8008130460C27F4F729
:10CCC800BFFA07FB05F708EB0705A8803046F4F71D
:10CCD800B7FAE8803046F4F7B3FA336828811A4681
:10CCE800591C316012F8021BA97232605B78EB7232
:10CCF8003046F4F78DFA012548F807002B46FFF770
:10CD080049BB7B1C33603878060600F14D851C4B07
:10CD18001B78DD073FF557AB032828BF0020012506
:10CD280003F000FD2B46FFF735BB154B1B78D807E2
:10CD38003FF549AB012503F0A5FF03F0B5FD2B46F0
:10CD4800FFF728BB0E4B1B78DA073FF53CAB174AB9
:10CD58001378012543F0040313702B46FFF71ABB21
:10CD6800074B1B78D9073FF52EAB114B4FF4C87210
:10CD780001251A802B46FFF70DBB00BF5428002061
:10CD8800FC480020DC2F00208C4200207049002045
:10CD9800885400209C420020645100202CF2020894
:10CDA80084420020D02700209031002078480020BD
:10CDB800F45F0020F05E0020E82E0020092B7FF7AA
:10CDC80011AFDFF8A4833B467A1CD8F800503260D4
:10CDD80013F8022B2A7033607B78AB70FB1C33602E
:10CDE800BB78642BA8BF64233A1D6B713260FB7853
:10CDF800642BA8BF64237A1DAB7132603B79EB7159
:10CE0800BB1D33607B79642BA8BF6423FA1D2B728A
:10CE18003260BB79EB7007F108033360FB792B7143
:10CE28003046F4F70DFA726833686881D11A002920
:10CE38000CDD591CD8F800003160521A002A197804
:10CE4800417203DD9A1C32605B78437001251DF046
:10CE5800ADFE2B46FFF79EBAB74B1868FB1C02467F
:10CE68002137991E316013F8031C1170591E316067
:10CE780013F8021C5170336013F8011C91700333CE
:10CE88009F4202F10302ECD109F0A8FBFFF79BBA1D
:10CE9800C3F34705122D3FF6A5AEBDB10CAB0DF19E
:10CEA8000A0803EB45094746A9F126093046F4F775
:10CEB800C7F927F8020F4F45F8D1A04B38F8022FD1
:10CEC80023F8022F4745F9D1112D09D89C4A6B0048
:10CED800023B13440021223223F8021F9A42FBD15D
:10CEE800984A01231D461370FFF754BA3B467A1C33
:10CEF800326013F8025B3360FB1C78783360B978D2
:10CF0800002D00F05C84012D7FF45DAA05F042FF3E
:10CF18002B46FFF73FBA7B1C33603B78002B00F0B1
:10CF280022844FF4004001251DF022F92B46FFF71B
:10CF380031BA854B1B7813F001017FF453AE7B1C8B
:10CF480033603878012505F067FE2B46FFF722BAD3
:10CF58003B467A1C32607D4A13F8021BD17033605D
:10CF68007B4A7B785371FB1C33607A4BBA78DA7052
:10CF780001252B46FFF70EBA3046F4F761F9304623
:10CF8800F4F75EF93046F4F75BF93046F4F764F9E4
:10CF98003368694D1946581C2A68306011F8020B2D
:10CFA80082F82C003160597882F83610D91C31602B
:10CFB8009B7882F837303046F4F74EF93046F4F76C
:10CFC8004BF93046F4F748F930462F68F4F738F94A
:10CFD800788730462F68F4F733F9336872683887F2
:10CFE800D11A01290ADD591C2A6831601B7882F898
:10CFF8002E303046F4F730F933687268D31A032BB1
:10D0080009DD30462F68F4F71BF9788630462E681C
:10D01800F4F716F9B086286836E77B1C3360464D6E
:10D02800DFF848813B7888F8053030462F68F4F7F8
:10D0380007F9388430462F68F4F702F972683368C4
:10D04800F883D11A072900F30984D11A032900F3B8
:10D05800F783D21A002A05DD591C2A6831601B782B
:10D0680082F8263003F080FB19F0BEFC3A4B1B68AF
:10D07800002B00F081832868012508F013FF2B4658
:10D08800FFF788B93B467A1C3260DFF8E08013F876
:10D09800022B88F802203360304A7B781370FB1C1F
:10D0A80033602F4DBB782B713B1D3360FB78092B08
:10D0B800A8BF09233046AB70F4F7C2F8336872682A
:10D0C8002880D11A012905DD3046F4F7B9F833680C
:10D0D8007268E8819A4240F0788303F045FB336830
:10D0E80072689A423FF46FA95A1C32601B78EB7041
:10D0F80001252B46FFF74EB91A4B1B78012B3FF63B
:10D1080062A97B1C39463360DFF8648011F8023B62
:10D1180088F80230FB1CD21A3160012A7878336013
:10D1280040F335833046F4F78BF80125A8F8000062
:10D138002B46FFF72FB900BF64510020EA330020C7
:10D14800EC33002010340020FC4800208C420020E2
:10D15800204000209C420020B44200208042002051
:10D1680070490020CF360020D45F0020885400206A
:10D17800D23600203046F4F763F805460DF0D6F9AC
:10D18800FF283FF420A93F2D00F2D6820DF1300888
:10D19800002308F8243DEF0841460DF10B008DF8F7
:10D1A8000B3001370DF0A2F99DF80B30FFB205F0F6
:10D1B8000705BB4205F1010503D19DF80C30AB42D0
:10D1C80003D0294638460DF09DF933687268D21AA3
:10D1D800012A7FF7F8A85A1C0CA8326000221D7893
:10D1E80000F8252D0DF076F99DF80B30AB420AD0EA
:10D1F800B54B1B683BB19A79AA4204D31B681B69DB
:10D208000BB12846984733685A1C326040460022C2
:10D218001D788DF80C200DF051F99DF80C30AB42BB
:10D228003FF4D1A8A84B1B68002B3FF4CCA81B687F
:10D238005B69002B3FF4C7A828469847FFF7C3B897
:10D248003B467A1CA14D326013F8022B2A713360D9
:10D258007B786B713046F3F7F3FF336828805A1CEC
:10D2680032601B78AB713046F3F7EAFF33686880A9
:10D278005A1C32601B78EB7101252B46FFF78AB8E0
:10D288007B1C3360924B3A78DFF868821A7000236F
:10D29800C8F800303046F3F7BBFF3268D8F80030E2
:10D2A8008C498D4D0343501CC8F80030306013780A
:10D2B8000B723046F3F7C4FF28603046F3F7C0FF1F
:10D2C80068603046F3F7BCFFA8603046F3F7B8FF54
:10D2D8003046F3F7B5FFFFF776B87B1C336097F855
:10D2E8000080B8F1110F3FF67DACBB1C33607B4D5D
:10D2F8007B7805F818303046F3F7A2FF40F6CA03EA
:10D308009842A8BF184640F2EE23984205EB480120
:10D31800B8BF18460125A0F2EE222B46192092FB31
:10D32800F0F24A70FFF736B86D4B07F10802013783
:10D33800376017F8011C03F8011FBA42F7D1FFF74D
:10D3480042B83B46791C3160664913F8020B887075
:10D3580033607878487093423FF435A8FB1C3360FB
:10D36800614BBA781A7101252B46FFF713B80722CB
:10D37800B3FBF2F2C2EBC2055B1B7FF433ACD2B253
:10D3880002F1FF395FFA89F9002A3FF41CA8DFF897
:10D3980068A109F101091D462DE09AF90A209A426F
:10D3A80000F0C8819AF912209A427FF41BAC022738
:10D3B8000AEBC708304688F80230F3F741FF3368B4
:10D3C8002AF837001A46591C316012F8021B88F8EF
:10D3D800031032605A7888F80420DA1C32609A7890
:10D3E80088F806201F1D37600135DB7888F805307E
:10D3F800A9453EF4E8AF7B1C336097F900309AF9F1
:10D4080002209A42C9D10027D2E77B1C33603B78BF
:10D418000E2B3FF6E7ABBA1C3260787803283FF64C
:10D42800E1AB3249062202FB03F28B18FD1C58714E
:10D438003560B87888543A1D3260FA785A707A1D87
:10D4480032603A799A70BA1D32607A79DA70FA1DC8
:10D458003260BA791A7101252B46FEF79BBF7B1CF7
:10D4680033601C4B3A785A7501252B46FEF792BF5C
:10D478007A1C32603D781F2D3FF6B4AB052B7FF444
:10D48800B1AB3046F3F7C4FE194B43F8250016F04C
:10D4980029F8FEF798BF164D05F140073046F3F717
:10D4A800CFFE3368A5F88000591C1A46316012F87F
:10D4B800021B85F8821032605B7885F8833004356A
:10D4C800AF42EBD1FEF77FBF08370020EC270020E2
:10D4D800CC420020DC4C0020CC2B002064350020FE
:10D4E800DB4C0020AC420020C82400202D26002060
:10D4F800383C002004370020605B00207B1CB74DBF
:10D5080033603B782B723046F3F79AFEA883304697
:10D51800F3F796FE28833046F3F792FE3268688365
:10D52800531C33601278EA747268D31A032B00F321
:10D53800E2803368D11A052900F37281D21A002AD1
:10D548007EF741AF5A1C32601B7885F821300125DF
:10D558002B46FEF71FBF7B1C3360A1493878087043
:10D56800D21A002A7EF72FAFBB1C33607B780033BA
:10D5780018BF012301254B702B46FEF70BBF304621
:10D58800F3F75EFE974F38603046F3F759FE786040
:10D598003046F3F755FE0125B8602B46FEF7FABE74
:10D5A8009149102B4FF0000228BF10230A604A60EF
:10D5B8008A60CA600A74002B3EF405AF32680139EC
:10D5C80013440132326012F8010C01F8010F934242
:10D5D800F7D1FEF7F8BE854F00233B603046F3F7DE
:10D5E80017FE3B68012503433B602B46FEF7D2BE7E
:10D5F8007B1C33603D780191132D3FF6F3AABB1CC9
:10D608003360787817F0A6F900283FF4EBAA784B36
:10D61800027803F82520FA1C326003EB8505BA78F6
:10D628006A703A1D3260FA78AA707A1D32603A79C7
:10D63800EA7003F15000019902E00433834207D0F5
:10D648001A78002AF9D19D78DA789542F5D2012125
:10D65800684B81F00101012519702B46FEF79ABE2F
:10D66800BD683968FFF706B83B467A1C3260624DE0
:10D6780013F8022B6A7033607B782B70FB1C3360C5
:10D68800BB78AB703046F3F7DBFD33682881591C53
:10D698001A46316012F8021B697132605B78AB710F
:10D6A80001252B46FEF776BE7B1C33603B780A2BA0
:10D6B80010D03046F3F7D0FD3046F3F7CDFD3046B5
:10D6C800F3F7CAFDFEF77FBE3046F3F7B9FD4B4FBF
:10D6D800FFF71DBABB1C3360494B7A781A70FA1CE5
:10D6E8003260BA785A703A1D3260FA789A70012519
:10D6F8002B46FEF74FBE3046F3F7A2FDA88430460E
:10D70800F3F79EFD33687268E884D11A03297FF71E
:10D7180011AF1A46591C316012F8021BA977326002
:10D728005B7885F820303046F3F78AFD33687268F5
:10D738006884FFE601273BE60DF10C0840460CF033
:10D74800B1FEBDF80C30AB423FF43FAD2D4B1B682A
:10D75800002B3FF43AAD1B689B69002B3FF435ADB5
:10D768002846984731E5284A1368012523F40043E1
:10D7780013602B46FEF70EBE24482549254A264B42
:10D78800036001250B6013602B46FEF703BE234B95
:10D79800B9781A88012512FB00F22B4692FBF1F2A8
:10D7A800A8F80020FEF7F6BD00F07F00032828BF88
:10D7B8000020012505F00AFB2B46FEF7EBBD0125ED
:10D7C80008F094FD2B46FEF7E5BD5A1C32601B7825
:10D7D800003318BF012388F807307EE4DC4C0020B2
:10D7E800CC420020CC2B00206842002004370020C7
:10D7F800D0420020F21C00206C3D00207C4200201A
:10D808009D35002008370020A03D0020543000201E
:10D81800A830002010310020F5030008E440002063
:10D828005A1C32601B78EB723046F3F7F1FC336810
:10D83800E8605A1C32601B782B74336872687DE686
:10D848003046F3F7FDFCA8F80E003046F3F7F8FC75
:10D8580033687268A8F81000FFF7FBBB3046F3F78F
:10D86800EFFCA8F80A003046F3F7EAFCA8F80C0029
:10D8780030462F68F3F7E4FC788430462F68F3F7D6
:10D88800DFFC33687268B884FFF7DFBB2DE9F04F1F
:10D898006F4B704A1C7895B000F59C412031814649
:10D8A80008911160002C00F079856B4A126890424B
:10D8B80040F2D581694A6A491768DFF8D8B1694DDD
:10D8C8000492013C03911C7007F48057002F40F02C
:10D8D800D381654B05931E7806F00106039B5B7D9B
:10D8E800002B40F03085049B1B68190400F19F87CA
:10D8F8005E4B9945AB7800F20184002B40F001841F
:10D90800049BD3F800A01AF4805740F0F084DFF8A5
:10D918008891039BBBF90620B3F81A804245B4BF2F
:10D928004FF000084FF00108514B1B6813F080536B
:10D9380000F0D681002E00F0D7810399498C9142DE
:10D9480040F3FF87B8F1000F40F0D681494C94F8B6
:10D95800A020002A40F0D0814749484A086890F83A
:10D968002D000021116051609160002840F0C481B1
:10D97800434A1070002E40F0C581424B1A78002AA5
:10D9880050D10399BBF900E0488B898BBBF9024061
:10D998007045B4BF8026002646F040037145D8BFC5
:10D9A80033469B0843F08006A042B8BF334643F095
:10D9B8004006A142C8BF33469B08BBF90440BBF9E7
:10D9C800066043F0800EA042B8BF734643F0400E95
:10D9D800A142C8BF73469B0843F0800E254C86427F
:10D9E800C8BF734643F0400E94F8A2C08E42B8BF39
:10D9F80073469C4501F04981A4F8A42084F8A62028
:10DA0800214984F8A2300E78002E01F0BD805F2BEA
:10DA180001F0F1806F2B00F0EC87059B1B78DE0787
:10DA280040F1AE87049B194A1B68069203F0040371
:10DA3800002B40F0F58412AF00237B60144C129346
:10DA480040F6330A4FF0190840F2833629E000BF48
:10DA5800C8340020E8330020C434002030570020A8
:10DA6800DC4C00207C3D0020FC480020404B4C0052
:10DA780054420020DC240020645100206040002033
:10DA88002421002033520020F21C0020A83E002050
:10DA9800D0420020AC5F0020204300200434A14580
:10DAA80020D0A278E3789A4218FB0261F6D2627815
:10DAB800043218FB03633BF912205245A8BF5246B3
:10DAC800B2F5617FB8BF4FF461728A42E6DD9A42CF
:10DAD800E4DC21782629E1D838460434F3F7CEFE71
:10DAE800A145DED1AC4BAD4A1B7897E8030082E82C
:10DAF8000300002B00F0D0840121A848F3F7CEFEE4
:10DB0800002840F05782EB78002B40F05382A44F56
:10DB1800A2483C8824F00104A4B202213C80F3F717
:10DB2800BDFE002840F0EB8624F00204A4B23C803D
:10DB38009C4B03931978DFF8BCA2A30708BF81F0B8
:10DB48000201DAF80400C1F34001FEF745FA242186
:10DB58009248F3F7A3FE30B9059A13785E0744BFDD
:10DB680023F004031370069B1B6813F00A0F40F0A0
:10DB780047813C8889480C21F3F790FE002800F083
:10DB8800B082894B1B7844F48074082B3C8000F0E9
:10DB9800B1820E2B00F0AE82049B1B685C0544D555
:10DBA800824B1B79002B00F0D98014217B48F3F7B6
:10DBB80075FE002840F0D7800FF004FB01201CF010
:10DBC80047FA90B3DFF8308200244FF0CC0902E026
:10DBD800DCB2022C29D809FB04F6631C58F806505D
:10DBE800002DF5D1C378724A90F9020052F823301B
:10DBF80001950322009201212A461CF03FF80346B2
:10DC080004EB440000EB0010049353B1294608EBE1
:10DC18008000CC221FF0B9FE049B48F8063001347E
:10DC2800E4B21BF095F90028D3D1059B1B78D807DF
:10DC380040F1CA815F49604A01230B701370039B4E
:10DC4800DAF80000197801F00101FEF7C5F9069B22
:10DC58001B685B0700F1288215B0BDE8F08F574BB1
:10DC6800574A1F68049307F480570392DFF88CB172
:10DC7800544D002F3FF42DAE00214848F3F70EFE17
:10DC880000287FF426AE504B059319461B7813F0F5
:10DC980001063FF423AE4D4A967803F0FE030B705D
:10DCA800002E3FF41BAE4A4C22780B2A0DD80121D6
:10DCB800914040F603060E4041F0CD8311F4C06F49
:10DCC80003D0093A012A41F28E84DFF820A1414AA3
:10DCD800DAF8001051600B2203F001062270FDE50E
:10DCE8001AF4800F7FF426AE3B4C002284F8A02063
:10DCF800B8F1000F3FF430AE384A01211170002E00
:10DD08003FF43BAE1AF0100F3FF437AE344A1278A6
:10DD1800D2063FF532AE002F7FF42FAE002B7FF4F2
:10DD28002CAE1AF4800F7FF428AE2E4B1B78002BF4
:10DD380001F0A4832C4B9B78B8F1000F41F08B8441
:10DD48003BB12A4A2A4B12681B689B1A002BC1F266
:10DD58006684214C012384F8A1300EE6059B1B78CC
:10DD6800D9077FF529AF4FF40F7014F0B7FE0028DC
:10DD78003FF45BAF05F0B4FA4FF40F7014F044FEB3
:10DD880000283FF452AF05F0ABFA4FF40F7014F0CF
:10DD98003BFE0028EED148E73D51002054420020C8
:10DDA800623D002088590020CC4200203C5C0020C5
:10DDB800F0F70208FD4800208C2100203057002091
:10DDC800DC4C00207C3D0020FC480020D23600209E
:10DDD800CF36002060420020DC24002024210020CF
:10DDE80078480020F21C0020AC4200209C590020FA
:10DDF800283C00208C5900206C4D0020AC5F00208E
:10DE08000621CB48F3F74AFD3C88002800F07185CD
:10DE1800650640F196860721C548F3F73FFD0028BF
:10DE28003FF4A8AEC34AB2F90030002BB8BF5B423A
:10DE3800B3F5E17FBFF69EAEB2F90230002BB8BF52
:10DE48005B42B3F5E17FBFF695AEBB4B93ED096A34
:10DE5800D3ED076A93ED057AD3ED037A76EE866AF9
:10DE680077EE877A76EEA66AB7EE007A37EE666ABC
:10DE780077EEA77AB0EEC66AF0EEE75AB4EEE56A36
:10DE8800F1EE10FAB4BFB0EE655AB0EE465AB5EEF0
:10DE9800405AF1EE10FA40F06E879FEDA87AB4EE82
:10DEA800E56AF1EE10FA44BF9FEDA56A36EE477AAF
:10DEB800B7EE006AF4EEC66AF1EE10FAC8BFDFEDFD
:10DEC800A16AF5EEC07AC8BF36EEC77AF1EE10FA4D
:10DED80048BFB1EE477AF6EE007A27EE677ADFEDB3
:10DEE800987A77EE276ABDEEE66A16EE103A203386
:10DEF800402B41F28981DFED946A944ADFED927AF2
:10DF0800C2ED006AFDEEC76AC2ED017A16EE903ADC
:10DF18002033402BC2ED027A49D8DFED8A7AB4EE7D
:10DF2800E77AF1EE10FA41F3A5829FED896ADFEDF9
:10DF3800896A01E0B0EE677AB4EEE67AF1EE10FA9B
:10DF480077EE467AF6DC9FED847AF4EEC77AF1EE46
:10DF580010FA41F1AE829FED7E6ADFED806A01E042
:10DF6800F0EE477AF4EEE67AF1EE10FA37EE867ABA
:10DF7800F6D4DFED737AB4EEE77AF1EE10FA41F3F6
:10DF88008A81DFED707A37EEC77A27EE076ADFED10
:10DF9800745ADFED746ADFED747AE6EE256A67EE8F
:10DFA800065AE6EE267AA5EEA77AF0EE477AC2ED93
:10DFB800037ADFE5069B1B6899077FF5A8AD6B4FD1
:10DFC8003C8844F00104AFE5694B93F80090B9F13F
:10DFD800000F5FD1DFF8E081664E18F8030C357842
:10DFE8004146A8F103040AF031F8002800F0C8837C
:10DFF800002D40F01A8404F1080160790AF026F82F
:10E00800002841F0C8815C49A07A0AF01FF800286E
:10E0180000F0C983022D41F0AE815849E07B0AF037
:10E0280015F8002841F082815549207D0AF00EF844
:10E03800002800F0C983042D41F0A1815149607E78
:10E048000AF004F8002841F09E814F49A07F09F0AA
:10E05800FDFF002800F0C983062D41F098814B4947
:10E0680094F8230009F0F2FF002840F0138748498C
:10E0780094F8280009F0EAFF002800F0C983082D69
:10E0880040F01E87434994F82D0009F0DFFF00286F
:10E0980040F0C983404B01221A701CF069FF069BAF
:10E0A8001B685B077FF5D8AD032009F0F9FF00284E
:10E0B80000F0E6853B8813F008047FF4CDAD082016
:10E0C8001CF04EF83548364D3649374A374BBBF8C1
:10E0D800066000682E80086014601C6015B0BDE8FA
:10E0E800F08F334B1B7824F48074A4B2082B3C8047
:10E0F8007FF44FAD24F040043C804DE50BB901237B
:10E10800AB701B2009F0CCFF95F8214095F8203022
:10E11800284FDFF8A8808146A246052B00F20D8122
:10E12800DFE813F0CE00C3004E0007010901FD002F
:10E1380054420020D4510020C0000020A7DFA8349A
:10E14800DB0FC93FDB0F494000000000240000201E
:10E15800DB0FC940E4CB1641DB0F49C0E4CB16C145
:10E1680092E741B99730083C15A82ABE623D0020C5
:10E17800FD480020AE00002021270020262700208F
:10E188002B27002030270020352700203A270020A1
:10E198003F270020442700208C21002078210020E0
:10E1A80068210020742100206C21002064210020B7
:10E1B800CC420020EC27002017270020A03D00209B
:10E1C800BAF1010F04BF052385F820308EB1039BF7
:10E1D8003888B3F918100022134661F30F0361F36E
:10E1E8000F0260F31F4261F31F43CBF80420CBF802
:10E1F80000309D4C6A6923689A4280F0928447F205
:10E2080030520323EA6185F8203002201BF0B0FF6A
:10E218000DF0ECF92268EB6913440422AB6185F830
:10E228002020BAF1010F40F085852368AA699A4237
:10E2380080F083808D4B187818B909F031FF0028D9
:10E248007BD1D8F8003023F00203C8F800302268E8
:10E258007B88642101FB03234FF4806000222B613B
:10E2680085F82020EA701BF073FF95F8203054E7FA
:10E278001CF040FC012806D17B4C7B882268642175
:10E2880001FB03232B61B9F1000F02D0BB79002BEE
:10E2980047D1BAF1010F50D0734C2A6923689A42CA
:10E2A800C0F05285012385F82030BAF1010F36D02D
:10E2B800FB79012B68D004F0BFFA95F820302CE7E1
:10E2C800002ED5D14FF48060B9F1000F00F00E8315
:10E2D8001BF046FF059B1E7800232B61049BD3F897
:10E2E80000A01AF4805706F001063FF410AB1D2178
:10E2F8005F48F3F7D3FA00287FF409AB5D4B03F1CD
:10E30800500903E004334B4500F0D7841A78262AD5
:10E31800F8D19978DA789142F4D2FFF7FABA524CE8
:10E3280095E704F089FA03224FF47A7385F82020E0
:10E33800EB614D4C69E74C4C73E7059B1E7806F082
:10E348000106FFF7DDBA039A013BD27D3BF9133092
:10E35800002A40F0DC82A3F57A73B3F57A7FA8BF70
:10E368004FF47A7323EAE37307EE903A9FED427A0B
:10E37800F8EEE77A67EE877A404AFCEEE77A17EE1E
:10E38800903A1380FFF7B4BA04F056FA032240F625
:10E39800B83385F82020EB61334C36E7384F3B78AB
:10E3A800002B00F08587374BDFF8E080DFF8E0B01E
:10E3B800DFF8E0A0039345465E46049099460EE0D8
:10E3C80019F804109847032C28DC88B93B782AF8F8
:10E3D800020F01349C4205F1040580F2D280072C1B
:10E3E800E1B23046DBF80430EADD984700B2EDE7E9
:10E3F80038F824206B88801A4FF47A719B1A01FB35
:10E4080000F040F6CA0290FBF3F00844904240F254
:10E41800EE23A8BF10469842B8BF184600B2D5E709
:10E42800194C94F8AA3053B1059B1B78D90706D527
:10E43800039BBBF906205B8B9A4200F3CD84112124
:10E448000B48F3F72BFA002800F0668294F8AE30F8
:10E458002BB994F8A83013B93223A4F8AC300123AF
:10E4680084F8AE30FFF7E7BA9C590020F21C002070
:10E4780054420020D0420020AAF1823F603D002093
:10E488001D350020DC4C0020DC2400203035002025
:10E49800DC510020DA240020DFF8D8A2DFF8D88287
:10E4A800A44C1F460AF15A064FF0010951461AF8C2
:10E4B800010C09F0CBFDF8B19AF804009AF8023083
:10E4C8009AF803E000EB400104EB8101013BD1F82D
:10E4D800B42003EB4303434493420DD094F8E02067
:10E4E80081F8B0E009FA00F022EA0000C1F8B4307F
:10E4F800C1F8B87084F8E0000AF1060AB245D5D12F
:10E508008D498E4A8E4B8F4C09681B78D2F800A033
:10E5180008910793A4F1B0090026636853B31F78E4
:10E5280047B3A168AAEB010100290ADB99F8E010BA
:10E538000120B04021EA00010AF5FA7089F8E010DC
:10E54800A060079AB2B1217858780431C9B200287E
:10E5580040F0FD81039A3BF91110108B00F1C80EB1
:10E56800714540F3BE8399F8E0109B783141CA07A2
:10E5780040F18E840136042E04F10C04CDD1FFF74E
:10E58800BBBADDF81090704A704904921268A1FB7A
:10E59800091B42F2010A4FEA9B1112EA0A0A069184
:10E5A80000F0CC816A4D6B48654C6B492E78007839
:10E5B800267008701EB168490E7886F001065D4C19
:10E5C8000F2184F82410002B00F0C082634B039DB8
:10E5D8000D93B5F824E0B5F826C0039DCDF828C002
:10E5E80018462D8B00785E4B109594F825500E95A3
:10E5F800A3FB00535B0803EB4303C31ADBB2099385
:10E60800069BCDF814A002F4805203F5967397F890
:10E618000080DFF85CB1DFF864C1DDF838A00C9049
:10E628000B917546119204F1280000210793CDF84B
:10E638003C90A646002E00F0F1813EF911201FFA09
:10E6480082F9A9454FEA410303D30A9CA14540F248
:10E658002A825CF82120069C944280F0E9813BF9EB
:10E668000320059C002C40F0FD81013141452BF829
:10E67800032000F10600DDDB0B9A3A4B8EF82420CC
:10E688000F2A74460CBF01220022DDF83C9084F862
:10E6980025A01A7000F06182334D2E492E4ADFF80A
:10E6A8009CA0012304200B7013701BF061FDDAF8A5
:10E6B8000030A9686A68EB605B1A934284BF002344
:10E6C80085F821303C78049B1F68002C00F00F86E9
:10E6D800039A264EB2F824C0B2F818E0244917F479
:10E6E8008057304640F069823A460EE0437803EBA3
:10E6F800830303EB830303F2EE239BB20132A242AE
:10E7080021F8023B00F102000ED016F81230002B5F
:10E7180000F0CD81022BE9D001320B8821F8023BB1
:10E72800A24200F10200F0D10D9A13780133137060
:10E73800FFF7CCB8DC240020D45F00209C590020CF
:10E74800353D00208C25002030570020D34D621025
:10E75800C43300203001002031010020C9340020DA
:10E76800ABAAAAAA525200207C3D002064350020A2
:10E77800AC5F00202E26002094DF0208CC34002055
:10E7880008F10501607909F061FC00283FF43BAC11
:10E79800012D40F0008604F10D01A07A09F056FC25
:10E7A800002840F0E885CB49E07B09F04FFC0028C1
:10E7B8003FF43AAC032D40F0B985C749207D09F0F4
:10E7C80045FC002840F0DB85C449607E09F03EFC2A
:10E7D80000283FF43AAC052D40F0D585C049A07F0C
:10E7E80009F034FC002840F0D285BE4994F8230093
:10E7F80009F02CFC00283FF43AAC072D40F04A837E
:10E80800B94994F8280009F021FC002840F0588301
:10E81800B64994F82D0009F019FC00283FF43AACE9
:10E82800092D3FF437AC4FF009094B4635E3B04C9E
:10E83800D4F88830A9EB0303002BFFF659A8AD4A9A
:10E8480094F88C30517C089AC4F888200133AA4A7D
:10E85800039F32F81120B97D03F00F0384F88C3040
:10E86800234492B292FBF1F283F8902094F890102E
:10E8780094F8912094F8923094F89C000A4494F803
:10E888009310134494F89420194494F895300A444A
:10E8980094F89610134494F89720194494F89830F3
:10E8A8000A4494F89910134494F89A20194494F857
:10E8B8009B300A44134494F89D1094F89F20184400
:10E8C80094F89E3001440B441A4442F30B12642A14
:10E8D800F97DA8BF642213B209B1C2F1640307EE3F
:10E8E800903A9FED867AF8EEE77A43E51BF030FC24
:10E8F800F0E424F04004A4B23C80FFF78CBAA207ED
:10E908003FF516A944F002043C80FFF711B9C3F59E
:10E918003B6308331BB21EE594F8A830002B3FF484
:10E928008AA8059B1B7813F001037FF484A80122B1
:10E9380084F8A83084F8A920FFF77DB870490E78CC
:10E9480038E66B4C012284F8A020FFF7D5B90128DE
:10E9580000F0288499F8E0200123B34001361343DE
:10E96800042E89F8E03004F10C047FF4D6ADFFF7EB
:10E97800C3B8059B634A1B781060DB0700F13A8235
:10E9880094F8A61000297FF44DA8B4F9A430322BCE
:10E998007FF748A894F8A2200120572A84F8A600F7
:10E9A80000F0A984049B1B6813F0040302D05A2AC0
:10E9B80000F089855D2A00F02B855B2A00F03C85F4
:10E9C8005E2A00F04585562A00F04885972A00F00F
:10E9D8006485A72A40F0E3844B49049B0A781B68A6
:10E9E80042F004020A70494A069203F00403FFF752
:10E9F8001FB8B2F5FA7FFFF615A894F8A620002AEA
:10EA08007FF410A8059B1B780121DF0784F8A61066
:10EA180000F108850DF078F8FFF704B8002D40D014
:10EA28005CF82120069C94424FEA4103FFF417AE9C
:10EA3800374A374CD25C04EB0309002A00F0B18056
:10EA4800022A6BD199F8012002EB820202EB8202C2
:10EA580002F2EE2292B2032933DD059C12B2002C99
:10EA68003FF403AE099C20F81420BAF1000F03D13B
:10EA78000C9C022C7FF6F9ADB0F800A04288B0F8E3
:10EA8800049052449144234A0FFA89F982FB0942BF
:10EA9800214CA2EBE97224F8039012B24FF0010A5C
:10EAA800E3E52A464B00079C4CF82140D9E5D3B250
:10EAB800022B04D9032B7FF42FAE63461EE6734660
:10EAC8001CE6012404FA01F90B9C24EA090412B299
:10EAD8000B94C6E5262700202B270020302700208E
:10EAE800352700203A2700203F2700204427002010
:10EAF800DC240020645900208059002014AE2341F2
:10EB0800353D00202C3C002078480020A83E0020FD
:10EB180064350020565555554C2500203BF80320F8
:10EB280099E7C34B1B78002B7FF469AB002E3FF4A9
:10EB380066ABBAF1010F7FF400AC95F82030FFF70F
:10EB4800ECBA44F040043C80FFF765B9B94ABA4BC7
:10EB58000D92DFF838B301221A701B21B748F2F77B
:10EB68009DFE00287FF498ADB54DDFF8E4A2EA6871
:10EB7800DAF80030AB609B1AC82B00F2AA83049B1A
:10EB88001F6807F48057CFE53146AC48F2F786FE98
:10EB980000283FF4EEAE84F8A7600CF0B5FFFEF74E
:10EBA8003CBFCAB2022A40F2F682032AB6D1109AB2
:10EBB800119C002C08BF2A464DE700220FE043783D
:10EBC80003EB830303EB830303F2EE239BB20132CF
:10EBD800A24221F8023B00F102003FF4A5AD16F86D
:10EBE80012301BB1022BEAD00B88F0E7D3B2032B0B
:10EBF800FAD87346EBE7B2F5FA7FFEF613AF94F84E
:10EC0800A630002B7EF40EAF059E3378012113EA5F
:10EC1800010084F8A61000F04F838A4A927823F006
:10EC280001033370002A3EF4FDAE874C23780B2B8A
:10EC380018D801FA03F240F603010A427EF4F2AE54
:10EC480012F4C06F0ED0093B012B0BD8452017F0EA
:10EC580075FBFF2017F072FB7C4817F05BFB002068
:10EC680017F06CFB7A497B4A049B09681B68516062
:10EC78000B222270784A069203F00403FEF7D8BEEE
:10EC880008201BF065FAFEF7E7BF744A744910685C
:10EC9800B4F9A420C66981FB06018911F617701A18
:10ECA80000F5FF407F3082423EF7AAAE891B0A4436
:10ECB80012B2A4F8A420FEF7A3BE6A4A039BB2F8D6
:10ECC80006801B8BBBF90620A3EB08018A427FDD77
:10ECD80043449A42B4BF4FF000084FF00108FEF7D2
:10ECE80023BEC838814239DA99F8E0109B7831415F
:10ECF800C8073FF53FACC3F10008791E162900F29A
:10ED08001D81DFE811F0FC011002E2015A01240222
:10ED18003502CF01BC01A70192017D011B015A01F7
:10ED28006A013502CF01BC01460132011E010B0107
:10ED3800F500E10005992268EB690E781344AB6190
:10ED480006F00106FEF7DCBD03F076FD032240F66F
:10ED5800B83385F82020EB61FFF757BA99F8E0300F
:10ED68000122B24023EA02030AF5FA7289F8E03078
:10ED7800A260FFF7FFBBB4EEE56AF1EE10FA8CBFB4
:10ED8800B0EE654AB0EE464AC4EE054A9FED362A13
:10ED98009FED365ADFED361ADFED362A9FED363A0B
:10EDA800DFED363A9FED364AA4EE825AE4EEE12AC8
:10EDB800A4EE857AA4EEA23AB0EE475AB0EE637A92
:10EDC800A4EE837AA4EE874A84EE057AFFF767B843
:10EDD8004FF00108FEF7A8BD00211848F2F75EFDC4
:10EDE80000287FF42CAB322384F8AA00A4F8AC30B6
:10EDF800FFF725BB234B1B78002B3EF413AEEB78B3
:10EE0800002B7EF40FAE94F8A7300133DBB2032B4E
:10EE180084F8A7307EF606AE1B4B5B781BB9B8F1B9
:10EE2800000F7EF4FFAD0CF0E1FBFEF7F6BD00BF6E
:10EE380014210020C93400205252002054420020DE
:10EE48007C3D0020D2360020CF3600204C0303083A
:10EE58009C59002060420020A83E00204440002029
:10EE6800D34D6210D027002099FB243F69A2163E9B
:10EE780039094E3DE3B59E3E88FA163E45FE7F3F72
:10EE8800A7DFA834353D0020AC420020AC5F00204D
:10EE9800984632E74FF007094B4603EB83031C44BF
:10EEA80086F80090A17860780BF02CFB059BBB4A94
:10EEB8001B7801211170DA077FF5EFA8FEF7BFBEB6
:10EEC8004FF008094B46E8E7D9F8E400B44B90F84E
:10EED80036109A7841446429A8BF642121EAE17177
:10EEE80080F83610002A40F0A88307F077FB31E558
:10EEF800D9F8E400AA4B90F837109A784144FE29D3
:10EF0800A8BFFE2121EAE17180F83710002AECD071
:10EF180016201BF031FED9F8E400E6E7089AA04B6A
:10EF280051784144B1F5967FA8BF4FF4967121EA14
:10EF3800E17151709B78002B40F07983D9F8E40097
:10EF4800D3E7D9F8E4008178954B4144C829A8BF94
:10EF5800C82121EAE17181709B78002BC5D014206B
:10EF68001BF00AFED9F8E400BFE7D9F8E4004178BD
:10EF78008B4B4144C829A8BFC82121EAE1714170DF
:10EF88009B78002BB1D013201BF0F6FDD9F8E400D4
:10EF9800ABE7D9F8E4000178814B4144C829A8BF00
:10EFA800C82121EAE17101709B78002B9DD01220C5
:10EFB8001BF0E2FDD9F8E40097E7089A784B9179BD
:10EFC800987841446429A8BF642121EAE1719171CC
:10EFD800002840F03C830D2FB0D00898704B417941
:10EFE8009A7841446429A8BF642121EAE1714171FA
:10EFF800002AA3D00E201BF0BFFDD9F8E40074E767
:10F00800D9F8E400664B017A9A784144C829A8BF28
:10F01800C82121EAE1710172002A3FF466AF0B2092
:10F028001BF0AAFDD9F8E4005FE7D9F8E4005C4BCF
:10F03800C1799A784144C829A8BFC82121EAE17159
:10F04800C171002A3FF451AF0A201BF095FDD9F891
:10F05800E4004AE7D9F8E400514B81799A784144B1
:10F06800C829A8BFC82121EAE1718171002A3FF4AB
:10F078003CAF09201BF080FDD9F8E40035E7D9F84A
:10F08800E400474B41799B784144C829A8BFC8216F
:10F0980021EAE1714171002B40F0D382112F7FF4F6
:10F0A80052AF22E7D9F8E4003D4B01799B784144FF
:10F0B800C829A8BFC82121EAE1710171002B40F0DD
:10F0C800A282102F7FF453AF0FE7089A1179884472
:10F0D800B8F1640FA8BF4FF0640828EAE87882F80E
:10F0E80004801BF063FD2E4B9B78002B3FF426AF6A
:10F0F800032041461BF040FDD9F8E400F5E6089AE4
:10F10800274B11784144FA29A8BFFA2121EAE17175
:10F1180011709B78002B3FF411AF01201BF02CFDE0
:10F12800D9F8E400E1E6089A1D4B91784144642936
:10F13800A8BF642121EAE17191709B78002B3FF40C
:10F14800FDAE02201BF018FDD9F8E400CDE60898C2
:10F15800134BC1799A78414481F30801C171002A9F
:10F168003FF4ECAE05201BF007FDD9F8E400BCE63F
:10F17800D9F8E4000A4BC1789B784144C829A8BF54
:10F18800C82121EAE171C170002B40F042820F2FA3
:10F198007FF401AFA9E6109A5DE400BF8C2100203E
:10F1A800D23600203BF91110987840F63303994283
:10F1B800A8BF1946B1F5617FB8BF4FF461710C2F34
:10F1C800A1F561714FF4966393FBF0F391FBF3F1B2
:10F1D80000F0B080182F7FF4BDABD9F8E430C9B285
:10F1E800C82993F817E00846A8BFC82086453FF409
:10F1F800B1ABD14AD8759278002A3FF4ABAB384608
:10F208001BF0BAFCFFF7A6BBB4EEE77AF1EE10FAF2
:10F2180040F35681DFEDC95A9FEDC96A01E0F0EE6F
:10F22800676AF4EEC66AF1EE10FA76EEE57AF6DC75
:10F23800DFEDC46AF4EEE67AF1EE10FA40F13D81B2
:10F24800DFEDBE5A9FEDC06A01E0F0EE667AF4EE9B
:10F25800C67AF1EE10FA77EEA56AF6D4DFEDBB7A3E
:10F26800F4EEE76AF1EE10FA79DDDFEDB97A77EEC0
:10F27800E66A66EEA65A9FEDB75A9FEDB76ADFEDCC
:10F28800B77AA5EE856A26EEA55AE5EE867AE5EE0A
:10F29800276AFEF732BEDFEDB27AB4EEE77AF1EE16
:10F2A80010FA44BFDFEDA77A37EEC77AFEF76DBED6
:10F2B800AC4A0392FFF767B9049B84F8A600FA3AB0
:10F2C8001B68A4F8A420A84A069203F00403FEF7DA
:10F2D800AFBBA64A049B1F68136823F0040313609E
:10F2E800012307F4805785F82130FFF71DBA07F48A
:10F2F8008057FFF719BA9C4A9D4B069210461A6828
:10F308009C494FF47A73B3FBF2F3C3EB431203EB5C
:10F3180082030268DB005007A1F8B43000F18F8047
:10F32800049B1B6803F00403FEF782BB4FF003093C
:10F338004B46B2E5904B5B785FFA81F843453FF462
:10F3480009AB404603F042FD7B4B9B78002B3FF412
:10F3580001AB414638461BF00FFCFFF7FBBADFED67
:10F36800807AF4EEE76AF1EE10FA44BFDFED757AC1
:10F3780077EEE66A7DE74FF002094B468DE54FF0E0
:10F3880004094B4689E54FF005094B4685E54FF0E2
:10F3980006094B4681E54FF001094B467DE5002102
:10F3A800BB2A129100F0C280B72A00F0BB80BE2AA7
:10F3B80000F0BF80BD2A00F09480792A00F00C810B
:10F3C8007A2A00F002819E2A00F0F9809D2A00F036
:10F3D800EF80AE2A00F06C81AD2A00F06281EF2A3E
:10F3E80000F05C81FD2A00F05681FB2A00F0508174
:10F3F800FE2A00F04A81F72A00F039817B2A7EF440
:10F4080011AB4FF4FA61022003F006FCFEF70ABBC9
:10F418005A4A00215A48584C0260534A21700692B1
:10F42800FEF706BB049B57491B680A604E4A0692C2
:10F4380003F00403FEF7FCBA534A0121EAE7049BF0
:10F44800524A1B680A21118003F00403FEF7F0BA40
:10F458004F4A0221DEE70646FEF740BA09F0B0FE41
:10F46800F1F7E6FC09F094FE01F01EFA94F8A220E8
:10F47800FFF7ACBAF0EE477AFEF765BDB8F1000FBA
:10F488003EF467AC434C94F8A130002B3EF475AAC7
:10F49800002384F8A130FEF770BA049B3E4A1B682B
:10F4A8004FF4C8711180304A069203F00403FEF746
:10F4B800BFBAB0EE677AFEF75CBDF0EE676ACDE6DC
:10F4C800F0EE667AB4E694F8A820002A68D194F899
:10F4D800AA202549069182F0010284F8AA20FEF7A5
:10F4E800A7BA4FF6FE732D4A1F4896890690D08911
:10F4F800334401449381D18109F062FEF1F798FC0D
:10F5080009F046FE01F0D0F9049BB4F8A4201B686A
:10F51800FA3A0021A4F8A42003F0040384F8A61002
:10F52800FEF786BA0B464FF6FE71DCE70B46022162
:10F53800D9E70223D7E700BFD2360020DB0FC94046
:10F54800E4CB1641DB0F49C0E4CB16C1DB0FC93F42
:10F55800DB0F494092E741B99730083C15A82ABE0D
:10F56800DB0FC9BFDC4C0020A83E0020A03D0020D6
:10F57800205700209C54002058510020B23500200C
:10F58800645100202C3C002000360020F25F00204F
:10F598004E360020DC240020F45F00208C4200203E
:10F5A800474A84F8A81084F8A9000692FEF740BAE2
:10F5B8000021FF201DF002F894F8A22009E701209D
:10F5C8001CF0FCFF94F8A22000E73E4A137A43F0AF
:10F5D80001031372FEF726BA3A4A137A23F001039D
:10F5E8001372FEF71FBA452016F0A8FEFF2016F08A
:10F5F800A5FE354816F08EFE304616F09FFE059B98
:10F608001B78FEF762BB10201BF0B6FAD9F8E400AD
:10F6180057E50F201BF0B0FAD9F8E400B7E52B4CFA
:10F628000BF0E4FF002384F8A130FEF7A6B91520FB
:10F638001BF0A2FAD9F8E40057E417201BF09CFA53
:10F648007CE411201BF098FAD9F8E40026E50D2097
:10F658001BF092FABFE4002B3FF414AF1C491D4A7B
:10F6680009684FF47A7000FB031313600AE700215E
:10F67800042003F0D1FAB4F8A4300022963BA4F891
:10F68800A43084F8A620FEF7CDB900210320F0E7C6
:10F6980000210220EDE700210120EAE700210846C9
:10F6A800E7E7FF2100201CF089FF94F8A22096E6E6
:10F6B800012100201CF082FF94F8A2208CE600BFF4
:10F6C800A83E0020385200204C030308DC24002008
:10F6D8009C590020283C002038B50B4C23688BB17E
:10F6E8005A68821A002A054604DA0CE05A68AA1AEF
:10F6F800002A07DB9A68226018461A689047236830
:10F70800002BF3D138BD38BD603400200B4B0022EC
:10F7180010B4027203F164040121890742BF197908
:10F72800815401329C4203F1140303D0072A01DCFF
:10F738009979F2E75DF8044B704700BF3001030880
:10F7480024230370704700BF012210230270437006
:10F75800704700BF08B507F005F9024B024ADA60A6
:10F76800FEE700BF00ED00E00400FA052DE9F04FC8
:10F778002DED028BA0F10A0389B00C46E72B00F2AD
:10F788006686DFE813F01C016406640664066406F6
:10F798006406640664066406640664066406640611
:10F7A8006406640664066406640664066406640601
:10F7B800640664066406750564066406640639050D
:10F7C80064066406640656066406C2056406A9054E
:10F7D80064069D05640694056406300664061606EC
:10F7E8006406640664060F06070664063D0364069D
:10F7F8006406360364060E03640664066406FC02A7
:10F808006406640664066406DD026406FC00640699
:10F818003F046E01640664066406640664066406B2
:10F8280064062D01640611046406DD03640664039E
:10F838006406500364066406640664061605DB0461
:10F84800D404A304E800640664066102370264066F
:10F85800FF01E3016406640664066406D8016406D1
:10F868006406B701640664066406A8019101C9022A
:10F8780087026406640664067802640664068304E4
:10F888006406640664066406640664066406640620
:10F89800640664066406640664066406640616055F
:10F8A8006406640664066406640664066406640600
:10F8B80064066406640664066406640664066406F0
:10F8C80064066406640664066406640664066406E0
:10F8D80064066406640664066406640664066406D0
:10F8E80064066406640664066406640664066406C0
:10F8F80064066406640664066406640664066406B0
:10F90800640664066406640664066406640664069F
:10F91800640664066406640664066406640664068F
:10F92800640664066406640664066406640664067F
:10F93800640664066406640664066406640664066F
:10F94800640664066406640664066406640664065F
:10F95800640678044E04AD4E337853B1AC4F00259D
:10F9680037F8021F2046F1F7ADFC33780135AB427A
:10F97800F6DC012009B0BDEC028BBDE8F08FA34E88
:10F988003378002BF5D0A34F0025B846236817F825
:10F998001520591C21601A7098F8011001EB81019B
:10F9A80001EB810101F2EE2189B22046F1F78AFCD0
:10F9B80033780135AB4208F10208E7DCD9E7964D08
:10F9C80028461BF041FF0028D3DD2B46054422685A
:10F9D80013F8011B501C9D4220601170F7D1C8E735
:10F9E8000AF0A4FDFF28064600F0238608A9002592
:10F9F80001F8125D0DF10D008DF80D500AF076FD3D
:10FA080008A800F8115D0AF065FD08A800F8105D67
:10FA18000AF054FD08A820F8085D0AF043FD2368A1
:10FA28005A1C22601E7023689DF80D20591C216005
:10FA38001A7023689DF80E20591C21601A702368DB
:10FA48009DF80F20591C21601A7023689DF810201A
:10FA5800591C21601A702046BDF81810F1F732FCC5
:10FA680087E70B686D4E01255A1C0A601D700B68EC
:10FA7800B278591921601A700EF0A6F82368684AFE
:10FA880068495F1927601870B1F90010B2F90000D1
:10FA9800F1F7A2FD23685A192260187031882046B0
:10FAA800F1F710FC284665E70A685F4B5F4918784C
:10FAB800551C2560107022685878551C25601070F8
:10FAC80022689B78501C206013702046C988F1F783
:10FAD800F9FB01204EE7554D08462988F1F7F2FB5E
:10FAE80069882046F1F7EEFB2046A988F1F7EAFB82
:10FAF80001203FE74E4D05F16006A9882046F1F741
:10FB0800E1FBE9882046F1F7DDFB29892046F1F77A
:10FB1800D9FB2368AA7A591C21601A702368EA7AEB
:10FB2800591C21601A7055F80C1B2046F1F7B2FBDE
:10FB3800AE42E2D11DE73F4952232268501C2060A3
:10FB4800137011F8013F002BF7D112E73A48002350
:10FB58002268056803EB4301561C6D5C266015702E
:10FB6800026825680A446E1C527826602A7002686A
:10FB780025680A4401339278691C0A2B21602A708F
:10FB8800E6D1F6E62D4D0B682A68591C12782160DB
:10FB98001A702B6822689978531C2360002311700F
:10FBA8002A6821681A4401335279481C032B2060C3
:10FBB8000A70F5D123682A68591C127A21601A70D4
:10FBC80023682A68591CD27821601A7023682A6829
:10FBD800591C127921601A702B6820465989F1F74F
:10FBE80071FB2A682368527A591C21601A702A68A6
:10FBF80000F025BC124B08461968F1F74BFB114B76
:10FC080020461988F1F75EFB0120B3E6DC5100209D
:10FC1800AA5F00206435002068420020D236002008
:10FC2800E4400020E640002084420020D027002045
:10FC3800E82E0020DCDF020864510020D45F002099
:10FC48007821002014230020AB4D08462988F1F7BD
:10FC580039FB69882046F1F735FBB5F90430A74A26
:10FC6800D91782FB0323C1EBA301204689B2F1F720
:10FC780029FB01207EE6A24D0846298AF1F722FBDE
:10FC8800698A2046F1F71EFB2046A98AF1F71AFB7C
:10FC980001206FE6DFF8A4E20027FEB271460023D8
:10FCA8002268501C206016702268501C2060137057
:10FCB800226811F8010F0133551C062B25601070BE
:10FCC800EED10137062F0EF1060EE6D18D4900233D
:10FCD8002268501C206017702268501C2060137026
:10FCE800226811F8010F0133551C0B2B2560107089
:10FCF800EED12368844A581C0721206019702368B4
:10FD08000021581C20601970236892F8F020591CB3
:10FD1800216001201A702DE60B687C4A7C49107816
:10FD28007C4A5D1C2560187023688978581C2060FF
:10FD3800197023689278591C216001201A7019E6FD
:10FD48000B68754D591C2A7921601A7023686A79E5
:10FD5800591C21601A7029882046F1F7B3FA2368E4
:10FD6800AA79591C21601A7069882046F1F7AAFA05
:10FD78002368EA79591C216001201A70FAE50B689A
:10FD880000255A1C0A60204629461D70F1F782FAA0
:10FD980029462046F1F77EFA29462046F1F77AFAF5
:10FDA800E7E50B685D4A5E4D11785E4A581C206095
:10FDB800197011682046F1F76DFA23685A4A591CE0
:10FDC800127A21601A7029882046F1F77BFAA988EF
:10FDD8002046F1F777FA29892046F1F773FA0021CE
:10FDE8002046F1F76FFA20460021F1F76BFA01205F
:10FDF800C0E5084608224C49F1F734FA0120B9E574
:10FE08000B684A4A4A4990785D1C25601870236837
:10FE18005278581C20601A7023680A79591C21608E
:10FE280001201A70A6E50B68394A4249D078394A48
:10FE38005D1C2560187023684979581C206019706A
:10FE48002368D278591C216001201A7092E500219C
:10FE58002046F1F737FA00212046F1F733FA00215E
:10FE68002046F1F72FFA2368334D00265A1C2260EA
:10FE78001E7023682A68591C92F82C2021601A7079
:10FE880023682A68591C92F8362021601A70236862
:10FE98002A68591C92F8372021601A7023685A1C66
:10FEA80022601E7023685A1C22601E7023685A1C28
:10FEB80022601E702B682046598FF1F703FA2B68D1
:10FEC8002046198FF1F7FEF923682A68591C92F821
:10FED8002E2021601A7023685A1C22601E702B681D
:10FEE8002046598EF1F7EEF92B682046998EF1F7E6
:10FEF800E9F901203EE500BFD45100206766666637
:10FF0800704900201B3D0020383C00208854002008
:10FF18008C4200209C420020EC270020CC4200208C
:10FF2800CC2B002004370020DC4C0020AC42002001
:10FF3800C82400202040002064510020F73C002005
:10FF4800B54E0B687279B54D591C21601A702B6833
:10FF58002046198CF1F7B6F92B682046D98BF1F7B2
:10FF6800B1F971892046F1F7ADF9B1892046F1F769
:10FF7800A9F92B682046598CF1F7A4F92B6820467B
:10FF8800998CF1F79FF9F1892046F1F79BF9318AAD
:10FF98002046F1F797F92A68236892F82620591C19
:10FFA800216001201A70E5E49B4EF378002B00F0E5
:10FFB80032830B680822591C21601A7023680122B9
:10FFC800991821601A702368954D591C2A79216067
:10FFD8001A702368AA78591C21601A70298820464B
:10FFE800F1F770F9E9892046F1F76CF92368F2799D
:08FFF800591C21601A702368F6
:020000040801F1
:10000000EA78591C216001201A70B7E40B680025BA
:100010005A1C0A601D700B685A1C0A601D700B6820
:100020005A1C0A6029461D70B7E6804B03F1700523
:1000300022681978501C2060117022685978501C71
:100040002060117022689978501C2060117022681D
:10005000D978501C2060117022681979501C2060DA
:10006000117022685979501C2060117022689979AA
:100070000733501C9D4220601170D9D17DE46C4D36
:100080000846E989F1F722F92046A989F1F71EF916
:10009000012073E40B68674F591C3A7821601A708D
:1000A0003B78002B3FF469AC0025EEB2304619F0E6
:1000B00067F923684278591C216030461A7019F09C
:1000C0005FF901892046F1F701F93B780135AB4230
:1000D000EBDC52E4584D594E9FED598ADFF88C8184
:1000E000DFED588A05F120070EE0FCEEE77ACDED52
:1000F000017ABDF8041020460435F1F7E7F8AF4265
:1001000006F118063FF439AC717C0029F3D04E4B50
:10011000D5ED007A1B78012BE7D14C4B1B68DB0433
:1001200040F17582F5EE407AF1EE10FA40F09982D6
:1001300040F2DC51DFE7084610224549F1F796F816
:1001400001201BE4434B9B8AB3F5006F00F27382DE
:10015000B3F5806F00F28382B3F5007F34BF0127CF
:1001600002273D4D05F10C0655F8041B91FBF7F1F4
:10017000204689B2F1F7AAF8AE42F5D1374D384F93
:1001800005F10C06B5EC010AD7ED087A80EE270AD6
:100190001CF042FC81B22046F1F798F8AE42F1D152
:1001A000304D05F10C0655F8041B204689B2F1F7D5
:1001B0008DF8AE42F7D1FFF7E0BB00258146DFF8AE
:1001C000B080DFF8B0B0059504950695079501213C
:1001D0004FF6FF7A05E001350B2D00F03F8118F94D
:1001E000011F4F1C4AFA05F3F5D0DE07F3D5BBF823
:1001F00000302B41D807EED506A8F1F743FBEAE71C
:10020000194D08462988F1F761F8A9882046F1F7C9
:100210005DF820462989F1F759F80120FFF7AEBBB8
:10022000885400206451002070490020DC2F0020F9
:100230008C420020F05E0020B44000207058002066
:100240000000404200E082449449002030570020E2
:10025000A44000208C510020C451002024570020CD
:100260009C54002004280020CC2B0020DB9B9141D3
:100270000CE00208623D00209A4D05F150062878F6
:1002800014F086FB2368027A591C21601A702368D7
:100290006A78591C21601A702368AA78591C216059
:1002A0001A702368EA780435591CB54221601A7027
:1002B000E5D1FFF762BB0B688B4A591C527D216068
:1002C00001201A70FFF75ABB884D05F1800655F8DA
:1002D000041F2046F0F7E2FFAE42F8D1FFF74DBB16
:1002E000834D05F14006B5F880102046F0F7EEFF8B
:1002F000236895F88220591C21601A70236895F8AC
:1003000083200435591CB54221601A70EBD1FFF7E8
:1003100034BB754D0B682A7A591C21601A70A98B61
:100320002046F0F7D3FF298B2046F0F7CFFF698BEB
:100330002046F0F7CBFF2368EA7C591C21601A7035
:10034000A98C2046F0F7C2FFE98C2046F0F7BEFFEB
:100350002368AA7F591C21601A70236895F8202011
:10036000591C21601A70698C2046F0F7AFFF236892
:10037000EA7A591C21601A70E9682046F0F78EFF6E
:1003800023682A7C591C21601A70236895F8212063
:10039000591C216001201A70FFF7F0BA0B68012286
:1003A0009918216010461A70FFF7E8BA0846002134
:1003B000F0F774FF0120FFF7E1BA4E4D4E4E05F104
:1003C000180795F9023096F906209A4200F0FD8050
:1003D00096F90E209A4200F0F88096F916209A427B
:1003E00000F0F3800835BD42EBD1FFF7C6BA434BAE
:1003F00003F15A0522685979501C20601170226857
:100400001978501C2060117022685978501C2060A7
:10041000117022689978501C206011702268D97878
:10042000501C20601170226819790633501C9D42BF
:1004300020601170DED1FFF7A0BA0B68304A581C5B
:1004400011782060197023685278591C21600120AE
:100450001A70FFF793BA0020FFF790BADFF8ACA04C
:1004600000254FF028080135C5F1200208FA02F2F4
:10047000A5F120032AFA05F6164328FA03F31E43D2
:10048000272D06F001024FF000030BD01343EAD0F2
:10049000E8B207F009FE0028E5D0294606A8F1F7E2
:1004A000F1F9E0E7174B184E1B78DA0748BF069BB7
:1004B0004FF0000544BF43F0010306932F4602E0CE
:1004C0000135272D24D029463046F1F7EBF90028D5
:1004D000F6D0294606A8F1F7E5F9002840F0928009
:1004E0000137EDE7D0420020DC4C0020343C0020F6
:1004F000383C0020605B0020C04C00202D260020EE
:10050000CC420020FC4800200453002090E33FF43C
:10051000724B734DB3F850102046F0F7D7FE714B75
:100520001988204689B2F0F7D1FE6F4B19684B014C
:1005300003F02002C1F340031343C1F3800243EAF6
:100540004203C1F3C00243EA8203C1F3401243EA0B
:10055000C20301F0100119432046F0F7B7FE04A9C9
:1005600004222046F0F782FE236829785F4A581C4F
:100570002060197011886429A8BF64212046F0F713
:10058000A5FEB9F1960F5FD000212046F0F79EFE40
:100590002168B7F1190348BFA7F11203A3F3C403FD
:1005A0004A1C226020461A460B7005A9F0F75EFE31
:1005B00023684F4A581C1121206019702046116889
:1005C000F0F76CFE0120FFF7D9B92268511C2160B9
:1005D000137029882046F0F779FE2368EA78591CC1
:1005E00021601A7023682A79591C21601A702368C7
:1005F000AA79591C21601A7023686A79591C2160F4
:100600001A70EFE6394604A8F1F73CF968E7F4EE12
:10061000C87AF1EE10FA40DA4FF47A716BE50B68A4
:10062000B178344A581C2060197023681278591C1C
:1006300021601A70CBE4082793E523685A1C2260D6
:1006400001201E70FFF79AB923680322591C21600C
:100650001A7023686A78591C21601A7098E7042779
:100660007FE5F4EEC87AF1EE10FA3FF561ADF4EEF5
:10067000E87AFDEEE77AF1EE10FA17EE901A1ED83E
:100680006FF4F973303903FB01F140F2E73391FB6A
:10069000F3F101F2DB5189B22DE5FDEEE77A40F28C
:1006A000E73217EE903A303B02FB03F388FB03126C
:1006B000D917C1EB622101F2E93189B21BE540F2A1
:1006C000F313A1F5836103FB01F140F2E73391FBE2
:1006D000F3F101F2DD5189B20DE500BF9007002072
:1006E00058510020482C0020A83E00204C2C00200F
:1006F000A03D00208042002008B501210220FBF728
:1007000079FC094B1B7803F00503052B08D0002169
:100710000120FBF76FFC00210846FBF76BFCFEE7AE
:1007200006F0B6F9F3E700BF1C290020022810B438
:1007300028BF0220064C074B207000EB8001064AC0
:100740005DF8044BC0EBC10003EB40001060704744
:1007500058510020B23500206451002008B508F03F
:1007600033FDF0F769FBBDE8084008F015BD00BF98
:1007700038B5444B5A899989914224BF00225A8145
:10078000198ADA89914224BF0022DA81DA7892B399
:10079000072A30D03C493D4D91F8570001240021F3
:1007A0000A282C709C70D9713ED00C2866D0DFEDE1
:1007B000387A002A31D1374C9FED370AA2780029C8
:1007C00018BFF0EE407A062A9EBF344901EB820141
:1007D00091ED0F0A217959B3013A032A4DD8F7EE6A
:1007E000007A87EE800A1CF017F92388984228BF08
:1007F0001846208038BDD97921B198780428B8BF2F
:1008000004209870204890F857000A280CD00C2833
:10081000CDD1DFED237A002ACDD0072ACBD00A280C
:100820002CD1DFED207AC6E70A20DFED1F7AC0E782
:100830009B78164A07EE103A1178B8EEC77A27EE81
:10084000277A07EE901AF8EEE77A67EE877AB4EE29
:10085000E70AF1EE10FA10DDC0EE077AFDEEE77A56
:1008600017EE903A102BA8BF1023012BB8BF01231D
:10087000DBB28B4238BF0B46137038BDDFED0B7A0D
:1008800099E700BF885400209C540020804200203B
:100890006F120339704900206F120338DCDF020841
:1008A0000AD7A3390F506E3A5304E9386F12833ACE
:1008B0002DE9F047B54FB64E08F086FCBE421ED279
:1008C000DFF85483DFF854934446258862197DB1DC
:1008D0004A450DD2052D0BD933886188C3F30B032C
:1008E000994200F0F180144625886219002DEFD15D
:1008F000716830461436F0F72BFABE42E4D3A54AAD
:100900001378A3F1170102290FD9A34911F8330075
:10091000002840F00581D8000144497829B19F4959
:1009200011F83330002B00F029819D4B5A78022AB0
:1009300040F2F08000229B495A701A789A48022AA5
:10094000016000F2E38002EB8201984BC2EBC1022E
:1009500003EB4203998C5A8C954C9142236001D34E
:1009600000225A84934B9A78042A00F0FE8032B910
:100970001A88B2F5F07F84BF4FF4F0721A808E4D62
:10098000FFF7F6FE2B688D4A1A40002A00F0F98026
:10099000DE0700F1E580580400F1DD80190700F161
:1009A000D5809A0100F1CC809B0400F1C28011F047
:1009B000C9FB10B9824819F08BF84020F0F7FEF916
:1009C0008020F0F7FBF94FF40070F0F7F7F94FF4DF
:1009D0008020F0F7F3F94FF40010F0F7EFF94FF043
:1009E0008060F0F7EBF94FF00060F0F7E7F91AF0EC
:1009F000E1F80021302273481CF0CBFF206805F09D
:100A000095FC714B266803F1500102E004339942D2
:100A10007AD01A78002AF9D19C78D8788442F5D215
:100A20006A496B4B91F804E06A486B4D5C6B6B4B09
:100A30002860C827642111FB0E71DFF8E4E15960DA
:100A4000674F30F8061C674DAEF800100021996022
:100A5000D960196159619961D96183F8201083F8CF
:100A600021103A702E600CB10FF0A6FC5E4B9FED8A
:100A70005F5A1B885E4A9FED5F6A55795E4C5F49FD
:100A80005F48086006EE903AF8EEE66A1388C5EE15
:100A9000265A07EE103A53881279C4ED005A07EE31
:100AA000903AB8EEC77A574BF8EEE77A1D725A7251
:100AB00027EE067A67EE867ABDE8F04783ED017A85
:100AC000C3ED007A08F068BB63799B077FF40BAF36
:100AD000716894F804A03046F0F73AF93388BAEB1D
:100AE000133F04D01436BE42FFF4EEAE07E773881E
:100AF0007068AA1FC3F30B039A4204F10601A8BF52
:100B00001A461BF05DFEEDE7012289E700221A700C
:100B1000264B1FE7234902EB420201EB82010CE75F
:100B2000D8000C186468002C7FF4F6AE17241470FB
:100B3000F2E63548F0F742F94020F0F73FF936E7A2
:100B400046F20900F0F73AF92B682DE72F48F0F745
:100B500035F92B6825E72E48F0F730F92B681DE7AB
:100B60002C48F0F72BF92B6815E79A8AB2F57A7FB3
:100B7000BFF405AF4FF47A729A8200E7182313701E
:100B8000D3E643F400532B6002E700BF2836030886
:100B9000F0310308CC42002030FA02087CF202084F
:100BA0005851002068510020D45F0020B235002049
:100BB00064510020704900200437002009600002C1
:100BC000605B00208C250020D0420020EC27002014
:100BD0008C510020924200208C5200207C3D00204D
:100BE000F21C0020C025002084210020C0C9FB4841
:100BF000C824002017B7D1388821002014260020EF
:100C00003661023DF025002009400002016000022B
:100C1000092000020860000202F003080000040836
:100C2000D044002008B508F0CFFAF0F705F908F035
:100C3000B3FABDE808403BE638B50D4C0D4DAC426B
:100C400006D2616820461434F0F782F8AC42F8D33B
:100C5000F0F736FE084A094B094C14600022094996
:100C60001A705A7008480860BDE8384012F03EBC5F
:100C7000F031030828360308645100205851002041
:100C8000B2350020D45F00206851002008B5FFF77E
:100C9000D3FF08F099FAF0F7CFF8BDE8084008F064
:100CA0007BBA00BF30B4134B1B78012B17D040F236
:100CB0002E414FF4F07201230182028083700E4BAB
:100CC000C0F812304FF4E175292428211122122393
:100CD000C58144718171C271037230BC70474FF499
:100CE0007A744FF47A510422037104820180827075
:100CF000E5E700BFC4250020D007E8033D4B3E4A8E
:100D0000D3ED015A93ED036AD3ED027AD3ED006A75
:100D10002DED048B25EEA59A26EE060A39EE097A0A
:100D200030EE005A27EEA78A26EE861A65EEA71A3D
:100D300066EEA72A26EEA52A67EE867A65EE865A23
:100D4000B1EE477AF0EE004AF0EE470AF0EE458A3F
:100D5000E8EE640AE8EE248A37EE457A71EEC13A8D
:100D600031EE214A72EEA54A35EEE25A37EEC26AFA
:100D700066EEA66A33EEA33A74EE043A34EEA44A61
:100D800075EE054A36EE065A32EE276AC3ED046A5E
:100D9000F7EE006A37EE267A70EEA60A36EE066A9D
:100DA00076EEE86A83ED089A83ED0B8A83ED0D0AEF
:100DB00082ED057AC2ED090AC2ED016A83ED071AD8
:100DC000C3ED091A82ED023AC2ED043A83ED052A19
:100DD000C3ED062AC3ED0A5AC3ED0C7A82ED034A2D
:100DE000C2ED074A82ED065A82ED086ABDEC048B1B
:100DF000704700BFB0000020C42500202DE9F0415D
:100E0000084B094C1B6899072DED088B02D594F807
:100E100044305BB9BDEC088B0023A363E363236418
:100E2000BDE8F081A83E00208C510020F54DA16B5B
:100E3000AE6AD4F83CE0F44B276CA862861B01FB39
:100E400001F20EFB0E22A08A93ED017AD3ED027A15
:100E500093ED035ADFEDED6A9FEDED6A05EE906AC2
:100E600007FB07226423F8EE658A03FB02F300FB0D
:100E700000F093FBF0F3523B262B27EE267A67EE29
:100E8000A67A68EE868A65EE266A19D806EE10EA1A
:100E9000B8EEC65A06EE107A65EE054AF8EEC65A66
:100EA00006EE101AE5EEA54AB8EEC66A9FEDD94ADD
:100EB000E6EE064AF4EEC44AF1EE10FA00F3A98217
:100EC000DFEDD54AF0EE642AF0EE643AD5ED0B5A28
:100ED0009FEDD13AF4EEC35AF1EE10FA40F30884D4
:100EE00027EEA76A9FEDCD5AA6EEA66AA7EE076A7F
:100EF000B4EEC56AF1EE10FA00F1768295ED0E4A75
:100F000095ED0F6A95ED105ADFF85483D5ED0C5A24
:100F100098F80030DA0740F19783B7EE003A65EEB3
:100F2000835A76EE856A37EE047AE3EEA56ABC4F03
:100F300077EE867AB6EE006A28EE866AA2EEA57A89
:100F4000E4EEA57A26EE865AD7ED024A97ED003AEE
:100F5000D7ED013A97ED034A27EE067A67EE867AD7
:100F600025EE246A64EEE75AA7EE036AE3EEC75A59
:100F700067EE046A36EE236AF1EE452AA7EEC46AEC
:100F8000E7EE836AE2EE845A67EEA37A75EE835A3F
:100F9000E5EE037A76EEA46A26EE065AE2EEA36A3E
:100FA000A5EEA55A77EE847AA6EEA65AE7EE647A05
:100FB000B0EE457AA7EEA77AF7EE00BAB1EEC75ABF
:100FC0008BEE857A65EE875A26EE076A66EE876AAB
:100FD00067EE877AC7ED005A87ED016AC7ED026AAE
:100FE000C7ED037AFFF78AFE8E4B1B885B0640F144
:100FF0002F82D7ED109A97ED0F6AD7ED116AD7EDD2
:101000000E7A29EEA98A69EEA65AB0EE487AA6EEC3
:10101000067AE7EE865A77EE074A75EEA55A3BEE5A
:10102000E45AB0EEE54AB0EEC57AB4EEC47AF1EE19
:1010300010FAB4BFB0EE445AB0EE475AB5EE405A7B
:10104000F1EE10FA27EEA9AA27EEA69A66EE299AE3
:1010500026EE26BA66EEA6AA00F05B83B4EEC47A4A
:10106000F1EE10FA8CBFF0EE447AF0EE477AC7EE5C
:10107000856ADFED6D3ADFED6D7A9FED6D6A9FED6C
:101080006D5AE6EEE37ADFED6C3AA6EEA76ADFED85
:101090006B7AA6EE865AE6EEA37A9FED696AE6EED3
:1010A000A7BAA6EE856AF0EE6B7AC6EE2B6A654F9C
:1010B000B4EEC47AF1EE10FA48BFDFED637A9FED2B
:1010C000630A48BF77EEE66AF7EE007AF4EEE74A85
:1010D000F1EE10FAC8BFDFED637AF5EEC05AC8BF73
:1010E00077EEE66AF1EE10FA48BFF1EE666A26EE98
:1010F000800A1BF091FC7AEE4B7AB7EE005A77EE3D
:10110000A77ADFED534ADFED535A9FED536A9FED07
:10111000537A3880F0EEE76A35EE665AE6EEA45A66
:10112000B1EEC50AA6EEA56AF5EEC07AA6EE867AFD
:10113000F1EE10FA48BFDFED4B7A27EE007A9FED13
:10114000430A48BF37EEC77ADFED3F7A37EEC77AFA
:1011500038EE2A8A27EE000A1BF05EFC38EE088A79
:1011600079EE297AB7EE006A77EEA77A36EE487AFA
:10117000F0EEE76AB0EEC77AB4EEE67AF1EE10FA76
:10118000B4BFF0EE665AF0EE475AF5EE405AF1EE73
:1011900010FA788000F0BA82B4EEE67AF1EE10FA36
:1011A0008CBFF0EE664AF0EE474A84EEA55ADFEDBA
:1011B000222ADFED225A9FED1C2A9FED1C3ADFED1B
:1011C0001C3A9FED1C4ADFED1E4AE5EE225AA5EEC1
:1011D000423AA5EE256AE5EE033AF0EE465AB0EE45
:1011E000446AA5EE236AE5EE064A84EEA56AB4EEEB
:1011F000E67AF1EE10FA48BF9FED137A9FED130ADD
:1012000032E000BFC42500202057002035FA8E3C74
:10121000BD3786350AD7233C00000000E68AF93D39
:10122000B0000020623D002039094E3DE3B59E3EEE
:1012300088FA163E45FE7F3F99FB243F69A2163E81
:10124000A7DFA834D4510020DB0FC93F4C3D0F4429
:10125000306E99BC2716983D843459BEA40DC93F01
:10126000FC480020DB0F494048BF37EE466AB7EE26
:10127000007AB4EEC78AF1EE10FAC8BF1FED077A04
:10128000F5EEC07AC8BF37EE466AF1EE10FA48BFF5
:10129000B1EE466A26EE400A1BF0BEFBD5ED099A78
:1012A000D5ED01AA95ED04BA95ED07AA95ED088A4A
:1012B00000B2B88094ED107AD5ED117A95ED069ACA
:1012C000D4ED0F6AE74A95ED030A137895ED026AAB
:1012D000B8EEC77AF8EEE66AF4EEE97A27EE099AF4
:1012E000D5ED057AA6EEA79A0028B8BF00F5616093
:1012F000D4ED0E7AB8BFB880F8EEE77A26EE888A89
:1013000027EE000AF1EE10FA4CBF43F0080303F099
:10131000F703A7EE8A8A137095F83430A7EE8B9AFC
:10132000012BA6EE860AA7EE298AB1EE499AA7EE0E
:10133000AA0A00F0B981A38A07EE903AF8EEE77A9C
:1013400038EE678A95ED147AD5ED137A38EE877A00
:1013500038EE678AC8EE876AE6EE887AB0EE678A6A
:10136000C5ED137A1BF058FB95F8364080EAE07320
:10137000A3EBE0739C4200F36381002840F3DA8121
:10138000001B6B6DB0EE490A184468651BF044FB06
:1013900080EAE073A3EBE0739C4200F353810028E2
:1013A00040F3C481001BAB6DB0EE480A1844A86539
:1013B0001BF032FB95F8373080EAE072A2EBE07266
:1013C000934200F33B81002840F3AC81C01A05F141
:1013D0005C010EC9BDEC088B014432440133E96560
:1013E0002A666B66BDE8F08168EEA55A95ED0E4A57
:1013F00095ED0F6A95ED105AA2EEA54AA4EEA56AE6
:10140000A3EEA55A85ED0E4A85ED0F6A85ED105ABB
:101410007AE5B1EEE44AF7EE003AC3EE844A95ED80
:10142000092A95ED084A95ED073A25EE245A65EE0E
:10143000A45A26EE246A64EE652A62EE464A63EEFA
:10144000453AE5EE022AE5EE834AE6EE043A3DE54A
:1014500095ED088AD5ED099AB0EEC87AF0EEE96A02
:10146000F4EEC76AF1EE10FAB4BFF0EE477AF0EE90
:10147000667AF5EE407AF1EE10FA00F05081F4EE63
:10148000C76AF1EE10FA8CBFF0EE475AF0EE665ADA
:1014900085EEA76A9FED743A9FED744ADFED744ABA
:1014A0009FED745ADFED743ADFED747ADFED7D5A0B
:1014B000A6EE434AE6EE237AE6EE044AE6EE27BAC3
:1014C000A6EE245AF0EE6B7AE6EE055A85EEAB6A8C
:1014D0006B4FF4EEC76AF1EE10FA48BFDFED697AA0
:1014E0009FED690AF5EEC09A48BF37EEC66AF1EE85
:1014F00010FA48BFDFED657AB5EEC08A48BF37EE17
:10150000C66AF1EE10FA48BFB1EE466A26EE000A4E
:101510001BF082FA95ED07AA9FED5D5A9FED5D6A7B
:10152000DFED5D6ADFED5D7A3880B0EECA7AF7EE06
:10153000005A75EEC75AA7EE056AB1EEE50AE7EE66
:10154000066AB5EEC0AAE7EE267AF1EE10FAC8BF39
:101550009FED4E7A67EE807A9FED4B0AC8BF77EE1B
:10156000677A9FED487A77EE677A27EE800A1BF05C
:1015700053FA95ED04BAD5ED01AA7880F0EECB7A56
:10158000B0EEEA7AB4EEE77AF1EE10FAB4BFB0EE5C
:10159000676AB0EE476AB5EE406AF1EE10FA00F005
:1015A000BB80B4EEE77AF1EE10FA8CBFF0EE675A2A
:1015B000F0EE475AC5EE866A9FED2B3A9FED2B6AF7
:1015C0009FED2B4A9FED2B5ADFED2B3ADFED2B4A97
:1015D000DFED345AA6EEC36AE6EEA34AA6EE864ACB
:1015E000B7EE006AA6EE845AA6EEA46AE6EE855A25
:1015F000C5EE866AB4EEE77AF1EE10FA48BFDFED89
:10160000217A9FED210AF5EEC0AA48BF77EEE66A7F
:10161000F1EE10FA48BFDFED1D7AB5EEC0BA48BF53
:1016200077EEE66AF1EE10FA48BFF1EE666A26EE52
:10163000C00A1BF0F1F900B2B8803BE60020C6E614
:1016400000209EE60020AEE6154B1A6844F61F63A4
:101650009A42B7EE003AB2EE042A98BFB0EE423A90
:101660005DE400BF7848002039094E3DE3B59E3E59
:1016700088FA163E45FE7F3F99FB243F69A2163E3D
:10168000D4510020DB0FC93F4C3D0F44DB0F4940D4
:10169000306E99BC2716983D843459BEA40DC93FBD
:1016A0009C590020A7DFA83498F8003013F0010FF0
:1016B000AB6C12D1002B1A46B8BF03F13F02A3EB6B
:1016C000A21307EE903AF8EEE77A77EE887AFDEE0D
:1016D000E77A17EE903AC5ED127A002BB8BF3F3388
:1016E0009B1107EE903AF8EEE77A38EE678A29E622
:1016F000B0EE435AB0EE436AB0EE434A85ED0E3A7F
:1017000085ED0F3A85ED103AFFF7FEBB1FED1B6A22
:101710006DE55FED1C6ACAE45FED1E6A6AE71FEDC6
:101720001F6AD5E63FF453AE184450E63FF43BAE93
:10173000204438E63FF425AE204422E638B5064D75
:10174000002455F83400013405F048FB05F0C7FBD0
:10175000222CF6D138BD00BF34E002087FB5094B1A
:101760000493094B0393094B0293094B0193094BD3
:101770000093094A094B0A490A4805F03BFC07B0A7
:101780005DF804FB370503083C050308440503081E
:101790004D05030859050308F40403085D510020B2
:1017A000010503080C05030838B50B4B03EBC00417
:1017B0000D4694F8D421094803EB8203D3F81011A5
:1017C00005F0EDFA94F8DA312BB1691C0448BDE854
:1017D000384005F0E4BA38BD34E002087A0E030858
:1017E000652003082DE9F04F324C87B00746324A96
:1017F0002378608802EB8303D3F81081EFF7CCFAEB
:101800002E4BD0F804A093F868308268A3B1D34679
:10181000924607F0400301260593A379002B06F1B9
:10182000FF3208BF0123934208DC254B08349C4259
:10183000DDD107B0BDE8F08F9B46EAE7A3881344EB
:101840001AF803501BF80330EA1AD2F1000949EBE9
:10185000020993B9009643461A4A4946384605F0AC
:101860001BFCC5B9059B33B900964346154A49464A
:10187000384605F027FC0136CFE703F00F021B09BD
:10188000403302920193009643460F4A4946384638
:1018900005F002FCE5E705F00F032D094035029342
:1018A000019500964346084A4946384605F00AFC29
:1018B000E1E700BF08E2020834E00208C425002086
:1018C000B0E202085F050308730503082DE9F04F35
:1018D0000E4691B0C349044603F026FA0546002897
:1018E00040F04582C049204603F01EFA0546002814
:1018F00040F03F82BD49204603F016FA0546002815
:1019000040F039822046BA4903F00EFA0028054615
:1019100012BF0824254601240EB144F01004B54E30
:10192000B54FBE42C0F02982B44B012283F8682033
:10193000FFF782F9EFF7C4FFB149284603F0F4F945
:1019400008B144F0200414F0090F00F0F7810020E2
:10195000FFF704FF04F01803182B04D1A94805F081
:101960003DFA05F0BCFAA84BA84F1A78A84EDFF84C
:1019700020B3002AA74A06BF012113460021A64A28
:10198000204605F09FFB2046FFF72CFFA34B3D7838
:101990001B78A34AA5EB0308D8F1000506EB8303E7
:1019A00045EB08052946D3F87832204605F074FB4C
:1019B0003B789B4A06EB830329469A4DD3F878324D
:1019C000204605F07FFBD5ED007A974AF5EE407A88
:1019D000F1EE10FA0CBF01210021204605F072FB48
:1019E0002A469249924D204605F040FD914A92497F
:1019F000204605F079FB95F90210904AB1FA81F181
:101A00004909204605F05EFB2A468D49204603F031
:101A1000A9F98C4BD3F800808B4BD3F800900027AA
:101A200006F53A7656F82750002D40F0AD81DFF8E4
:101A300064A22E4669EA080B844B53F82650002D09
:101A400040F0C2818248834FDFF84CE201262B5CD4
:101A5000EA5D10A919440DF1400C01F8202C15F88D
:101A60000E108C440CF8102C2EB1A3EB010CDCF101
:101A7000000646EB0C060135082DE8D10CAB764A82
:101A8000764DDFF818B231464FF0000820468DF849
:101A9000288005F001FB08AB6F4A3146204605F06F
:101AA00011FB6F4A6F49204605F0D0FD6E4A6F4921
:101AB000204605F067FC6E4A6E49204605F026FC7C
:101AC000694A6A49204605F0A7FB6B4A6B492046E4
:101AD00005F036FE6A4A204602F15A0105F054FD2F
:101AE000684A6949204605F087FC05F133074FF045
:101AF000190A2B783A78797893423B7940F08581BE
:101B00006878884240F08181AE78B878864240F0AB
:101B10007C81EE78F878864240F077812E79F01A51
:101B2000464246414FF461791AFB03930493FB78D4
:101B30001AFB03930393BB780293019143460092EF
:101B400031465A46204605F0A7FA2B791AFB039333
:101B50000493EB781AFB03930393AB7802936B78AF
:101B6000019315F8053B00935A46434631462046FB
:101B700008F1010805F0A6FAB8F10A0F07F1050708
:101B8000B7D1DFF81C91DFF81CB1012700256B00ED
:101B9000079319F815201BF815309A4240F0378149
:101BA00017F8096017F80B10711A4E424E41022ABD
:101BB000DFF85C8040F02D811BF8072043444FF094
:101BC000190A40F2EE211AFB021293F864330192D3
:101BD00000932E4A2B463146204605F05DFA17F851
:101BE000093061E08905030890050308980503089A
:101BF0009E050308F031030828360308C425002099
